:100000000C942B160C9458160C9458160C945816E5
:100010000C9458160C9458160C9458160C945816A8
:100020000C9458160C9458160C9458160C94581698
:100030000C9458160D949E060C9458160C94581651
:100040000C9458160C94366A0C9458160C94581646
:100050000C9458160C944E670C9451690D943E0301
:100060000C9458160C94A2670C94CC670C945816F8
:100070000C9458160C9458160C9458160C94581648
:100080000C9458160C9458160C9458160C94581638
:100090000C9458160C9458160C9458160C94581628
:1000A0000C9458160C9458160C9458160C94581618
:1000B0000C9458160C9458160C9458160C94581608
:1000C0000C9458160C9458160C9458160C945816F8
:1000D0000C9458160C9458160C9458160C945816E8
:1000E0000C9458163DD8DDD87BD9DFDAF0EAF0EA77
:1000F000F0EAF0EAF0EAF0EAF0EAF0EAF0EA1ADA16
:100100005BDA9CDAF0EAF0EAF0EAF0EAF0EAF0EA28
:10011000F0EAF0EAF0EAF0EAF0EAD1DD32DE93DE6E
:10012000F4DE55DFB6DF17E0F0EAAAE49BE013E166
:100130008BE103E27BE2F2E266E3D2E33EE4F0EA43
:10014000F0EAF0EAF0EAF0EAA2DC07DDF0EA00E526
:100150007FE5FBE57AE6A8E604E741E77EE7E9E725
:1001600058E8C5E832E964E9D6E614EAF0EAF0EACC
:10017000F0EAF0EAF0EAF0EAF0EAF0EAF0EAF0EAAF
:10018000F0EA3CDC6EDCF0EAF0EAF0EAF0EAF0EAF1
:10019000F0EAF0EAF0EA83EAF0EAC9DCF0EAF0EA31
:1001A000F0EA9DE9DBE9F0EAF0EAF0EAF0EA2FD8BC
:1001B000F0EAF0EA21DBCFDB1CDC6CDD084AD73B40
:1001C0003BCE016E84BCBFFDC12F3D6C74319ABD26
:1001D00056833DDA3D00C77F11BED9E4BB4C3E914A
:1001E0006BAAAABE000000803F05A84CCDB2D44E39
:1001F000B93836A9020C50B9918688083CA6AAAA3B
:100200002ABE000000803F000001003600370026B3
:1002100000030002003C003D0038000E000F002EDD
:100220000030003E00120013000D000C000A000810
:100230000009001A001C0018000D000E00350053C4
:100240006574204D6963726F7374657070696E6751
:100250000048656174696E672042656400486561A5
:1002600074696E67204578747275646572004649DA
:10027000524D574152455F4E414D453A526570656A
:10028000746965725F302E3931204649524D5741AD
:1002900052455F55524C3A68747470733A2F2F6709
:1002A00069746875622E636F6D2F7265706574690D
:1002B00065722F52657065746965722D4669726D3D
:1002C000776172652F2050524F544F434F4C5F5609
:1002D000455253494F4E3A312E30204D4143484903
:1002E0004E455F545950453A44656C7461204558F9
:1002F0005452554445525F434F554E543A31205263
:10030000455045544945525F50524F544F434F4C0E
:100310003A320044656275673A006F6B000D0A005F
:100320004E414E00494E46004572726F723A004986
:100330006E666F3A005761726E696E673A00526579
:1003400073656E643A004563686F3A006F6B200016
:1003500057726F6E6720636865636B73756D004DD0
:10036000697373696E6720636865636B73756D008D
:10037000466F726D6174206572726F7200446F6EA9
:1003800065207072696E74696E672066696C6500BD
:10039000205800205900205A002045002046002007
:1003A0005300205000204900204A002052005344AE
:1003B0002072656164206572726F72004572726F9F
:1003C000723A6578706563746564206C696E652047
:1003D0000020676F742000736B69702000424C4BE3
:1003E0002000737461727400506F776572557000ED
:1003F00045787465726E616C205265736574004255
:10040000726F776E206F7574205265736574005734
:1004100061746368646F6720526573657400536F1D
:1004200066747761726520526573657400556E6BF2
:100430006E6F776E20636F6D6D616E643A00467209
:1004400065652052414D3A00583A0020583A002044
:10045000593A00205A3A0020453A00543A002042C6
:100460003A0020403A002054002040002042403A08
:100470000020524157003A002F00202F0053706592
:1004800065644D756C7469706C793A00466C6F7771
:100490004D756C7469706C793A0046616E73706565
:1004A00065643A005072696E7465642066696C61B7
:1004B0006D656E743A005072696E74696E6720746F
:1004C000696D653A006D2000206461797320002019
:1004D000686F7572732000206D696E00496E7661D9
:1004E0006C696420617263002C002000593A005A44
:1004F0003A0045303A0045313A004D53312C4D53C6
:10050000322050696E7300536574206F7574707576
:1005100074200020746F20004820004C2000785F79
:100520006D696E3A00785F6D61783A00795F6D6948
:100530006E3A00795F6D61783A007A5F6D696E3A64
:10054000007A5F6D61783A004A65726B3A00205A12
:100550004A65726B3A00206C696E65617220737433
:100560006570733A0020717561647261746963200B
:1005700073746570733A002C2073706565643D0078
:10058000454550524F4D2075706461746564006C30
:10059000696E656172204C3A002071756164726108
:1005A000746963204B3A004D6561737572656D65C2
:1005B0006E742072657365742E004D65617375727B
:1005C000652F64656C7461202853746570732920ED
:1005D0003D004D6561737572652F64656C746120B3
:1005E0003D004D65617375726564206F726967695E
:1005F0006E207365742E204D6561737572656D652F
:100600006E742072657365742E004F726967696E2F
:10061000206D6561737572656D656E742063616EC2
:100620006E6F74206265207365742E20205573658B
:10063000206F6E6C79205A2D436172746573696105
:100640006E20287374726169676874207570206108
:100650006E6420646F776E29206D6F76656D656EB0
:10066000747320616E642074727920616761696EB1
:100670002E00496E76616C69642064656C7461203B
:10068000636F6F7264696E617465202D206D6F7683
:10069000652069676E6F726564004C6576656C698C
:1006A0006E672063616C633A00546F776572203126
:1006B0003A00546F77657220323A00546F77657252
:1006C00020333A00416C7068612041283231302972
:1006D0003A00416C706861204228333330293A0077
:1006E000416C7068612043283930293A0044656CB8
:1006F00074612052616469757320412830293A0081
:1007000044656C74612052616469757320422830BD
:10071000293A0044656C74612052616469757320E4
:10072000432830293A004E6F206D6F766520696E40
:100730002064656C7461207365676D656E742077E5
:10074000697468203E2031207365676D656E742E74
:1007500020546869732073686F756C64206E6576C9
:1007600065722068617070656E20616E64206D61D5
:100770007920636175736520612070726F626C65AA
:100780006D2100546172676574457874720054611C
:10079000726765744265643A00504944204175743B
:1007A0006F74756E65207374617274002062696184
:1007B000733A200020643A2000206D696E3A2000D0
:1007C000206D61783A2000204B753A200020547546
:1007D0003A200020436C61737369632050494400E0
:1007E000204B703A2000204B693A2000204B643A9D
:1007F0002000504944204175746F74756E65206601
:1008000061696C6564212054656D706572617475F1
:10081000726520746F206869676800504944204100
:1008200075746F74756E65206661696C65642120EE
:1008300074696D656F757400504944204175746F1B
:1008400074756E652066696E697368656420212021
:10085000506C61636520746865204B702C204B6977
:1008600020616E64204B6420636F6E7374616E74DC
:100870007320696E2074686520436F6E66696775C2
:10088000726174696F6E2E68206F722045455052F8
:100890004F4D004D54454D503A0068656174656494
:1008A0002062656400657874727564657220003A30
:1008B0002074656D702073656E736F722064656659
:1008C000656374003A20776F726B696E67005072CF
:1008D000696E7465722073657420696E746F20642C
:1008E00072792072756E206D6F646520756E746903
:1008F0006C207265737461727421005A2D70726F6E
:1009000062653A005A2D70726F6265206176657279
:10091000616765206865696768743A005265736548
:1009200074205A20686569676874005A2D70726F68
:1009300062652073746174653A0047312058302035
:100940005930205A32300000486974207A2D707274
:100950006F6265004175746F6C6576656C206D61C2
:1009600074726978207265736574005A2D70726FA5
:1009700062652064697374616E63653A00417574E1
:100980006F6C6576656C696E6720656E61626C651B
:1009900064004175746F6C6576656C696E67206480
:1009A000697361626C6564005A2D70726F626520B4
:1009B0006661696C6564005A2D70726F6265206DA6
:1009C00061783A005072696E746572206865696773
:1009D00068743A0077616974005A2D70726F6265AD
:1009E00020686569676874205B6D6D5D004D617896
:1009F0002E207A2D70726F6265202D206265642032
:100A0000646973742E205B6D6D5D005A2D70726F7A
:100A10006265206F66667365742078205B6D6D5D1E
:100A2000005A2D70726F6265206F66667365742060
:100A300079205B6D6D5D005A2D70726F6265207359
:100A400070656564205B6D6D2F735D005A2D70724B
:100A50006F626520782D792D7370656564205B6DFC
:100A60006D2F735D005A2D70726F626520583100D2
:100A70005A2D70726F6265205931005A2D70726F55
:100A80006265205832005A2D70726F6265205932AB
:100A9000005A2D70726F6265205833005A2D7072A3
:100AA0006F6265205933004175746F6C6576656CB3
:100AB000206163746976652028312F302900436FE7
:100AC0006E66696775726174696F6E2073746F7298
:100AD000656420746F20454550524F4D2E00436F82
:100AE0006E66696775726174696F6E206C6F6164A0
:100AF00065642066726F6D20454550524F4D2E0043
:100B0000436F6E66696775726174696F6E20726596
:100B100073657420746F2064656661756C74732EE0
:100B20000050726F746F636F6C2076657273696FBB
:100B30006E206368616E6765642C207570677261F2
:100B400064696E6700457874722E004550523A30E1
:100B500020004550523A3120004550523A32200090
:100B60004550523A332000426175647261746500E9
:100B700046696C616D656E74207072696E7465642F
:100B8000205B6D5D005072696E74657220616374E4
:100B9000697665205B735D004D61782E20696E611A
:100BA00063746976652074696D65205B6D732C30A4
:100BB0003D6F66665D0053746F702073746570706E
:100BC000657220616674657220696E61637469760E
:100BD000697479205B6D732C303D6F66665D0058DB
:100BE00020686F6D6520706F73205B6D6D5D0059BF
:100BF00020686F6D6520706F73205B6D6D5D005AAE
:100C000020686F6D6520706F73205B6D6D5D00589F
:100C1000206D6178206C656E677468205B6D6D5D1A
:100C20000059206D6178206C656E677468205B6D7B
:100C30006D5D005A206D6178206C656E6774682068
:100C40005B6D6D5D0058206261636B6C6173682041
:100C50005B6D6D5D0059206261636B6C6173682030
:100C60005B6D6D5D005A206261636B6C617368201F
:100C70005B6D6D5D004D61782E206A65726B205B47
:100C80006D6D2F735D00416363656C65726174699E
:100C90006F6E205B6D6D2F735E325D0054726176F6
:100CA000656C20616363656C65726174696F6E2049
:100CB0005B6D6D2F735E325D0053746570732070D1
:100CC0006572206D6D004D61782E206665656472D9
:100CD000617465205B6D6D2F735D00486F6D696E8B
:100CE00067206665656472617465205B6D6D2F7346
:100CF0005D00446961676F6E616C20726F64206C87
:100D0000656E677468205B6D6D5D00486F72697A0F
:100D10006F6E74616C20726164697573205B6D6DB8
:100D20005D005365676D656E74732F7320666F7217
:100D3000207072696E74696E67005365676D656EC9
:100D400074732F7320666F722074726176656C0005
:100D5000546F776572205820656E6473746F7020CD
:100D60006F6666736574205B73746570735D0054A1
:100D70006F776572205920656E6473746F70206F91
:100D80006666736574205B73746570735D00546F81
:100D9000776572205A20656E6473746F70206F6679
:100DA00066736574205B73746570735D004D617864
:100DB0002E20726164697573205B6D6D5D00436FF9
:100DC00072722E20646961676F6E616C2041205BD6
:100DD0006D6D5D00436F72722E20646961676F6E86
:100DE000616C2042205B6D6D5D00436F72722E203E
:100DF000646961676F6E616C2043205B6D6D5D009F
:100E00004F5053206F7065726174696F6E206D6F03
:100E10006465205B303D4F66662C313D436C6173E9
:100E20007369632C323D466173745D004F505320EB
:100E30006D6F766520616674657220782520726515
:100E40007472616374205B255D004F5053206D699F
:100E50006E2E2064697374616E636520666F722004
:100E600066696C2E2072657472616374696F6E209E
:100E70005B6D6D5D004F50532072657472616374D9
:100E8000696F6E206C656E677468205B6D6D5D00C8
:100E90004F50532072657472616374696F6E206283
:100EA00061636B6C617368205B6D6D5D00426564AE
:100EB0002048656174204D616E61676572205B300A
:100EC0002D335D0042656420504944206472697688
:100ED00065206D6178004265642050494420647249
:100EE000697665206D696E00426564205049442032
:100EF000502D6761696E0042656420504944204965
:100F00002D6761696E004265642050494420442D7C
:100F10006761696E0042656420504944206D6178C4
:100F20002076616C7565205B302D3235355D007340
:100F30007465707320706572206D6D006D61782E20
:100F4000206665656472617465205B6D6D2F735DED
:100F500000737461727420666565647261746520E3
:100F60005B6D6D2F735D00616363656C65726174A9
:100F7000696F6E205B6D6D2F735E325D0068656119
:100F800074206D616E61676572205B302D335D008A
:100F9000504944206472697665206D61780050493B
:100FA00044206472697665206D696E005049442062
:100FB000502D6761696E2F646561642D74696D657C
:100FC0000050494420492D6761696E005049442012
:100FD000442D6761696E00504944206D6178207628
:100FE000616C7565205B302D3235355D00582D6F95
:100FF0006666736574205B73746570735D00592D4C
:101000006F6666736574205B73746570735D0074DE
:10101000656D702E2073746162696C697A652074E5
:10102000696D65205B735D0074656D702E20666F61
:10103000722072657472616374696F6E207768657F
:101040006E2068656174696E67205B435D0064694A
:101050007374616E636520746F207265747261636E
:1010600074207768656E2068656174696E67205BBF
:101070006D6D5D00657874727564657220636F6F65
:101080006C6572207370656564205B302D32353578
:101090005D00616476616E6365204B205B303D6F5F
:1010A00066665D00616476616E6365204C205B302E
:1010B0003D6F66665D005344204361726420726533
:1010C0006D6F766564005344204361726420696EDD
:1010D00073657274656400534420696E6974206698
:1010E00061696C006572726F722077726974696EE3
:1010F0006720746F2066696C6500426567696E20C1
:1011000066696C65206C69737400456E642066695D
:101110006C65206C6973740046696C65206F70653E
:101120006E65643A002053697A653A0046696C65D9
:101130002073656C65637465640066696C652E6F09
:1011400070656E206661696C65640053442070723E
:10115000696E74696E67206279746520004E6F74E1
:10116000205344207072696E74696E67006F7065F9
:101170006E206661696C65642C2046696C653A2056
:101180000057726974696E6720746F2066696C65B8
:101190003A2000446F6E6520736176696E67206641
:1011A000696C652E0046696C652064656C657465C4
:1011B000640044656C6574696F6E206661696C6576
:1011C00064004469726563746F727920637265614B
:1011D000746564004372656174696F6E206661694D
:1011E0006C6564005344206572726F72436F64656E
:1011F0003A000D0E1C151C141C00002243141F1F66
:1012000029129912ED125D13AD13000000001D1498
:10121000A514B11501167D164D313137204578746E
:101220007275646572203100000000A00F5C0060E0
:1012300009690010097900C0088C007008A200201C
:1012400008BD00D007DE008007050130073401E04B
:10125000066D019006B20140060702F0056D02A07E
:1012600005E80250057B0300052B04B004F8046078
:1012700004EB06C003350920037F0B8002650DE0F7
:1012800001B00E40011D0FF000480FC8006C0FA008
:1012900000ED0F60FFFE0F48FE0400801AD8009892
:1012A00008AC012007800250065403C805280458E2
:1012B00005FC040005D005B004A4066804780728DE
:1012C000044C08E8032009B003F4097003C80A3885
:1012D000039C0BF802700CB002440D6802180E0853
:1012E00002EC0E8801C00F8800F00F00000400001F
:1012F0001B54006009640010097400C00884007069
:10130000089C002008B800D007D8008007000130F2
:10131000072C01E00668019006AC0140060002F0CF
:10132000056802A005E0025005740300052404B01E
:1013300004F0046004DC051004E406C00304087033
:101340000330092003780B8002600DE001A80E40F5
:1013500001680FA000C00F0000E80F60FF040070DC
:101360000DD8004804AC0158038002D80254038011
:101370000228043802FC040002D005C801A4069823
:1013800001780770014C08480120091801F409F0A0
:1013900000C80AC8009C0BA000700C7000440D38F7
:1013A00000180E0000EC0EA8FFC00FE8FE040000BD
:1013B0001B54006009640010097400C008840070A8
:1013C000089C002008B800D007D800800700013032
:1013D000072C01E00668019006AC0140060002F00F
:1013E000056802A005E0025005740300052404B05E
:1013F00004F0046004DC051004E406C00304087073
:101400000330092003780B8002600DE001A80E4034
:1014100001680FA000C00F0000E80F60FF0000404F
:101420001F450060094F0010095C00C0086B007088
:10143000087D0020089200D007AC008007CC003067
:1014400007DE00E006230190065E014006A601F0DB
:1014500005FF01A0056D025005F30200059603B0DB
:10146000045A046004400510044806C0036E077067
:1014700003A8082003EB09D002230B8002410C30A3
:1014800002390DE001040E9001A20E4001170FF089
:1014900000690FA000A20F5000C60F0000DD0FB0C2
:1014A000FFEB0F60FF0400681D4C00500B940058C8
:1014B00009DC0050082401A8076C012807B401C00A
:1014C00006FC017006440228068C02F005D402B81E
:1014D000051C03880564035805AC033005F40310AC
:1014E000053C04E8048404C804CC04A80414059052
:1014F000045C057004A4055804EC05380434062087
:10150000047C060804C406F0030C07D8035407C87B
:10151000039C07B003E40798032C08800374087049
:1015200003BC085803040948034C09300394091804
:1015300003DC090803240AF0026C0AE002B40AC8BA
:1015400002FC0AB002440BA0028C0B8802D40B7080
:10155000021C0C5802640C4002AC0C2802F40C1063
:10156000023C0DF001840DD801CC0DB801140E9889
:10157000015C0E7001A40E4801EC0E1801340FD866
:10158000007C0F8800C40F0800FC0F000000000062
:10159000000000000000000000000000000000004B
:1015A000000000000000000000000000000000003B
:1015B0000004000016D800C006AC0178058002C007
:1015C00004540348042804E803FC049803D005509D
:1015D00003A40618037807D8024C08A80220097053
:1015E00002F4093802C80A08029C0BD001700C9062
:1015F00001440D5001180EF800EC0E8800C00F00D9
:10160000000400401D900060091C01B007A801D033
:101610000634023806C002C8054C036805D8031812
:10162000056404D804F00498047C056004080630BE
:1016300004940600042007D003AC07A803380880F0
:1016400003C408580350093003DC090803680AE0A2
:1016500002F40AB802800B88020C0C6002980C306D
:1016600002240DF801B00DC0013C0E8001C80E30FF
:1016700001540FB800B40F2800E00F000004000868
:101680001D900058091C01B007A801C8063402309B
:1016900006C002C0054C036805D80318056404D0D1
:1016A00004F00498047C05600408063004940600E5
:1016B000042007D003AC07A80338088003C40858E7
:1016C0000350093003DC090803680AD802F40AB0A1
:1016D00002800B88020C0C6002980C3002240DF87A
:1016E00001B00DC0013C0E8001C80E3001540FB88E
:1016F00000B40F2800E00F00005344206572726FA1
:1017000072206669786564005344206572726F7256
:1017100020646964206E6F74207265636F766572F1
:10172000210053442052656164204572726F72003B
:1017300042696E6172793A00436F6D6D616E644209
:101740007566666572000000000000000000000081
:1017500000000000000024F403D950C38EB1C2A2DF
:101760003D96828B3582127AE372816CCB66A861DA
:10177000015DC758EB546151204E1E4B5648C14580
:1017800059431A41013F093D2F3B7139CD3740364E
:10179000C93465331432D430A32F802E6B2D632CC3
:1017A000672B752A8E29B028DC2710274B268F251A
:1017B000D9242B248223E0224322AC211A218D201C
:1017C0000420801F001F841E0C1E971D261DB81CA0
:1017D0004E1CE61B821B201BC11A641A0A1AB2197E
:1017E0005D190A19B9186A181C18D11788174017FB
:1017F000FA16B51673163116F115B31576153A1596
:101800000015C7148F1458142214EE13BA1388133A
:1018100056132513F612C71299126C1240121512A4
:10182000EB11C1119811701148112111FB10D61044
:10183000B1108D106910461024100210E10FC00F76
:10184000A00F800F610F420F230F060FE80ECB0E83
:10185000AF0E930E770E5C0E410E270E0D0EF30D9C
:10186000DA0DC10DA80D900D780D600D490D320DEA
:101870001B0D050DEF0CD90CC30CAE0C990C850C8F
:10188000700C5C0C480C350C210C0E0CFB0BE80B9F
:10189000D60BC40BB20BA00B8E0B7D0B6B0B5A0B34
:1018A0004A0B390B290B180B080BF80AE90AD90A5D
:1018B000CA0ABB0AAC0A9D0A8E0A800A710A630A28
:1018C000550A470A390A2C0A1E0A110A040AF7099E
:1018D000EA09DD09D009C409B709AB099F099209D2
:1018E00087097B096F09630958094C0941093609C1
:1018F0002B09200915090A090009F508EB08E00879
:10190000D608CC08C208B808AE08A4089A089008FF
:1019100087087D0874086B08610858084F08460856
:101920003D0834082C0823081A0812080908010881
:10193000F807F007E807E007D807D007C807C0078F
:10194000B807B007A807A1070000420FA1071605B6
:10195000D0030D038B022E02E801B2018601630160
:1019600045012C0117010401F40049646C6500492C
:10197000646C650049646C6500486F6D6520446562
:101980006C74610053746570706572204469736192
:10199000626C6564004B696C6C65640055706C6FBB
:1019A0006164696E672E2E2E005344207072696E3A
:1019B000742073746F70706564206279207573652C
:1019C000722E005344206361726420696E736572E5
:1019D000746564005344204361726420696E7365CA
:1019E0007274656400534420436172642072656DB3
:1019F0006F76656400534420636172642072656D84
:101A00006F7665640000002110422063308440A599
:101A100050C660E770088129914AA16BB18CC1ADB5
:101A2000D1CEE1EFF13112100273325222B552944D
:101A300042F772D662399318837BB35AA3BDD39C05
:101A4000C3FFF3DEE36224433420040114E664C7D9
:101A500074A44485546AA54BB528850995EEE5CF55
:101A6000F5ACC58DD55336722611163006D776F6ED
:101A7000669556B4465BB77AA719973887DFF7FEA5
:101A8000E79DD7BCC7C448E5588668A77840086179
:101A90001802282338CCC9EDD98EE9AFF9488969F5
:101AA000990AA92BB9F55AD44AB77A966A711A508D
:101AB0000A333A122AFDDBDCCBBFFB9EEB799B5845
:101AC0008B3BBB1AABA66C877CE44CC55C222C0319
:101AD0003C600C411CAEED8FFDECCDCDDD2AAD0B95
:101AE000BD688D499D977EB66ED55EF44E133E322D
:101AF0002E511E700E9FFFBEEFDDDFFCCF1BBF3AE5
:101B0000AF599F788F8891A981CAB1EBA10CD12DD3
:101B1000C14EF16FE18010A100C230E320045025D6
:101B20004046706760B9839893FBA3DAB33DC31C4A
:101B3000D37FE35EF3B1029012F322D23235421426
:101B40005277625672EAB5CBA5A89589856EF54F96
:101B5000E52CD50DC5E234C324A014810466744776
:101B60006424540544DBA7FAB79987B8975FE77EEA
:101B7000F71DC73CD7D326F2369106B016576676C6
:101B800076154634564CD96DC90EF92FE9C899E936
:101B9000898AB9ABA94458654806782768C018E116
:101BA000088238A3287DCB5CDB3FEB1EFBF98BD88A
:101BB0009BBBAB9ABB754A545A376A167AF10AD066
:101BC0001AB32A923A2EFD0FED6CDD4DCDAABD8BD6
:101BD000ADE89DC98D267C076C645C454CA23C83B6
:101BE0002CE01CC10C1FEF3EFF5DCF7CDF9BAFBA2A
:101BF000BFD98FF89F176E367E554E745E932EB206
:101C00003ED10EF01E7C3C3E5E2B3D3F2F5B5D3B8C
:101C10002C2A225C004E6F206572726F7220666FF4
:101C2000756E642E0043616E2774206F70656E20A0
:101C3000726F6F74206469726563746F72792E00BD
:101C4000496E76616C696420666F726D61742C20D8
:101C50007265666F726D61742053442E004E6F2062
:101C6000636172642C2077726F6E6720636869709D
:101C70002073656C6563742070696E2C206F722010
:101C80005350492070726F626C656D3F0043616E06
:101C9000277420616363657373205344206361720A
:101CA000642E20446F206E6F74207265666F726DB3
:101CB00061742E000000000000000000000000FF22
:101CC00000000100416374696F6E3A256C61000386
:101CD00010270200B41E0310270200B81E010000E6
:101CE0000100BC1E0200000600BE1E03ED0304003E
:101CF000CA1E03EE030400D21E03EF030400DA1E23
:101D000003FA030400E21E03FB030400EA1E03FCC3
:101D1000030400F21E0200000B00FA1E020000067F
:101D200000101F02000006001C1F526571756573CC
:101D30007450617573653A004E6F205344204361BF
:101D4000726400436F6F6C646F776E0050726568E9
:101D5000656174204142530050726568656174206A
:101D6000504C41008025000040380000004B00002E
:101D70008070000000960000C0DA000000E1000062
:101D8000002C010008B2010000C2010000F40100B3
:101D90000084030090D0030000E80300000807005F
:101DA00020A1070000100E0040420F0060E3160063
:101DB000000000000200000900281F3A1F411F48D0
:101DC0001F4F1F4F6E004F666600596573004E6FC0
:101DD00000030004004E2F4100003A0020646179A6
:101DE0007320005E464A404E055F4A44494A440516
:101DF0004844460042616E6742616E6700536C6FF3
:101E00007742616E6700446561642054696D6500C6
:101E1000504944005072696E74696E672E2E2E0010
:101E20002064656620000000003FCDCC4C3D0AD701
:101E3000A33B6F12033A6642485944464A404E0B50
:101E40001A051B18005C5C5C054642485944464A2A
:101E5000404E054845005E464A404E055F4A4449AB
:101E60004A4405484446000E2A20312C2E222826BA
:101E700063312622273A6D0000401454040E1504E5
:101E80001C000000040A040000000000001F1F1FC7
:101E90001F1F0000001F1111111F0000040A0A0A71
:101EA0000E1F1F0E001C1F11111F0000110A04112C
:101EB000040A1111561F5D1F641F6B1F721F721FD2
:101EC000791F801F871F8E1F951F9C1FA31FAA1F8E
:101ED000B11FB81FBF1FC61FCD1FD41FDB1FE21FBE
:101EE000E91FF01FF71FFE1F05200C2013201A20EA
:101EF000212028202F2036203D20721F44204B20F7
:101F000052205920602067206E2075207C2083207D
:101F1000721F8A20912098209F20A620721F4420A3
:101F2000AD20B420BB209F20721FC220791FC92082
:101F3000D020D720DE20E520EC200000000400F3B4
:101F4000200000000400FB2000000004000321002A
:101F5000000004000B2113210000000000212100DB
:101F600000000000322100000000004021000000BD
:101F70000000512103E8030000582103F50301028A
:101F8000632103F60302046F2103540402007A2143
:101F900003F7030400892103F403010295210000E3
:101FA0000000009E210000000000AE2100000000A3
:101FB00000BE210000000000BF210000000000C89A
:101FC000210000000000D8210000000000E82100EE
:101FD00000000000E9210000000000F221000000E4
:101FE0000000022200000000001222000000000099
:101FF000132200000000001C2200000000002C2220
:1020000000000000003C2200000000003D22000013
:1020100000000046220000000000562200000000E0
:10202000006622000000000067220000000000702F
:10203000220000000000802200000000009022002A
:1020400000000000912203FD0300109A22045704AF
:102050000000A922041F040000BB22044804000061
:10206000CD220337040000D9220347040000E522F3
:102070000338040000EE220331040010FC22034266
:102080000400100C2303360400001D23043C04004C
:10209000002D23043D0400003D23033A0400004CBE
:1020A00023025B230000622303430400006D23022C
:1020B000EB1C0000782302F21C0000832302F91CB1
:1020C00000008E2302151D00009D2302231D000029
:1020D000A623021C1D0000AF2302B9230000C02369
:1020E00002E41C0000C82302D2230000D92302E727
:1020F000230000EE23F523FC2303240A24112418D3
:10210000241F2426242D2434243B244224492450F3
:10211000245724436F6E66696775726174696F6EC8
:102120000073746F72656420696E20454550524F8C
:102130004D00436F6E66696775726174696F6E00FA
:102140006C6F6164656420662E20454550524F4D8A
:10215000004261636B2001005072696E74206669F1
:102160006C65005061757365205072696E74005320
:10217000746F70205072696E7400436F6E74696E74
:102180007565205072696E740044656C65746520D5
:1021900066696C6500583A257830206D6D004D6990
:1021A0006E20656E6473746F703A257378004D61AC
:1021B0007820656E6473746F703A25735800005907
:1021C0003A257831206D6D004D696E20656E64731F
:1021D000746F703A257379004D617820656E647371
:1021E000746F703A25735900005A3A257832206D81
:1021F0006D004D696E20656E6473746F703A25735F
:102200007A004D617820656E6473746F703A25733F
:102210005A0000583A257830206D6D004D696E20C7
:10222000656E6473746F703A257378004D61782021
:10223000656E6473746F703A2573580000593A25BF
:102240007831206D6D004D696E20656E6473746F1A
:10225000703A257379004D617820656E6473746FF0
:10226000703A25735900005A3A257832206D6D0076
:102270004D696E20656E6473746F703A25737A00D1
:102280004D617820656E6473746F703A25735A00DF
:1022900000486F6D6520416C6C005A204261627984
:1022A0007374657070696E67005370656564204D66
:1022B000756C2E3A256F6D25252500466C6F7720AD
:1022C0004D756C2E203A256F6625252500507265C8
:1022D0006865617420504C41005072656865617496
:1022E0002041425300436F6F6C646F776E005365FB
:1022F0007420746F204F726967696E00446973615E
:10230000626C65207374657070657200415458206A
:10231000706F776572206F6E2F6F6666004265641E
:102320002054656D703A2025456202430054656D66
:10233000702E20313A202025453002430045787424
:1023400072756465722031204F666600457874723C
:102350002E20706F736974696F6E0003F0030200C2
:102360005E24536574204F726967696E005820506F
:102370006F736974696F6E005920506F7369746967
:102380006F6E005A20506F736974696F6E005175DB
:1023900069636B2053657474696E677300506F7363
:1023A0006974696F6E004578747275646572004671
:1023B000616E20737065656400020000070062248E
:1023C0005344204361726400446562756767696EB7
:1023D000670002000005007024436F6E6669677530
:1023E000726174696F6E0002000009007A248C2407
:1023F00000000000009F240000000000B124000045
:10240000000000C6240000000000CA2400000000F4
:1024100000D3240000000000DC240000000000E5E0
:10242000240000000000E9240000000000FA24005D
:10243000000000000B2500000000000C250000003B
:102440000000102500000000001E25000000000014
:10245000222500000000003325000000000039257F
:102460004025721F47254E2555255C2563256A2585
:10247000721F712578257F258625721F8D2594254D
:102480009B25A225A925B025B725BE250525656371
:102490002F25456302422565422F25456202005AD9
:1024A0003A25783220202020204275663A256F4256
:1024B000004D756C3A20256F6D202020466C6F779B
:1024C0003A20256F6600256F7300583A2578302032
:1024D0006D6D00593A257831206D6D005A3A257896
:1024E00032206D6D00256F730045313A2565302F20
:1024F00025453002437E256F300020423A25656233
:102500002F25456202437E256F620000256F730010
:102510005072696E74696E672074696D6500255527
:10252000740046696C616D656E74207072696E74BA
:10253000656400255566206D00C52500000000007B
:10254000CE250000000000DD250452040000EE2529
:10255000031A040800FB25031B0400000926031CC2
:102560000400001726031D0400002526031E040096
:1025700000322603320400003E2603330400004AE2
:1025800026033404000056260335040000622602A8
:102590006A2600007126027E2600008526028E260D
:1025A00000009526029E260000A5260306040000D2
:1025B000B5260307040000C42602CD260000D42659
:1025C00002E0260000453A257833206D6D00312069
:1025D000636C69636B203D2031206D6D0046616E38
:1025E0002073706565643A2546732525250054756A
:1025F000726E2046616E204F6666005365742046F9
:10260000616E203235252525005365742046616EA4
:10261000203530252525005365742046616E20370E
:1026200035252525005365742046616E2046756C5E
:102630006C004563686F2020203A25646F00496E66
:10264000666F2020203A256469004572726F7273AC
:10265000203A256465004472792072756E3A2564CB
:10266000640047656E6572616C000200000400E75B
:1026700026416363656C65726174696F6E00020068
:10268000000900EF2646656564726174650002000A
:1026900000070001274578747275646572000200B6
:1026A0000011000F2753746F726520746F20454529
:1026B00050524F4D004C6F616420662E20454550AE
:1026C000524F4D005A2043616C69622E0002000097
:1026D000040031274C6576656C2064656C7461007C
:1026E00002000008003927721F4927502757277218
:1026F0001F5E2765276C2773277A27812788278FF6
:1027000027721F96279D27A427AB27B227B92772C8
:102710001FC027C727CE27D527DC27E327EA27F1C5
:1027200027F827FF2706280D2814281B28222829E8
:1027300028721F442030283728721F3E2845284C15
:10274000285328AD20B420BB205A280410040000D0
:10275000672802782800007F28028D28000094282E
:102760000408040000A0280409040000AC28040A9E
:10277000040000B828040B040000C428040C040062
:1027800000D028040D040000DC28040E040000E83A
:1027900028040F040000F4280414040000FE280498
:1027A000150400000829041604000012290411046D
:1027B00000001D290412040000282904130400004D
:1027C000332904290400004029042C0400004D2969
:1027D000042B0400005829042A0400006229042E56
:1027E0000400007029044D0400008329044C0400F7
:1027F0000094290446040000A4290430040000B514
:1028000029042D040000C1290422040000CE29045B
:1028100023040000D8290424040000E2290425042C
:102820000000F0290426040000FE29042F04000003
:102830000A2A02152A00001C2A03AC0F0000242AD1
:1028400003AD0F00002B2A03AE0F0000322A03AFA6
:102850000F0000392A03B00F0000426175647261F5
:1028600074653A256F630053746570706572204912
:102870006E6163746976650003200402004C2A4D82
:1028800061782E20496E616374697665000358048F
:102890000200502A5072696E7420583A25617800FF
:1028A0005072696E7420593A256179005072696ED0
:1028B00074205A3A25617A004D6F76652058203A87
:1028C000256158004D6F76652059203A25615900E1
:1028D0004D6F7665205A203A25615A004A65726B21
:1028E0002020203A25616A005A2D4A65726B203AF1
:1028F00025614A004D617820583A256678004D617F
:102900007820593A256679004D6178205A3A256633
:102910007A00486F6D6520583A25665800486F6DFB
:102920006520593A25665900486F6D65205A3A2549
:10293000665A0053746570732F4D4D3A25536500E8
:1029400053746172742046523A255866004D61787E
:102950002046523A25584600416363656C3A255833
:102960004100537461622E54696D653A25587700B1
:102970005761697420556E6974733A202558552043
:102980006D6D00576169742054656D702E20255857
:1029900054024300416476616E6365206C696E3A4F
:1029A00025586C00416476616E63652071756164C1
:1029B0003A25586100436F6E74726F6C3A255868FF
:1029C0000044542F50494420503A25587000504933
:1029D0004420493A2558690050494420443A255832
:1029E00064004472697665204D696E3A25586D0021
:1029F0004472697665204D61783A25584D005049FA
:102A000044204D61783A255844005A20506F73692C
:102A100074696F6E000355040400542A53657420D2
:102A20005A3D300053657420503100536574205076
:102A300032005365742050330043616C63756C61E0
:102A40007465204C6576656C696E67005C2A632A44
:102A50006A2A712A782A7F2A862A8D2A942A0000D7
:102A6000000000A32A0000000000AD2A00000000C2
:102A700000BC2A0000000000C62A0000000000CFB1
:102A80002A0000000000DF2A0000000000EF2A00FA
:102A9000000000004469732E2041667465723A2577
:102AA0006973005B735D20303D4F66660044697357
:102AB0002E2041667465723A256970005B735D2053
:102AC000303D4F6666005A3A257832206D6D004DD4
:102AD000696E20656E6473746F703A25737A004D69
:102AE000617820656E6473746F703A25735A0000C4
:102AF00000002100240027002A002D0030003300B0
:102B000001010000040107010A0100002200250064
:102B100028002B002E0031003400020100000501C6
:102B200008010B01000020002300260029002C00D2
:102B30002F00320000010000030106010901050514
:102B40000505070508080808020202020A0A080823
:102B50000404040401010101010101010303030351
:102B600003030303040707070C0C0C0C0C0C0C0CE0
:102B70000202020206060606060606060B0B0B0BF1
:102B80000B0B0B0B01021020200808102040102016
:102B90004080020102010804020101020408102021
:102BA000408080402010080402018004020180401F
:102BB0002010080402010804020101020408102088
:102BC000408001020408102040800000090A020829
:102BD0000B0C0D07060304010000000000000000BC
:102BE00000000000000000000000000000000000E5
:102BF00000000000000011100F00000000000000A5
:102C000000000000000000000000000000000000C4
:102C100002494E46494E4954594E414ECDCCCC3DC9
:102C20000AD7233C17B7D13877CC2B329595E624B9
:102C30001FB14F0A000020410000C84200401C465E
:102C400020BCBE4CCA1B0E5AAEC59D740D942C06FA
:102C50000D69CCB560D611241FBECFEFD1E2DEBF27
:102C6000CDBF00E00CBF13E0A0E0B2E0ECE4FEE179
:102C700002E00BBF02C007900D92A834B107D9F74C
:102C80001BBE1DE1A8E4B3E001C01D92AE37B10741
:102C9000E1F71CE2C6E5DCE204C02297FE010F94D6
:102CA000D60EC035D107C9F70F941D060D94240F19
:102CB0000C940000A0E0B0E0E0E6F6E10D94F30E25
:102CC000EC015B016115710519F0FB0191838083B3
:102CD000F9908F2D90E00F94DA0E892BC9F7FDE261
:102CE000FF1621F4F990EE24E39405C02BE2F216CE
:102CF00009F4F990EE248E0101501040C80161E101
:102D00007CE243E050E062D2892BF9F48E010E5F41
:102D10001F4FC80164E17CE245E050E057D2892BA7
:102D200019F48E01095F1F4FA114B10419F0F501C8
:102D300011830083E0FC04C070E090E080E813C0E1
:102D400070E090E080E86FEF07C1C80169E17CE2C4
:102D500043E050E03BD2892B69F4A114B10429F47B
:102D600070E090E080EC6FE7F7C02296F501D18328
:102D7000C083F6CF8824992440E050E060E070E002
:102D8000EF2DE053EA30A0F5F2E0EF2A8E2D90E02F
:102D90009C0128703070E2FE06C0232B79F5089460
:102DA000811C911C2BC0232B19F0089481089108D9
:102DB000DB01CA0112E0880F991FAA1FBB1F1A95D9
:102DC000D1F7480F591F6A1F7B1F440F551F661FFD
:102DD000771F4E0F511D611D711D483929E952079A
:102DE00029E9620729E1720748F084E0E82A06C071
:102DF000EE3F31F4E3FC39C098E0E92AF990C0CF06
:102E0000E53311F0E53189F529912D3219F4E0E12E
:102E1000EE2A05C02B3219F081E090E003C0299121
:102E200082E090E0E22FE053EA3018F0C81BD90BA3
:102E30001CC020E030E0FCE020383F075CF4C90112
:102E4000880F991F880F991F280F391F220F331FD2
:102E50002E0F311DE991E053EA3068F3E4FE03C020
:102E6000309521953F4F820E931ECE2CDD24E1FE3E
:102E700007C0A114B10421F02197F501D183C083CB
:102E8000CB01BA010F94520B7B018C01F3E0CF22EE
:102E9000DD2423E0C216D10421F417FB109517F9A5
:102EA000109557016801C801B70120E030E040E00B
:102EB00050E00F94B20A882309F44AC097FE0DC06F
:102EC00020E3E22E2CE2F22E9094819491089394C8
:102ED000C0E2D0E000E010E012C098E4E92E9CE2ED
:102EE000F92EF6CFF7012591359145915491C60100
:102EF000B5010F94620D5B016C018C1A9D0A8C1652
:102F00009D0684F7D595C7950F5F1F4F06301105B5
:102F100029F08CEF9FEFE80EF91EF1CFC501D60125
:102F20007C018D018C2D880F8D2D881F8F3F51F0D6
:102F3000C601B50120E030E040E050E00F94B20A55
:102F4000882331F482E290E090937D1D80937C1D74
:102F50007E2D9F2D802F612F272F392F482F562F01
:102F6000B901CA01CDB7DEB7ECE00D940F0F2F9277
:102F70003F925F926F927F928F929F92AF92BF9299
:102F8000CF92DF92EF92FF920F931F93CF93DF9335
:102F90008C011B01EA016115710519F0FB01918398
:102FA0008083209749F0CE010297839728F020E094
:102FB00030E040E050E0F6C0F801A1908F018A2D8A
:102FC00090E00F94DA0E892BB9F7FDE2AF1631F4D9
:102FD000F801A1908F015524539407C0FBE2AF166E
:102FE00019F4F801A1908F015524209719F0C031F0
:102FF000D105C1F4F0E3AF1679F4F8018081883788
:1030000011F0883549F4F801A1800E5F1F4FF2E0FE
:103010005F2AC0E1D0E006C0209721F480E3A81623
:10302000E9F427C0C830D10531F1C930D10524F405
:10303000C230D10531F50CC0CA30D10589F0C0319C
:10304000D105F9F4C12CD12CE12CB8E0FB2E28C01D
:10305000C12CD12CE12CA0E4FA2E22C0CAE0D0E091
:10306000FCECCF2EFCECDF2EFCECEF2EFCE0FF2E78
:1030700017C0C8E0D0E0C12CD12CE12CE0E1FE2E3D
:103080000FC09E01442737FD4095542F60E070E04B
:1030900080E090E80F948B0EC901DA016C017D018C
:1030A00020E030E040E050E060E03E01882477FC22
:1030B0008094982C70EDB72EBA0CE9E0EB1570F403
:1030C0008A2D81548A3118F499ECB92E06C08A2DC4
:1030D00081568A3150F589EAB82EBA0C8B2D90E0D2
:1030E0008C179D0714F56F3FE1F0C216D306E40676
:1030F000F506B0F0CA01B901A40193010F94380E8E
:103100009B01AC012B0D311D411D511D2130F0E003
:103110003F07F0E04F07F0E85F0710F461E001C0FF
:103120006FEFF801A1908F01C5CF2114310481F018
:10313000662331F001501040F1011183008308C073
:1031400051FE1AC002501040F1011183008314C0D7
:1031500067FF12C050FC05C02FEF3FEF4FEF5FE756
:1031600004C020E030E040E050E882E290E090933C
:103170007D1D80937C1D16C050FE08C05095409563
:10318000309521953F4F4F4F5F4F0CC057FF0AC0FE
:1031900082E290E090937D1D80937C1D2FEF3FEFA6
:1031A0004FEF5FE7B901CA01DF91CF911F910F91F6
:1031B000FF90EF90DF90CF90BF90AF909F908F9057
:1031C0007F906F905F903F902F900895FB01DC01FE
:1031D0004150504088F08D9181341CF08B350CF4B7
:1031E000805E659161341CF06B350CF4605E861B6B
:1031F000611171F3990B0895881BFCCFFB01DC0171
:1032000002C001900D9241505040D8F70895FB0143
:10321000DC010D900020E9F7119701900D9200203C
:10322000E1F70895FC018191861721F08823D9F7F1
:10323000992708953197CF010895FB01DC018D9105
:10324000019080190110D9F3990B0895FB01DC015D
:1032500001900D920020E1F70895FB01DC0141503F
:10326000504048F001900D920020C9F701C01D9216
:1032700041505040E0F70895FC0181E090E001905A
:10328000061609F4CF010020D1F70197089508959B
:1032900060911102709112028091130290911402B8
:1032A0006817790744F470931402609313028EE355
:1032B00094E00C9464360895BC01893191051CF4A6
:1032C00069E170E005C0893C910514F068EC70E09C
:1032D00070930C1960930B198CE894E00C9464368D
:1032E000EF92FF920F931F93CF93DF93EC018931FD
:1032F00091051CF4C9E1D0E006C081E0C53FD807C4
:1033000014F0C4EFD1E0BE01882777FD8095982F97
:103310000F94540B7B018C016091091970910A196B
:10332000882777FD8095982F0F94540B9B01AC0153
:10333000C801B7010F94B90A9B01AC01609105194E
:103340007091061980910719909108190F94620DD8
:1033500060930519709306198093071990930819C3
:10336000D0930A19C09309198DE794E0BE010E9419
:103370006436DF91CF911F910F91FF90EF900895E8
:103380000E943B6B9C0180911102909112022817C0
:10339000390724F4309312022093110208950C94FB
:1033A000086708952F923F924F925F926F927F929B
:1033B0008F929F92AF92BF92CF92DF92EF92FF9245
:1033C0000F931F93DF93CF93CDB7DEB728970FB638
:1033D000F894DEBF0FBECDBFA090F417B090F517E4
:1033E000C090F617D090F7172090F8173090F91783
:1033F0004090FA175090FB178091FC179091FD17A1
:10340000A091FE17B091FF1789839A83AB83BC8389
:1034100020911C1830911D1840911E1850911F18B2
:103420006090201870902118809022189090231896
:103430008091241890912518A0912618B0912718F2
:103440008D839E83AF83B88780919F17882359F41B
:103450000F2EF0E0EF2EF0E0FF2EF0E80F2FFFE34D
:103460001F2FF02D0AC00F2EF0E7EF2EF2E4FF2EF3
:10347000F1E20F2FFDE31F2FF02DC601B5010F94D0
:10348000EC09A80197010F94620DAB01BC0188E41F
:1034900094E022E00E94933780919F17882359F48B
:1034A0000F2EF0E0EF2EF0E0FF2EF0E80F2FFFE3FD
:1034B0001F2FF02D0AC00F2EF0E7EF2EF2E4FF2EA3
:1034C000F1E20F2FFDE31F2FF02DC201B101A40186
:1034D00093010F94EC09A80197010F94620DAB01C1
:1034E000BC018FE494E022E00E94933780919F1703
:1034F000882359F40F2EF0E0EF2EF0E0FF2EF0E8D5
:103500000F2FFFE31F2FF02D0AC00F2EF0E7EF2E35
:10351000F2E4FF2EF1E20F2FFDE31F2FF02D698162
:103520007A818B819C812D813E814F8158850F94BA
:10353000EC09A80197010F94620DAB01BC0183E572
:1035400094E022E00E9493372091F0173091F11718
:103550004091F2175091F317A090AC17B090AD17AF
:10356000C090AE17D090AF1780919F17882359F461
:103570000F2EF0E0EF2EF0E0FF2EF0E80F2FFFE32C
:103580001F2FF02D0AC00F2EF0E7EF2EF2E4FF2ED2
:10359000F1E20F2FFDE31F2FF02DCA01B9010F94A7
:1035A000540BA60195010F94620DA80197010F9489
:1035B000620DAB01BC0187E594E022E00E94CB37AD
:1035C00028960FB6F894DEBF0FBECDBFCF91DF9126
:1035D0001F910F91FF90EF90DF90CF90BF90AF9031
:1035E0009F908F907F906F905F904F903F902F9023
:1035F00008950F931F9304E015E0C8016DE00E9449
:10360000DC68C8016AE00E94DC681F910F91089590
:103610006F927F928F929F92AF92BF92CF92DF92E2
:10362000EF92FF920F931F93DF93CF9300D00F92EF
:10363000CDB7DEB740911F19509120196091211923
:1036400070912219FE01319621E830E0F999FECF00
:1036500032BD21BDF89A80B581932F5F3F4F253849
:103660003105A1F7CB01BA012FE632E143E85AE375
:103670000F94620D29813A814B815C810F94EC0992
:10368000AB01BC0184EA94E022E00E94933785EC10
:1036900094E00E943236E091CF02F091D00263852F
:1036A00074858585968520E030E040E751E40F94ED
:1036B000C00C18160CF496C0AA24BB246501F99915
:1036C000FECF8DE790E092BD81BDF89A50B5F99993
:1036D000FECF8EE790E092BD81BDF89A40B5F99992
:1036E000FECF8FE790E092BD81BDF89A30B5F99991
:1036F000FECF80E890E092BD81BDF89A20B5852F7D
:10370000942FA32FB22FA80EB91ECA1EDB1EC6010E
:10371000B50120E831E541E050E00F94AD0E922E66
:10372000832E742E652E622F732F842F952F20E801
:103730003EEA4EEF5FEF0F94380E7B018C01EA0CEE
:10374000FB1C0C1D1D1D86EB94E0492D582D672D8B
:10375000762D0E948736C801B70120E13EE040E0A7
:1037600050E00F94AD0ED22EC32EB42EA52E88ECB1
:1037700094E0422F5C2D6B2D7A2D0E9487366D2DA3
:103780007C2D8B2D9A2D20EF31EF4FEF5FEF0F94B3
:10379000380EE60EF71E081F191FC801B7012CE3EB
:1037A00030E040E050E00F94AD0E8FEC94E0BA01B1
:1037B000A9010E94873687ED94E00E94BC360F90E5
:1037C0000F900F900F90CF91DF911F910F91FF906D
:1037D000EF90DF90CF90BF90AF909F908F907F90B1
:1037E0006F9008950F94860320911B1930911C1936
:1037F00040911D1950911E19621B730B840B950B80
:1038000028EE33E040E050E00F948B0EC901DA015E
:103810005C016D0154CF1F93182FE0915603F09176
:10382000570346A957A960AD71AD8BE594E022E03E
:103830000E949337E0915603F091570342AD53AD88
:1038400064AD75AD8AE794E020E00E9493370E9452
:103850008751AB01BC018EE594E022E00E949337D2
:103860004091990250919A0260919B0270919C0242
:103870008AE794E020E00E949337112391F081E7DA
:1038800094E061E070E00E9496366CEF7FE08091FA
:10389000910290919202681B790B86E794E00E9456
:1038A0009636E0918E02F0E0EE5CFA4F60818CE695
:1038B00094E070E00E949636E0911702EF3F29F401
:1038C000E0915603F0915703E081F0E0EE5CFA4F8F
:1038D000608182E694E070E00E9496368ADE1F9155
:1038E000089580914A038823C1F010924A030E94F0
:1038F000F65A80911602815080931602882349F46B
:1039000080911502833010F40E94595485E0809311
:10391000160285E29CE10C94D9FF089507C00E942D
:10392000C963DFDF85E29CE10E945FD680918B173F
:103930008823A9F70895CF93DF9397FD10C0EC017A
:103940008F3F910521F01CF0CFEFD0E002C000972F
:1039500031F080912A18886080932A1807C08091DE
:103960002A18877F80932A18C0E0D0E0662309F0E8
:10397000D5DF8091350590E0C817D90729F08AE98D
:1039800094E0BE010E946436C0933505DF91CF916B
:1039900008952F923F924F925F926F927F928F92F3
:1039A0009F92AF92BF92CF92DF92EF92FF920F93CE
:1039B0001F93DF93CF93CDB7DEB7C95DD0400FB66D
:1039C000F894DEBF0FBECDBF4C0180912E03282F8F
:1039D00084FF19C0D4018C9182FD09C081FF13C0FE
:1039E00016968D919C9117978F36910561F00F94E3
:1039F000860360932205709323058093240590939A
:103A000025050C943135F4010081118102FD02C0BD
:103A10000C94A72A808591858E31910509F4C0C444
:103A20008F31910500F58430910509F432C285305B
:103A3000910520F4029708F44DC06EC085319105C0
:103A400009F469C28631910528F4449711F00C9469
:103A50009B2A5CC28C31910509F461C24D9711F02B
:103A60000C949B2A9DC28C35910511F40C947D25F4
:103A70008D359105A0F48032910509F4C9C48032D6
:103A8000910508F4B5C48A35910511F40C94762596
:103A90008B35910511F00C949B2A0C947925843870
:103AA000910511F40C949F268538910538F48338DC
:103AB000910511F00C949B2A0C94372685389105BA
:103AC00011F40C94D727853E910511F00C949B2A94
:103AD0000C94962812FF12C0F401878D90A1A1A129
:103AE000B2A1209129180097A105B10519F0822FE4
:103AF000806202C0822F8F7D80932918C4010E94AA
:103B0000ACA5882311F40C949B2A81E061E041E08C
:103B10000E944F8C0C949B2A8091F4179091F5177A
:103B2000A091F617B091F7178D879E87AF87B88B56
:103B30008091F8179091F917A091FA17B091FB179F
:103B4000898B9A8BAB8BBC8B8091FC179091FD1766
:103B5000A091FE17B091FF178D8B9E8BAF8BB88F06
:103B6000C4010E94ACA5882311F40C949B2AFE0189
:103B7000359688E0DF011D928A95E9F7F40182818C
:103B800080FD05C020E030E040E050E007C0D401F7
:103B900097962D913D914D915C919A9780919F17A9
:103BA000882351F0CA01B90123E333E34BEC51E41C
:103BB0000F94620D9B01AC012D833E834F83588788
:103BC000F401828181FD05C020E030E040E050E05A
:103BD00007C0D4019B962D913D914D915C919E978C
:103BE00080919F17882351F0CA01B90123E333E381
:103BF0004BEC51E40F94620D9B01AC0129873A878D
:103C00004B875C87FE01799680E1DF011D928A95E2
:103C1000E9F78091F4179091F517A091F617B091FC
:103C2000F717898F9A8FAB8FBC8F8091F81790917F
:103C3000F917A091FA17B091FB178D8F9E8FAF8F58
:103C4000B8A38091FC179091FD17A091FE17B09139
:103C5000FF1789A39AA3ABA3BCA360911818709116
:103C6000191880911A1890911B180F94540B2091D9
:103C7000AC173091AD174091AE175091AF170F941C
:103C8000620D6DA37EA38FA398A7F401828182FFAA
:103C9000DCC0A7A4B0A8C1A8D2A880919F17882390
:103CA00051F0C601B50123E333E34BEC51E40F942B
:103CB000620D5B016C01698D7A8D8B8D9C8D2D85DC
:103CC0003E854F8558890F94EB09C255DF4F6883B5
:103CD00079838A839B83CE5AD0406D8D7E8D8F8D64
:103CE00098A129893A894B895C890F94EB092B01AA
:103CF0003C01C601B50120E030E040E850E40F94FB
:103D0000620DA60195010F94620D7B018C01C255D5
:103D1000DF4F688179818A819B81CE5AD0409B0197
:103D2000AC010F94620D9B01AC01C801B7010F9467
:103D3000EB097B018C01C301B201A30192010F9435
:103D4000620D9B01AC01C801B7010F94EB090F9400
:103D5000CF0D7B018C01C255DF4F688179818A814B
:103D60009B81CE5AD040A30192010F94CD0C9B01B0
:103D7000AC0117FB109517F91095C801B7010F9406
:103D8000B90A7B018C01A80197010F941C0E8823AE
:103D900031F08CED94E00E94BF360C949B2AD40144
:103DA00018968D919C911997039721F417FB109504
:103DB00017F91095C601B50120E030E040E050E071
:103DC0000F94B20A882344F417FB109517F9109545
:103DD000D7FAD094D7F8D094C301B201A8019701C3
:103DE0000F94620D9B01AC01C255DF4F6881798150
:103DF0008A819B81CE5AD0400F94EB0920E030E0BD
:103E000040E05FE30F94620D6D837E838F8398871C
:103E1000C255DF4F688179818A819B81CE5AD0401B
:103E2000A80197010F94620D9B01AC01C301B2017F
:103E30000F94EC0920E030E040E05FE30F94620D66
:103E400069877A878B879C870CC06D817E818F8183
:103E5000988529853A854B855C850F94CD0C5B014F
:103E60006C01E0E0D40118968D919C91199702970E
:103E700009F4E1E0CE010D96BE01675E7F4FAE0111
:103E80004B5F5F4F96018501EE2E0E94A6780C9441
:103E90009B2A44DDF4018081918193FD04C0EE24CE
:103EA000FF24870107C0D4019396ED90FD900D91FA
:103EB0001C91969792FF0DC0F401678D70A181A1AE
:103EC00092A128EE33E040E050E00F94380E7B01E1
:103ED0008C010F9486035B016C01AE0CBF1CC01EED
:103EE000D11E03C00E94C963FCDC0F948603250128
:103EF0003601461A570A680A790AD301C20180506E
:103F00009449A543B74770F30C949B2A81E08093B2
:103F10009F170C949B2A10929F170C949B2AC80100
:103F200088739070892B11F080E008C0C80156E0BA
:103F3000969587955A95E1F78095817006FF08C0A0
:103F40001092F0171092F1171092F2171092F317C7
:103F5000882321F041E061E051E01EC0D4012D91A1
:103F60003C91C90188739070892B09F4E4C6C9019A
:103F700043E0969587954A95E1F7582F5170C9010E
:103F800004E0969587950A95E1F7682F617025FD05
:103F900002C040E001C041E0852F0E943FACCBC68B
:103FA0008AE399E00E9461623090281880E00E94C4
:103FB0009D9C4090051950900619609007197090CB
:103FC0000819CA55DF4F488259826A827B82C65AD5
:103FD000D040FE01319620E333E0F999FECF32BDA7
:103FE00021BDF89A80B581932F5F3F4F43E0243382
:103FF000340799F7E980FA800B811C81FE01319624
:1040000024E333E0F999FECF32BD21BDF89A80B5A3
:1040100081932F5F3F4F53E02833350799F729816C
:104020003A814B815C81DE011196E8E4F3E0F99975
:10403000FECFF2BDE1BDF89A80B58D93319683E055
:10404000EC34F807A1F700D00F9289819A81AB81F7
:10405000BC81EDB7FEB781839283A383B483C8018B
:10406000B7010F2EF0E8EF2EFFE4FF2EF3EC0F2F39
:10407000F7E41F2FF02D570168010E9482A10F90D5
:104080000F900F900F9081E060E043E020E00E94ED
:10409000BF9CC655DF4F688379838A839B83CA5A46
:1040A000D04020E030E040E050E00F94B20A87FFBB
:1040B00002C00C949B2AFE01319628E333E0F99963
:1040C000FECF32BD21BDF89A80B581932F5F3F4F5F
:1040D00043E02C33340799F7E980FA800B811C8187
:1040E000FE0131962CE333E0F999FECF32BD21BDBC
:1040F000F89A80B581932F5F3F4F53E02034350706
:1041000099F729813A814B815C81DE011196E8E4BF
:10411000F3E0F999FECFF2BDE1BDF89A80B58D9339
:10412000319683E0EC34F807A1F700D00F92898133
:104130009A81AB81BC81EDB7FEB781839283A38363
:10414000B483C801B7010F2EF0E8EF2EFFE4FF2E75
:10415000F3EC0F2FF7E41F2FF02D570168010E9499
:1041600082A10F900F900F900F9080E060E043E0ED
:1041700021E00E94BF9C2B013C0120E030E040E0A8
:1041800050E00F94B20A87FF02C00C949B2AFE01F4
:10419000319620E433E0F999FECF32BD21BDF89A83
:1041A00080B581932F5F3F4F43E02434340799F764
:1041B000E980FA800B811C81FE01319624E433E012
:1041C000F999FECF32BD21BDF89A80B581932F5F5A
:1041D0003F4F53E02834350799F729813A814B81C5
:1041E0005C81DE011196E8E4F3E0F999FECFF2BDBF
:1041F000E1BDF89A80B58D93319683E0EC34F807F1
:10420000A1F700D00F9289819A81AB81BC81EDB773
:10421000FEB781839283A383B483C801B7010F2EB5
:10422000F0E8EF2EFFE4FF2EF3EC0F2FF7E41F2F43
:10423000F02D570168010E9482A10F900F900F90FE
:104240000F9080E061E043E021E00E94BF9C7B0191
:104250008C0120E030E040E050E00F94B20A87FF8C
:1042600002C00C949B2AC655DF4F688179818A81F0
:104270009B81CA5AD040A30192010F94EC09A80176
:1042800097010F94EC092BEA3AEA4AEA5EE30F94AD
:10429000620D7B018C0184E099E0B801A70122E066
:1042A0000E94CB37D4018D919C91119792FF45C00C
:1042B0005F968D919D910D90BC91A02D0097A105C9
:1042C000B105D9F180E00E949397C801B701209110
:1042D000FC173091FD174091FE175091FF170F9476
:1042E000EB099B01AC016091FD187091FE18809163
:1042F000FF18909100190F94EC096093FD187093CA
:10430000FE188093FF18909300190E943AAE81E046
:1043100061E041E00E943FAC8CE199E00E94CA3626
:104320004091FD185091FE186091FF18709100198E
:1043300084EC99E022E00E94CB37CA55DF4F4880D9
:1043400059806A807B80C65AD040409205195092AD
:1043500006196092071970920819832D90E015E0F4
:10436000969587951A95E1F781700E949D9CD401DE
:104370008D919C91119792FD02C00C94962A5F96A4
:104380008D919D910D90BC91A02D0297A105B10535
:1043900011F00C94962A80E00E94873B0C94962A98
:1043A00013FD03C0B3E0FB2E02C0F401F3A00091A3
:1043B000281810E0A5E016950795AA95E1F7017079
:1043C00080E00E949D9C6F2D70E0F1E0EF2EF12CBB
:1043D000E622F7227695679561708E2D43E021E005
:1043E0000E94BF9C802F0E949D9C8E2D0C94972A2A
:1043F0008BE299E00E9432364B9902C06CE401C016
:1044000068E484E095E00E94DC68F3D80C949B2A71
:104410008AE399E00E94616280E090E0A0E0B0E071
:104420008093241890932518A0932618B0932718EA
:104430008093201890932118A0932218B0932318EA
:1044400080931C1890931D18A0931E18B0931F18EA
:1044500080E00E949D9C4090051950900619609044
:10446000071970900819C656DF4F488259826A8230
:104470007B82CA59D040FE01319620E333E0F9999E
:10448000FECF32BD21BDF89A80B581932F5F3F4F9B
:1044900043E02433340799F7E980FA800B811C81CB
:1044A000FE01319624E333E0F999FECF32BD21BD00
:1044B000F89A80B581932F5F3F4F53E0283335073B
:1044C00099F729813A814B815C81DE011196E8E4FC
:1044D000F3E0F999FECFF2BDE1BDF89A80B58D9376
:1044E000319683E0EC34F807A1F700D00F92898170
:1044F0009A81AB81BC81EDB7FEB781839283A383A0
:10450000B483C801B7010F2EF0E8EF2EFFE4FF2EB1
:10451000F3EC0F2FF7E41F2FF02D570168010E94D5
:1045200082A10F900F900F900F9081E060E043E028
:1045300020E00E94BF9CCE55DF4F688379838A8339
:104540009B83C25AD04020E030E040E050E00F941E
:10455000B20A87FF01C0EFC7FE01319628E333E0BE
:10456000F999FECF32BD21BDF89A80B581932F5FB6
:104570003F4F43E02C33340799F7E980FA800B81F1
:104580001C81FE0131962CE333E0F999FECF32BD58
:1045900021BDF89A80B581932F5F3F4F53E02034BF
:1045A000350799F729813A814B815C81DE011196AB
:1045B000E8E4F3E0F999FECFF2BDE1BDF89A80B5E9
:1045C0008D93319683E0EC34F807A1F700D00F9279
:1045D00089819A81AB81BC81EDB7FEB781839283DB
:1045E000A383B483C801B7010F2EF0E8EF2EFFE4D8
:1045F000FF2EF3EC0F2FF7E41F2FF02D570168016A
:104600000E9482A10F900F900F900F9080E060E0C9
:1046100043E021E00E94BF9CC256DF4F688379834C
:104620008A839B83CE59D04020E030E040E050E0C8
:104630000F94B20A87FF01C07EC7FE01319620E4C5
:1046400033E0F999FECF32BD21BDF89A80B5819350
:104650002F5F3F4F43E02434340799F7E980FA8015
:104660000B811C81FE01319624E433E0F999FECFE1
:1046700032BD21BDF89A80B581932F5F3F4F53E043
:104680002834350799F729813A814B815C81DE0115
:104690001196E8E4F3E0F999FECFF2BDE1BDF89A96
:1046A00080B58D93319683E0EC34F807A1F700D004
:1046B0000F9289819A81AB81BC81EDB7FEB781836E
:1046C0009283A383B483C801B7010F2EF0E8EF2EC5
:1046D000FFE4FF2EF3EC0F2FF7E41F2FF02D57010F
:1046E00068010E9482A10F900F900F900F9080E0C0
:1046F00061E043E021E00E94BF9C2B013C0120E0EF
:1047000030E040E050E00F94B20A87FD14C7CE5568
:10471000DF4F688179818A819B81C25AD040C2561D
:10472000DF4F288139814A815B81CE59D040830196
:1047300072010E94919920912B1830912C18409170
:104740002D1850912E18CA52DF4F288339834A837F
:104750005B83C65DD04080913F1890914018A09136
:104760004118B0914218CE52DF4F88839983AA83B3
:10477000BB83C25DD04020913318309134184091F2
:10478000351850913618C253DF4F288339834A8336
:104790005B83CE5CD0408091371890913818A091FF
:1047A0003918B0913A18C653DF4F88839983AA838A
:1047B000BB83CA5CD040A090E817B090E917C090C6
:1047C000EA17D090EB172091A4173091A5174091CC
:1047D000A6175091A717CA53DF4F288339834A83FE
:1047E0005B83C65CD04080913B1890913C18A091AF
:1047F0003D18B0913E18CE53DF4F88839983AA832A
:10480000BB83C25CD04020912F183091301840916A
:10481000311850913218C254DF4F288339834A83AC
:104820005B83CE5BD0408091E4179091E517A09117
:10483000E617B091E717C654DF4F88839983AA83A0
:10484000BB83CA5BD0402091A0173091A117409143
:10485000A2175091A317CA54DF4F288339834A8384
:104860005B83C65BD04080E090E0A0E0B0E0809346
:10487000011990930219A0930319B0930419D4015C
:104880008D919C91119792FF11C15F968D919D9191
:104890000D90BC91A02D0097A105B10509F406C1AA
:1048A000CA52DF4F688179818A819B81C65DD04081
:1048B000CE52DF4F288139814A815B81C25DD04071
:1048C0000F94620D7B018C01C253DF4F68817981A7
:1048D0008A819B81CE5CD040C653DF4F28813981CD
:1048E0004A815B81CA5CD0400F94620D9B01AC0190
:1048F000C801B7010F94EB097B018C01C601B5011A
:104900000F94540B9B01AC01C801B7010F94620DC9
:10491000CA53DF4F288139814A815B81C65CD04010
:104920000F94620D5B016C01C253DF4F6881798186
:104930008A819B81CE5CD040CE53DF4F2881398164
:104940004A815B81C25CD0400F94620D7B018C0177
:10495000C254DF4F688179818A819B81CE5BD040D0
:10496000CE52DF4F288139814A815B81C25DD040C0
:104970000F94620D9B01AC01C801B7010F94EB09C4
:104980007B018C01C654DF4F688179818A819B81CC
:10499000CA5BD0400F94540B9B01AC01C801B70116
:1049A0000F94620DCA54DF4F288139814A815B819F
:1049B000C65BD0400F94620D9B01AC01C601B501EE
:1049C0000F94EC097B018C0117FB109517F91095DA
:1049D000C254DF4F688179818A819B81CE5BD04050
:1049E000C653DF4F288139814A815B81CA5CD04040
:1049F0000F94620D5B016C01CA52DF4F68817981AF
:104A00008A819B81C65DD040CE53DF4F288139819A
:104A10004A815B81C25CD0400F94620D9B01AC0166
:104A2000C601B5010F94EB099B01AC01C801B701A8
:104A30000F94B90A9B01AC01C301B2010F94EC09B8
:104A40002091FC173091FD174091FE175091FF17F0
:104A50000F94EB092091FD183091FE184091FF183A
:104A6000509100190F94EC099B01AC01CB01DA01C4
:104A70008093FD189093FE18A093FF18B09300192F
:104A800084EC99E0A901BD0122E00E94CB3781E0CE
:104A90000E949D9CF401878D90A1A1A1B2A10297D3
:104AA000A105B10519F480E00E94873B81E00E94D6
:104AB0009D9C0E943AAE81E00E9493970E94D21979
:104AC00081E061E041E00E943FACC656DF4F488084
:104AD00059806A807B80CA59D04040920519509213
:104AE0000619609207197092081925C51092E217ED
:104AF00022C581E08093E2171EC5C0901C18D0909B
:104B00001D18E0901E18F0901F18609020187090EB
:104B10002118A0902218B0902318209024183090CB
:104B20002518409026185090271803FF23C0D40161
:104B30001A962D913D914D915C911D9780919F17F3
:104B4000882351F0CA01B90123E333E34BEC51E46C
:104B50000F94620D9B01AC01CA01B9012091F417B9
:104B60003091F5174091F6175091F7170F94EB0914
:104B70006B017C0104FF21C0F40126853785408943
:104B8000518980919F17882351F0CA01B90123E30D
:104B900033E34BEC51E40F94620D9B01AC01CA016D
:104BA000B9012091F8173091F9174091FA175091F7
:104BB000FB170F94EB093B015C0105FF23C0D401F7
:104BC00052962D913D914D915C91559780919F17F3
:104BD000882351F0CA01B90123E333E34BEC51E4DC
:104BE0000F94620D9B01AC01CA01B9012091FC1721
:104BF0003091FD174091FE175091FF170F94EB096C
:104C00001B012C01B601C7019301A50171018201AD
:104C10000E947297F401808186FF8DC426893789AE
:104C2000408D518D80919F17882351F0CA01B901A1
:104C300023E333E34BEC51E40F94620D9B01AC0191
:104C4000CA01B9012091EE023091EF024091F002C9
:104C50005091F1020F94620D0F94210B6093F017A5
:104C60007093F1178093F2179093F31764C46091D7
:104C7000F4177091F5178091F6179091F71720911E
:104C8000F8173091F9174091FA175091FB17E090FF
:104C9000FC17F090FD170091FE171091FF17609020
:104CA00005197090061980900719909008190F2E19
:104CB000F0E0AF2EF0E0BF2EF0E0CF2EF0E0DF2EE0
:104CC000F02DA0921119B0921219C0921319D0921E
:104CD0001419A0921519B0921619C0921719D092F2
:104CE000181900D00F92A0900203B0900303C09057
:104CF0000403D0900503ADB7BEB71196AD92BD9237
:104D0000CD92DC9214970F2EF0E8AF2EFFE4BF2E69
:104D1000F3ECCF2EF7E4DF2EF02D0E94F8A960927D
:104D200005197092061980920719909208190F9030
:104D30000F900F900F9080E00E949397FCC380E04B
:104D40000E949D9C80E090E0A0E0B0E080931C1861
:104D500090931D18A0931E18B0931F1880932018CD
:104D600090932118A0932218B093231880932418AD
:104D700090932518A0932618B093271860910A03E2
:104D800070910B0380910C0390910D030E94E7A298
:104D90000091A1181091A2182091A3183091A41885
:104DA000A090A518B090A618C090A718D090A818E9
:104DB00040919D1850919E1860919F187091A01875
:104DC000D601C5017501FA2FEB2FA016B106C20658
:104DD000D3062CF4D901C8017801FA2FEB2FC701B3
:104DE000AF2FBE2F84179507A607B70714F4DB0172
:104DF000CA012C013D01401A510A620A730A83015B
:104E000072012C013D014A185B086C087D086301A2
:104E100052012C013D01441A550A660A770A89EAB3
:104E200096E0B801A7010E94533682EB96E0B601E6
:104E3000A5010E9453368BEB96E0B301A2010E94BC
:104E40005336D4018D919C91119792FF69C15F9661
:104E50008D919D910D90BC91A02D181619061A06E2
:104E60001B060CF05DC12F2D4E2DF999FECF1FBAF8
:104E70008DE793E092BD81BD40BD0FB6F894FA9ADC
:104E8000F99A0FBEF999FECF1FBA8EE793E092BD53
:104E900081BD20BD0FB6F894FA9AF99A0FBE0E9410
:104EA0008242282FF999FECF88E690E092BD81BD1D
:104EB000F89A80B5281769F0F999FECF1FBA88E6ED
:104EC00090E092BD81BD20BD0FB6F894FA9AF99A90
:104ED0000FBE2B2D4A2DF999FECF1FBA8FE793E015
:104EE00092BD81BD40BD0FB6F894FA9AF99A0FBEF3
:104EF000F999FECF1FBA80E893E092BD81BD20BD35
:104F00000FB6F894FA9AF99A0FBE0E948242282F9F
:104F1000F999FECF88E690E092BD81BDF89A80B500
:104F2000281769F0F999FECF1FBA88E690E092BD84
:104F300081BD20BD0FB6F894FA9AF99A0FBE252DBF
:104F4000442DF999FECF1FBA81E893E092BD81BD4F
:104F500040BD0FB6F894FA9AF99A0FBEF999FECFB0
:104F60001FBA82E893E092BD81BD20BD0FB6F894D0
:104F7000FA9AF99A0FBE0E948242282FF999FECF21
:104F800088E690E092BD81BDF89A80B5281709F4B3
:104F9000C7C0F999FECF1FBA88E690E092BD81BDE7
:104FA00020BD0FB6F894FA9AF99A0FBEB9C00091D5
:104FB000281810E075E0169507957A95E1F70170CD
:104FC00080E00E949D9C1092E4171092E5171092C9
:104FD000E6171092E7171092E8171092E91710924F
:104FE000EA171092EB172091DD183091DE184091EE
:104FF000DF185091E0182093EC173093ED17409391
:10500000EE175093EF1780E090E0A0E0B0E08093BF
:105010001C1890931D18A0931E18B0931F1880930E
:10502000201890932118A0932218B09323188093EE
:10503000241890932518A0932618B093271810923F
:10504000D0171092D1171092D2171092D317109236
:10505000D4171092D5171092D6171092D717209305
:10506000D8173093D9174093DA175093DB17609114
:105070000A0370910B0380910C0390910D030E9421
:10508000E7A26091DD187091DE188091DF18909191
:10509000E0180F94540B20E030E040EC5FE30F94F5
:1050A000620D0F94210BAB01BC018091A51890916A
:1050B000A618A091A718B091A8186A017B01C81A78
:1050C000D90AEA0AFB0A80919D1890919E18A09136
:1050D0009F18B091A0184A015B01881A990AAA0A80
:1050E000BB0A8091A1189091A218A091A318B09129
:1050F000A418481B590B6A0B7B0B89EA96E00E94A7
:10510000533682EB96E0B701A6010E9453368BEB33
:1051100096E0B501A4010E945336802F0E949D9C09
:1051200081E061E041E00E943FAC05C212FF14C083
:10513000D4015F964D905D906D907C909297CA5689
:10514000DF4F488259826A827B82C659D04041141F
:1051500051046104710469F462E3462E512C612C00
:10516000712CCA56DF4F488259826A827B82C659A7
:10517000D04081E061E041E00E943FAC8AE399E0E9
:105180000E94616250902818C757DF4F5882C95853
:10519000D04080E00E949D9C209105193091061915
:1051A0004091071950910819CE56DF4F2883398353
:1051B0004A835B83C259D040CA56DF4F68817981E8
:1051C0008A819B81C659D0400F94540BCE54DF4F37
:1051D000688379838A839B83C25BD04028ED33EB5D
:1051E0004DE55FE30F94620D6B017C01CE54DF4F00
:1051F000688179818A819B81C25BD04020E030E068
:1052000040E05FE30F94620D4B015C018E01075B90
:105210001F4F80E4D8011D928A95E9F7A7019601F6
:105220005058D801D0962D933D934D935C93D397CE
:10523000F80120873187428753872401350177FAA7
:10524000709477F870941C964D925D926D927C925A
:105250001F97CA56DF4F688179818A819B81C65921
:10526000D04090958095709561957F4F8F4F9F4F5F
:105270000F94540BF801648B758B868B978BD80138
:105280005896CD92DD92ED92FC925B97448E558EAE
:10529000668E778E9096CD92DD92ED92FC929397EA
:1052A00084A295A2A6A2B7A2CE54DF4F488059800F
:1052B0006A807B80C25BD0409C964D925D926D92DD
:1052C0007C929F9784AA95AAA6AAB7AAC080D180EB
:1052D000E280F3802481358146815781DE01119679
:1052E000E8E4F3E0F999FECFF2BDE1BDF89A80B5AC
:1052F0008D93319683E0EC34F807A1F700D00F923C
:1053000089819A81AB81BC81EDB7FEB7818392839D
:10531000A383B483C701B6010F2EF0E8EF2EFFE49C
:10532000FF2EF3EC0F2FF7E41F2FF02D570168012C
:105330000E9482A10F900F900F900F9081E060E08B
:1053400043E020E00E94BF9C69A77AA78BA79CA797
:10535000CE01875B9F4F58E0852E912C880E991EB9
:105360004DE2442E512C4C0E5D1E3C0138E3232EA1
:10537000312C280E391ED401ED90FD900D911C9119
:10538000139714962D913D914D915C911797DE01E5
:105390001196E8E4F3E0F999FECFF2BDE1BDF89A89
:1053A00080B58D93319683E0EC34F807A1F700D0F7
:1053B0000F9289819A81AB81BC81EDB7FEB7818361
:1053C0009283A383B483C801B7010F2EF0E8EF2EB8
:1053D000FFE4FF2EF3EC0F2FF7E41F2FF02D570102
:1053E00068010E9482A10F900F900F900F9080E0B3
:1053F00060E043E021E00E94BF9CD2016D937D9369
:105400008D939D932D01E8E0F0E08E0E9F1E821497
:10541000930409F0B0CFD301D896ED90FD900D9193
:105420001C91DB97DC962D913D914D915C91DF971E
:10543000DE011196E8E4F3E0F999FECFF2BDE1BD9B
:10544000F89A80B58D93319683E0EC34F807A1F794
:1054500000D00F9289819A81AB81BC81EDB7FEB7F4
:1054600081839283A383B483C801B7010F2EF0E830
:10547000EF2EFFE4FF2EF3EC0F2FF7E41F2FF02D9C
:10548000570168010E9482A10F900F900F900F901A
:1054900080E061E043E021E00E94BF9CFE01EB5B05
:1054A000FF4F608371838283938380E00E94939790
:1054B0006091FD187091FE188091FF18909100196D
:1054C0002091FC173091FD174091FE175091FF1766
:1054D0000F94EB0969A77AA78BA79CA78BE699E0A5
:1054E000BE01675D7F4F48E022E00E94A637CE569E
:1054F000DF4F488059806A807B80C259D0404092FB
:105500000519509206196092071970920819C75729
:10551000DF4F5880C958D040852D90E025E0969502
:1055200087952A95E1F781700E949D9C81E00E94F9
:1055300093970E94D2190F9486036093220570936B
:10554000230580932405909325050C94313501FDA6
:1055500002C00C941F35D40116968D919C9117971B
:105560008537910509F48AC78637910508F091C0FF
:105570008235910509F490C68335910508F040C045
:105580008A31910509F46DC18B319105C0F48631E2
:10559000910509F440C18731910548F484319105A2
:1055A00009F42DC1459711F00C9431352EC1883185
:1055B000910509F449C1499708F04CC132C18032C4
:1055C000910509F499C18132910568F48C319105F6
:1055D00009F471C18C31910508F467C14E9711F03F
:1055E0000C94313575C18035910509F441C681357A
:1055F000910508F04CC68A9711F00C9431358EC194
:105600008936910509F492C28A369105F8F48535F8
:10561000910509F464C68635910550F483359105EA
:1056200009F43DC68435910511F00C9431353BC623
:105630008336910509F4BDC68836910509F4C1C1C8
:105640008C35910511F00C9431356AC68F36910571
:1056500009F4F8C68037910570F48B36910509F48A
:10566000FDC58B36910508F4E7C58D36910511F01F
:105670000C94313565C28337910509F4F6C6843739
:10568000910508F012C58237910511F00C9431355F
:10569000F2C6883E910511F40C94D333893E9105EE
:1056A00008F047C08B3C910509F4B7C78C3C9105C5
:1056B000F8F48C38910509F4FFC18D38910550F448
:1056C0008737910509F4EBC68837910511F00C94E2
:1056D00031350DC7893C910509F413C78A3C910502
:1056E00008F055C78E3B910511F00C94313534C448
:1056F0008F3C910509F4F1C7803D910548F48D3C3C
:10570000910509F4E3C78E3C910508F0E2C798C7FC
:105710008D3D910511F40C94AE338F3D910511F43C
:105720000C94C0338C3D910511F00C9431350C94E0
:105730009E33B1E08E359B0711F40C949134E1E077
:105740008F359E0768F5F1E08F329F0709F440C559
:1057500021E08033920788F48B3F910511F40C947B
:10576000DE3431E08C32930709F410C5893E91058F
:1057700011F00C9431350C94023441E081349407DB
:1057800011F40C94A93451E08234950711F40C946F
:10579000CA348054914011F00C9431350C949534F6
:1057A000B1E0843F9B0711F40C947B34E1E0853F2A
:1057B0009E0798F4F1E081399F0711F40C94453469
:1057C00021E08239920711F40C94483480599140B9
:1057D00011F00C9431350C94423441E0863F94072B
:1057E00011F40C948E3451E0863F950710F40C941C
:1057F0008134875F914011F00C94313567C78DE893
:1058000099E10E9456B70C9431358DE899E10E94D8
:10581000D8BA0C9431358DE899E10E948DB50C947D
:10582000313517FD02C00C9431358DE899E160E007
:105830000E940FC6F40163A974A98DE899E140E0C4
:105840000E94BFB60C9431358DE899E10E94A5B550
:105850000C9431358DE899E160E00E9415BA0C9402
:10586000313512FD02C00C943135D4015F964C9154
:105870005F9790965C91909791966C919197929684
:105880007C918091F719882311F40C943135409361
:10589000EE195093EF196093F0197093F1198DEC94
:1058A00099E10E94AFC30C9431358DE899E10E94D3
:1058B0009AB60C94313517FD02C00C943135F401C1
:1058C00063A974A98DE899E10E945AB60C94313508
:1058D00017FD02C00C9431358DE899E160E00E941B
:1058E0000FC6D401D3966D917C91D4978DE899E140
:1058F0000E940BB60C94313517FD02C00C94313563
:105900008DE899E160E00E940FC6F40163A974A9D3
:105910008DE899E10E94CFB50C94313512FD02C09B
:105920000C94313513FD02C00C943135F401878D90
:1059300090A1A1A1B2A1B7FF02C00C9431358F3F55
:105940009105A105B10519F014F00C94313503A1AE
:1059500014A120E030E0F901EE0FFF1FE95FFD4FD9
:10596000E4918E2F90E08017910711F40C9431355B
:105970002F5F3F4F2833310571F717FF02C00C949A
:105980003135802F61E00F943705802FD4015F9669
:105990006C910F94EA05F401678D70A1802F0F942C
:1059A000590487E095E0B8010E949636D4015F96CD
:1059B0006D917C91909783E195E00E9464360C9400
:1059C00031350E940B54882311F00C9431350F941B
:1059D000860360932205709323058093240590939A
:1059E000250580912E0383FF02C00C943135F4010C
:1059F0008081918193FD0AC092FF0AC0878D90A19A
:105A0000A1A1B2A10097A105B10511F40E948E1CBD
:105A1000D4018D919C91119792FD02C00C94313567
:105A20005F96CD90DD90ED90FC9092979C01207058
:105A3000317091FF1EC05E960C91232B11F410E083
:105A40000FC010E0F401628D738D848D958D20E080
:105A500030E040E050E00F94C00C18160CF411E058
:105A6000C701B6010F94540B402F212F0E945658A6
:105A7000F8C7E0915603F09157030081232B11F4EE
:105A800010E011C010E0D4015A966D917D918D9176
:105A90009C915D9720E030E040E050E00F94C00C16
:105AA00018160CF411E0C701B6010F94540B402FE7
:105AB000212F0E945658D5C70E940B54882309F005
:105AC000D0C70F94860360932205709323058093BB
:105AD00024059093250580912E0383FDC2C7F40110
:105AE0008081918192FFBDC7E78CF0A001A112A136
:105AF00090FD02C0DD2412C0DD24D4015A966D91C0
:105B00007D918D919C915D9720E030E040E050E0E8
:105B10000F94C00C181614F4DD24D394C801B701F7
:105B20000F94540B4D2D0E9494549BC783E01695FF
:105B300007958A95E1F7802F81700E940B1C91C711
:105B40000E940B54882309F08CC70F94860360933E
:105B50002205709323058093240590932505809159
:105B60002E0383FD7EC785E29CE16DE572E040E097
:105B700020E00E9460D585E29CE10E9491F60E949F
:105B80008E1C6090560370905703F4012081318180
:105B900031FF07C0868D882321F418E1612E12E0C1
:105BA000712E32FF27C0D4015F96ED90FD900D91CC
:105BB0001C919297F301C08030FD02C0DD2412C019
:105BC000DD24D4015A966D917D918D919C915D97C4
:105BD00020E030E040E050E00F94C00C181614F4C0
:105BE000DD24D394C801B7010F94540B4C2D2D2DF7
:105BF0000E945658F30166A977A980AD91AD22ADF8
:105C000033AD44AD55AD0F94EB097B018C0120E021
:105C100030E040E050E00F94C00C18165CF4C8016E
:105C2000B70120E030E040E050E40F94B20A88234E
:105C300064F417C7C801B70120E030E040E050EC41
:105C40000F94C00C18160CF40CC79924D301D496E9
:105C50002D913C91D597D2968D919C91D397821797
:105C6000930714F4992493940F948603C257DF4F3B
:105C7000688379838A839B83CE58D040222433243F
:105C8000210110E00F948603C657DF4F68837983A4
:105C90008A839B83CA58D040DC01CB01C257DF4FB7
:105CA000288139814A815B81CE58D040821B930B79
:105CB000A40BB50B895E9340A040B04098F080E003
:105CC0000E940B1CC657DF4F88819981AA81BB8136
:105CD000CA58D040C257DF4F88839983AA83BB83B9
:105CE000CE58D0400E94711C80915603909157036A
:105CF0006816790609F066C0D3019396ED90FC9082
:105D000094971E141F040CF05DC0112309F05AC0B3
:105D1000992009F457C091966D917C9192978827AC
:105D200077FD8095982F0F94540B9B01AC01F301E4
:105D300066A977A980AD91AD0F94C00C18160CF030
:105D400041C000D000D00DB71EB70F5F1F4F6627B0
:105D500077276E197F09882777FD8095982F0F94F4
:105D6000540B2091EE023091EF024091F0025091DD
:105D7000F1020F94620D0F94210B5B016C01F30192
:105D800087859089A189B289F80180839183A28354
:105D9000B3831482158260E070E080E090E020E040
:105DA00030E040E050E0EE24FF2487010E94999605
:105DB00011E02DB73EB72A5F3F4F0FB6F8943EBFB4
:105DC0000FBE2DBF211431044104510409F057C006
:105DD0009920C9F0D301DA966D917D918D919C91B6
:105DE000DD9720E030E040E85FE30F94EB099B0192
:105DF000AC01F30166A977A980AD91AD0F94C00CF9
:105E000087FF1AC03FCFD301DA966D917D918D91B6
:105E10009C91DD9720E030E040E85FE30F94EC09CF
:105E20009B01AC01F30166A977A980AD91AD0F94F8
:105E3000B20A18160CF426CFD3015F966D917C91AF
:105E40009097882777FD8095982F28EE33E040E0E3
:105E500050E00F94380E1B012C01C657DF4F2881EC
:105E600039814A815B81CA58D040220E331E441EBC
:105E7000551E211431044104510409F403CFD20109
:105E8000C101C657DF4F288139814A815B81CA58D9
:105E9000D040821B930BA40BB50B80509449A543B3
:105EA000B74708F4EFCE112309F449C08091560397
:105EB000909157036816790609F041C000D000D0D0
:105EC0000DB71EB70F5F1F4FD30193966D917C9155
:105ED0009497882777FD8095982F0F94540B2091E5
:105EE000EE023091EF024091F0025091F1020F94D6
:105EF000620D0F94210B5B016C01F3018785908982
:105F0000A189B289F80180839183A283B38314822B
:105F1000158260E070E080E090E020E030E040E05A
:105F200050E0EE24FF2487010E9499962DB73EB7DA
:105F30002A5F3F4F0FB6F8943EBF0FBE2DBF1092A1
:105F4000651C0F948603609322057093230580934C
:105F500024059093250585C523FD83C585E29CE135
:105F600061E572E040E020E00E9460D585E29CE1BE
:105F70000E9491F60E948E1CD4018D919C911197E4
:105F800092FF21C05F96ED90FD900D911C9192972C
:105F900090FD02C0DD2410C0DD24F401628D738DFC
:105FA000848D958D20E030E040E050E00F94C00CEF
:105FB000181614F4DD24D394C801B7010F94540BC0
:105FC0004D2D0E949454609195027091960280919B
:105FD0009702909198022091990230919A024091F3
:105FE0009B0250919C020F94EB097B018C0120E0F5
:105FF00030E040E050E00F94C00C18165CF4C8018B
:10600000B70120E030E040E450E40F94B20A882366
:1060100064F427C5C801B70120E030E040E450EC4B
:106020000F94C00C18160CF41CC50F9486037B014A
:106030008C0114C00F9486036E197F09800B910B9D
:10604000695E73408040904038F080E00E940B1CF5
:106050000F9486037B018C010E94711C6091950254
:1060600070919602809197029091980220E030E022
:1060700040E05FE30F94EC092091990230919A027D
:1060800040919B0250919C020F94B20A87FDD2CF9F
:106090001092651C0F94860360932205709323056C
:1060A0008093240590932505DCC423FDDAC40F9466
:1060B00086034B015C010F948603681979098A09EC
:1060C0009B09695E73408040904038F080E00E94F8
:1060D0000B1C0F9486034B015C010E94711CC09045
:1060E000CF02D090D002D6011B96ED90FD900D917D
:1060F0001C911E97C801B70120E030E040EF51E449
:106100000F94C00C1816A4F4C801B701F60127813A
:106110003085418552850F94EB099F7720E030E070
:1061200040E85FE30F94C00C181614F4772402C003
:1061300077247394C090D102D090D202D6011B96DE
:10614000ED90FD900D911C911E97C801B70120E0C4
:1061500030E040EF51E40F94C00C18169CF4C801D5
:10616000B701F60127813085418552850F94EB09EF
:106170009F7720E030E040E85FE30F94C00C1816F2
:106180000CF499CF772009F496CF6BC412FD03C0AD
:1061900061E070E005C0D4015F966D917C919097AD
:1061A00013FD03C008EE13E003C0F40103A114A122
:1061B00085E220E030E040E050E00F94FD06B801B9
:1061C00080E090E00F94940385E20F94890649C41F
:1061D00012FD03C026E930E005C0D4015F962D9181
:1061E0003C91909713FD03C0CC24DD240AC0F40138
:1061F000C3A0D4A0F2E0CF16D1041CF0B2E0CB2EA5
:10620000D12CF601EE0FFF1FE153FD4FE080F1802E
:10621000B901882777FD8095982F0F94540BAB0117
:10622000BC01E3E016950795EA95E1F70170C70117
:106230002C2D0E94FA5415C412FD03C08FEF90E07C
:1062400005C0D4015F968D919C919097612F6695C2
:106250006695669561700E949B1C03C4612F6695CC
:1062600066956695617080E090E00E949B1CF9C382
:106270000E948E1C0F948603609322057093230561
:106280008093240590932505269A2E98EAC30E94B0
:106290008E1C269A2E9AE5C31092E317E2C381E082
:1062A0008093E317DEC312FF14C0F401678D70A161
:1062B00081A192A128EE33E040E050E00F94380E27
:1062C0006093D4027093D5028093D6029093D70244
:1062D000C8C30E948E1C81E00E9486ADC2C312FF1B
:1062E00016C0D4015F966D917D918D919C9192978E
:1062F00028EE33E040E050E00F94380E609326051E
:10630000709327058093280590932905AAC31092BE
:106310002605109227051092280510922905A1C381
:1063200003FF0DC0F40182859385A485B585809314
:10633000E2029093E302A093E402B093E502D40159
:106340008C9184FF0EC01E968D919D910D90BC91F5
:10635000A02D8093E6029093E702A093E802B09309
:10636000E902F401808185FF0CC082899389A489A8
:10637000B5898093EA029093EB02A093EC02B0936C
:10638000ED020E943AAED4018C9186FF6AC3E0917F
:106390005603F091570356962D913D914D915C9186
:1063A0005997218732874387548780810E941B59E0
:1063B00058C312FD07C040E1A42E47E2B42EC12C01
:1063C000D12C0DC0F401678D70A181A192A128EE9E
:1063D00033E040E050E00F94380E5B016C0103FDA8
:1063E0005F9A04FD8A9A05FF05C0809108018160CB
:1063F000809308010F9486037B018C01EA0CFB1C3F
:106400000C1D1D1D02C00E94DCAD0F9486032701E8
:106410003801461A570A680A790AD301C201805A1C
:106420009648A140B04078F3D4013C9133FD5F9889
:1064300034FD8A9835FF15C3809108018E7F8093C3
:1064400008010FC312FF04C0F401878D80932E034F
:1064500080912E0383FF05C360E070E080E090E050
:1064600040E020E00E945658FCC28EE692E084D4C0
:106470000E94081BF6C20E94D219F3C217FFF1C294
:10648000D401D3966D917C91D49785E29CE140E054
:106490000E9491D585E29CE10E9491F6E2C20E94A1
:1064A0008E1C85E295E0DED3649903C08BE195E014
:1064B00002C088E195E0D6D383E395E0D3D3809101
:1064C000030180FD03C08BE195E002C088E195E007
:1064D000C9D381E495E0C6D34A9903C08BE195E026
:1064E00002C088E195E0BED30E94F91ABAC212FF39
:1064F000B8C213FFB6C2F401878D63A10E9491F563
:10650000B0C203FF0DC0F40182859385A485B585D3
:1065100080930E0390930F03A0931003B093110385
:10652000D4018C9184FF0EC01E968D919D910D908B
:10653000BC91A02D8093120390931303A093140396
:10654000B0931503F401808185FF0CC08289938983
:10655000A489B5898093160390931703A093180319
:10656000B0931903D4018C9186FF0EC056968D917D
:106570009D910D90BC91A02D80931A0390931B03C5
:10658000A0931C03B0931D030E943AAE6AC203FF9E
:106590000DC0F40182859385A485B58580931E0383
:1065A00090931F03A0932003B0932103D4018C91F7
:1065B00084FF0EC01E968D919D910D90BC91A02DD3
:1065C0008093220390932303A0932403B093250385
:1065D000F401808185FF0CC082899389A489B589E3
:1065E0008093260390932703A0932803B093290355
:1065F000D4018C9186FF0EC056968D919D910D9081
:10660000BC91A02D80932A0390932B03A0932C037D
:10661000B0932D030E943AAE24C212FF22C2F401AD
:10662000278D30A141A152A112161306140615069A
:106630001CF02093150215C281E08093150211C24F
:10664000809156039091570312FD03C0FC01BF9641
:1066500010C0F401878D90A1A1A1B2A1B7FD01C224
:106660000097A105B10519F4E7E4F2E002C0EEE8F5
:10667000F2E003FF0BC0D4011A962D913D914D918C
:106680005C911D97228F338F448F558FD4018C914D
:1066900084FF0AC01E962D913D914D915C915197BA
:1066A000268F378F40A351A3D4018C9185FF0AC058
:1066B00052962D913D914D915C91559722A333A314
:1066C00044A355A3CF010E943D51CBC10E948543F5
:1066D000C8C1C4010E94C54EC4C103FF0DC0F4016E
:1066E00082859385A485B58580930D1990930E19A5
:1066F000A0930F19B0931019D4018C9186FF11C08B
:10670000E0915603F091570356962D913D914D918E
:106710005C915997278B308F418F528F80810E94D7
:106720001B5940910D1950910E1960910F197091DC
:10673000101988E495E022E02ED493C112FD05C023
:1067400024E630E040E050E005C0F401278D30A1A0
:1067500041A152A1C9010E94701983C112FD05C057
:1067600024E630E040E050E007C0D4015F962D9170
:106770003D914D915C919297C9010E945C1971C144
:1067800012FF6FC18FB7F89420919D1730919E171B
:10679000F401478D50A1240F351F30939E1720938D
:1067A0009D178FBF5EC160912C0570912D0586E508
:1067B00095E0BCD260912A0570912B0585E695E0A5
:1067C000B5D240912E0550912F0560913005709102
:1067D000310587E795E022E0DED310922B05109279
:1067E0002A0510922D0510922C0580E090E0A0E083
:1067F000B0E080932E0590932F05A0933005B093C1
:1068000031052FC104FF0EC020915603309157036C
:10681000F40186859785A089B189F90181A792A79E
:10682000A3A7B4A7E0915603F091570341A552A541
:1068300063A574A58FE895E022E075D3D4018C910F
:1068400083FF0FC020915603309157031A968D9104
:106850009D910D90BC91A02DF90185A396A3A7A3AE
:10686000B0A7E0915603F091570345A156A167A147
:1068700070A589E995E022E056D30E94F91A0E949A
:106880004297EFC00E948E1CECC00E943299E9C072
:1068900010FF08C0D4015A96CD90DD90ED90FC9089
:1068A0005D9708C0C0900519D0900619E0900719AF
:1068B000F0900819B80134E0769567953A95E1F7BC
:1068C0006170A80125E0569547952A95E1F741703A
:1068D000980196E0369527959A95E1F7217083E027
:1068E000169507958A95E1F7802F817087017601CB
:1068F0000E94D8ACB6C080E00AD78EEB9AE055D2A1
:10690000B0C00E94F245E0915603F0915703808198
:106910000E941B598EED9AE048D2A3C00E94624F9C
:10692000A0C08FE392E028D29CC081E00E949D9C91
:10693000F4018081918192FF94C0878D90A1A1A1E3
:10694000B2A10097A105B10509F48BC080E0DFD6A4
:1069500088C080E00E949D9CD4018D919C911197EC
:1069600092FF7FC05F96ED90FD900D911C919297E4
:10697000E114F1040105110509F473C0B3E0EB164D
:10698000F1040105110519F480E00E94469C80E0A5
:10699000BED667C080E00E94469CF4018081918150
:1069A00092FF5FC0878D90A1A1A1B2A10097A10520
:1069B000B10509F456C080E0AAD653C06091FD1815
:1069C0007091FE188091FF18909100192091FC178A
:1069D0003091FD174091FE175091FF170F94EB096E
:1069E0006093FD187093FE188093FF189093001920
:1069F0001092EC171092ED171092EE171092EF17FD
:106A00000E943AAE84EE97E160ED77E10E94078A3A
:106A100080E00E9493974091FD185091FE1860917C
:106A2000FF187091001984EC99E022E0B4D280E064
:106A30006ED680E895E0A0D10E94D21912C011FF55
:106A400008C00E948E1CD4015E968C910E941B5936
:106A500008C022FF06C08DE294E004D1C4010E9468
:106A6000155EC752DF4F0FB6F894DEBF0FBECDBF25
:106A7000CF91DF911F910F91FF90EF90DF90CF901A
:106A8000BF90AF909F908F907F906F905F904F904E
:106A90003F902F900895CF93DF930E94C9630E9487
:106AA000045EEC0185E29CE10E945FD62097D1F064
:106AB0008091F819882381F0888181FF04C08E813C
:106AC0009F814D9791F08DE899E1BE010E94FCB73E
:106AD000CE010E94C56203C0CE010E94C91CCE0136
:106AE0000E94D5620E94DCADD8CF8DE899E10E946A
:106AF0003AB6EECFCF93DF9320C08091F819882368
:106B000081F0888181FF04C08E819F814D9739F18A
:106B10008DE899E1BE010E94FCB7CE010E94C562DA
:106B200003C0CE010E94C91CCE010E94D5620E9402
:106B3000711C85E29CE10E945FD680918B178823AF
:106B400029F40E94045EEC01009771F00E94C96371
:106B500085E29CE10E945FD6209779F6E8CF8DE828
:106B600099E10E943AB6D9CFDF91CF910895CF93A2
:106B7000DF93EC0105C0219684E095E00E94DC687B
:106B800068816623C1F7DF91CF910895AF92BF92DC
:106B9000CF92DF92EF92FF920F931F93DF93CF93E9
:106BA000CDB7DEB72B970FB6F894DEBF0FBECDBFC3
:106BB000C62ED92E1B869BE0A92EB12CAC0EBD1E75
:106BC0006C2D9D2D2AE030E040E050E00F948B0EBC
:106BD000D52E7901042F152F80E3C80EC801B70107
:106BE0002AE030E040E050E00F94380EC61AF5017C
:106BF000C2925F01CE2C7F2D802FE114F10401059C
:106C00001105F1F6CF01B3DF2B960FB6F894DEBF76
:106C10000FBECDBFCF91DF911F910F91FF90EF90ED
:106C2000DF90CF90BF90AF900895EF92FF920F93B7
:106C30001F937B018C0197FF0DC084E095E06DE20E
:106C40000E94DC6810950095F094E094E11CF11C22
:106C5000011D111DC801B70199DF1F910F91FF9010
:106C6000EF900895CF93DF93EC0104C084E095E0AA
:106C70000E94DC68FE01649121966623B9F7DF91DA
:106C8000CF910895EF92FF920F931F937A018B019A
:106C9000E9DFC801B7017ADF0E94F91A1F910F914D
:106CA000FF90EF900895EF92FF920F931F937A0158
:106CB0008B01D8DFC801B701B8DF0E94F91A1F9114
:106CC0000F91FF90EF900895EF92FF920F931F9313
:106CD0007B01C8DF0027F7FC0095102FC801B70122
:106CE000A4DF0E94F91A1F910F91FF90EF90089571
:106CF000EF92FF920F931F937A018B01B3DFC801CC
:106D0000B70144DF1F910F91FF90EF900895EF922C
:106D1000FF920F931F937A018B01A4DFC801B70183
:106D200084DF1F910F91FF90EF900895EF92FF92F3
:106D30000F931F937B0196DF0027F7FC0095102F20
:106D4000C801B70172DF1F910F91FF90EF90089576
:106D50000F931F938B0186DFC80109DF1F910F91ED
:106D600008950F931F938B017DDFC80100DF0E9400
:106D7000F91A1F910F91089575DF0C94F91A0F936A
:106D80001F938C0188E293E06DDFC801F5DF1F914E
:106D90000F9108950F931F938C018FE293E062DFB0
:106DA000C801EADF1F910F9108950F931F938C0183
:106DB0008FE293E057DFC80155DF1F910F910895CF
:106DC0000F931F938C0185E393E04CDFC801D4DF60
:106DD0001F910F9108959F92AF92BF92CF92DF9231
:106DE000EF92FF920F931F93CF93DF937B018C0160
:106DF000942EA80197010F941C0E882319F080E2AD
:106E000093E020C0C0E0D0E057016801E894D7F8D3
:106E1000C601B5012FEF3FEF4FE75FE70F941C0E60
:106E2000882351F4C601B5012FEF3FEF4FE75FE72D
:106E30000F94B20A181614F0C1E0D0E0219721F0A7
:106E400084E293E00FDF63C0C801B70120E030E0C7
:106E500040E050E00F94B20A88234CF484E095E0BF
:106E60006DE20E94DC6817FB109517F9109520E081
:106E700030E040E05FE3DD240BC0CA01B90120E04F
:106E800030E040E251E40F94B90A9B01AC01D39485
:106E9000D91498F3C801B7010F94EC095B016C0198
:106EA0000F94260B7B018C0171DE992029F084E080
:106EB00095E06EE20E94DC68C801B7010F94520BA6
:106EC0009B01AC01C601B5010F94EB091EC020E087
:106ED00030E040E251E40F94620D7B018C010F948D
:106EE000210B5B016C01CC24B7FCC094DC2CC601E7
:106EF000B5019BDEC601B5010F94540B9B01AC019B
:106F0000C801B7010F94EB099A94992001F7DF911A
:106F1000CF911F910F91FF90EF90DF90CF90BF9096
:106F2000AF909F900895DF92EF92FF920F931F937F
:106F30007A018B01D22E96DEC801B7014D2D4BDFB1
:106F40001F910F91FF90EF90DF900895EF92FF92C5
:106F50000F931F93CF93DF93162F072FE42EF22E5C
:106F600081DE212F302FC901EC0110E009C04991C9
:106F70005991699179918AEE94E02F2DD4DF1F5FAA
:106F80001E15A8F30E94F91ADF91CF911F910F915E
:106F9000FF90EF900895DF92EF92FF920F931F936F
:106FA0007A018B01D22E5EDEC801B7014D2D13DFB1
:106FB0000E94F91A1F910F91FF90EF90DF900895B2
:106FC000F999FECF1FBA92BD81BD60BD0FB6F8948E
:106FD000FA9AF99A0FBEF999FECF1FBA019692BD9F
:106FE00081BD70BD0FB6F894FA9AF99A0FBE089554
:106FF000F999FECF1FBA92BD81BD40BD0FB6F8947E
:10700000FA9AF99A0FBEF999FECF1FBA019692BD6E
:1070100081BD019750BD0FB6F894FA9AF99A0FBE48
:10702000F999FECF1FBA029692BD81BD029760BD4D
:107030000FB6F894FA9AF99A0FBEF999FECF1FBAD3
:10704000039692BD81BD70BD0FB6F894FA9AF99A75
:107050000FBE0895F999FECF92BD81BDF89A60B533
:10706000F999FECF019692BD81BD0197F89A70B54E
:10707000F999FECF029692BD81BD0297F89A20B58C
:10708000F999FECF039692BD81BDF89A90B5822FF3
:107090000895DF93CF9300D00F92CDB7DEB780E095
:1070A00090E0A0E0B0E089839A83AB83BC83FE01CB
:1070B000319688E293E0AE014B5F5F4F0EC02081B6
:1070C000F999FECF31961FBA92BD81BD20BD0FB692
:1070D000F894FA9AF99A0FBE0196E417F50779F732
:1070E00080E090E0A0EAB0E489839A83AB83BC831C
:1070F000FE0131968CE293E0AE014B5F5F4F0EC014
:107100002081F999FECF31961FBA92BD81BD20BD75
:107110000FB6F894FA9AF99A0FBE0196E417F5079C
:1071200079F780E090E0A0E2B2E489839A83AB83B0
:10713000BC83FE01319688E493E0AE014B5F5F4F64
:107140000EC02081F999FECF31961FBA92BD81BD44
:1071500020BD0FB6F894FA9AF99A0FBE0196E4177B
:10716000F50779F780E090E0A0E0B0E089839A83AA
:10717000AB83BC83FE01319680E293E0AE014B5FAE
:107180005F4F0EC02081F999FECF31961FBA92BD94
:1071900081BD20BD0FB6F894FA9AF99A0FBE0196F8
:1071A000E417F50779F780E090E0A0E0B0E089838C
:1071B0009A83AB83BC83FE01319684E293E0AE01F7
:1071C0004B5F5F4F0EC02081F999FECF31961FBAF9
:1071D00092BD81BD20BD0FB6F894FA9AF99A0FBE00
:1071E0000196E417F50779F780E090E0A0E5B2ECAE
:1071F00089839A83AB83BC83FE01319680E393E05D
:10720000AE014B5F5F4F0EC02081F999FECF3196E2
:107210001FBA92BD81BD20BD0FB6F894FA9AF99AB3
:107220000FBE0196E417F50779F780E090E0A0EF34
:10723000B1EC89839A83AB83BC83FE01319684E3EE
:1072400093E0AE014B5F5F4F0EC02081F999FECFF6
:1072500031961FBA92BD81BD20BD0FB6F894FA9A3F
:10726000F99A0FBE0196E417F50779F780E090E0F0
:10727000A0E5B2E489839A83AB83BC83FE01319697
:1072800088E393E0AE014B5F5F4F0EC02081F99918
:10729000FECF31961FBA92BD81BD20BD0FB6F894C6
:1072A000FA9AF99A0FBE0196E417F50779F780E08C
:1072B00090E0A0EFB1EC89839A83AB83BC83FE019D
:1072C00031968CE393E0AE014B5F5F4F0EC020819F
:1072D000F999FECF31961FBA92BD81BD20BD0FB680
:1072E000F894FA9AF99A0FBE0196E417F50779F720
:1072F00080E090E0A0E0B0E089839A83AB83BC8318
:10730000FE01319680E493E0AE014B5F5F4F0EC00B
:107310002081F999FECF31961FBA92BD81BD20BD63
:107320000FB6F894FA9AF99A0FBE0196E417F5078A
:1073300079F780E090E0A0E7B2E489839A83AB8399
:10734000BC83FE01319684E493E0AE014B5F5F4F56
:107350000EC02081F999FECF31961FBA92BD81BD32
:1073600020BD0FB6F894FA9AF99A0FBE0196E41769
:10737000F50779F780E090E0A0EAB0E489839A838A
:10738000AB83BC83FE01319681EA93E0AE014B5F93
:107390005F4F0EC02081F999FECF31961FBA92BD82
:1073A00081BD20BD0FB6F894FA9AF99A0FBE0196E6
:1073B000E417F50779F780E090E0A9E5B3E4898365
:1073C0009A83AB83BC83FE01319681E793E0AE01E3
:1073D0004B5F5F4F0EC02081F999FECF31961FBAE7
:1073E00092BD81BD20BD0FB6F894FA9AF99A0FBEEE
:1073F0000196E417F50779F780E090E0A8ECB2E495
:1074000089839A83AB83BC83FE01319685E793E041
:10741000AE014B5F5F4F0EC02081F999FECF3196D0
:107420001FBA92BD81BD20BD0FB6F894FA9AF99AA1
:107430000FBE0196E417F50779F789E793E064EB4F
:1074400070E0BEDD8BE793E066E470E0B9DD8DE7C8
:1074500093E064E670E0B4DD8FE793E064E670E00B
:10746000AFDD81E893E064E670E0AADD80E090E0C3
:10747000A2E5B3E489839A83AB83BC83FE01319692
:1074800085E893E0AE014B5F5F4F0EC02081F99914
:10749000FECF31961FBA92BD81BD20BD0FB6F894C4
:1074A000FA9AF99A0FBE0196E417F50779F780E08A
:1074B00090E0A5EAB3E489839A83AB83BC83FE01A1
:1074C000319689E893E0AE014B5F5F4F0EC020819B
:1074D000F999FECF31961FBA92BD81BD20BD0FB67E
:1074E000F894FA9AF99A0FBE0196E417F50779F71E
:1074F00080E090E0A4EBB2E489839A83AB83BC8301
:10750000FE0131968DE893E0AE014B5F5F4F0EC0F8
:107510002081F999FECF31961FBA92BD81BD20BD61
:107520000FB6F894FA9AF99A0FBE0196E417F50788
:1075300079F780E090E0A0E0B0E089839A83AB83A4
:10754000BC83FE01319681E993E0AE014B5F5F4F52
:107550000EC02081F999FECF31961FBA92BD81BD30
:1075600020BD0FB6F894FA9AF99A0FBE0196E41767
:10757000F50779F780E090E0A0E0B0E089839A8396
:10758000AB83BC83FE01319685E993E0AE014B5F8E
:107590005F4F0EC02081F999FECF31961FBA92BD80
:1075A00081BD20BD0FB6F894FA9AF99A0FBE0196E4
:1075B000E417F50779F780E090E0A0E0B0E0898378
:1075C0009A83AB83BC83FE01319689E993E0AE01D7
:1075D0004B5F5F4F0EC02081F999FECF31961FBAE5
:1075E00092BD81BD20BD0FB6F894FA9AF99A0FBEEC
:1075F0000196E417F50779F780E090E0A8ECB2E493
:1076000089839A83AB83BC83FE0131968DE993E035
:10761000AE014B5F5F4F0EC02081F999FECF3196CE
:107620001FBA92BD81BD20BD0FB6F894FA9AF99A9F
:107630000FBE0196E417F50779F780E090E0A0E02F
:10764000B0E089839A83AB83BC83FE01319685EADF
:1076500093E0AE014B5F5F4F0EC02081F999FECFE2
:1076600031961FBA92BD81BD20BD0FB6F894FA9A2B
:10767000F99A0FBE0196E417F50779F780E090E0DC
:10768000A0E0B0E089839A83AB83BC83FE0131968E
:1076900089EA93E0AE014B5F5F4F0EC02081F999FC
:1076A000FECF31961FBA92BD81BD20BD0FB6F894B2
:1076B000FA9AF99A0FBE0196E417F50779F780E078
:1076C00090E0A0E0B0E089839A83AB83BC83FE01A5
:1076D00031968DEA93E0AE014B5F5F4F0EC0208183
:1076E000F999FECF31961FBA92BD81BD20BD0FB66C
:1076F000F894FA9AF99A0FBE0196E417F50779F70C
:107700000F900F900F900F90CF91DF910895DF921F
:10771000EF92FF920F931F93DF93CF9300D00F92BE
:10772000CDB7DEB7D82E4091D8025091D9026091E2
:10773000DA027091DB028BE490E05ADC409126057E
:107740005091270560912805709129058FE490E0FC
:107750004FDC4091D4025091D5026091D6027091D5
:10776000D70283E590E044DC8091E2029091E3024D
:10777000A091E402B091E50289839A83AB83BC8334
:10778000FE01319683E090E0AE014B5F5F4F0EC08B
:107790002081F999FECF31961FBA92BD81BD20BDDF
:1077A0000FB6F894FA9AF99A0FBE0196E417F50706
:1077B00079F78091E6029091E702A091E802B091FA
:1077C000E90289839A83AB83BC83FE01319687E00B
:1077D00090E0AE014B5F5F4F0EC02081F999FECF64
:1077E00031961FBA92BD81BD20BD0FB6F894FA9AAA
:1077F000F99A0FBE0196E417F50779F78091EA022E
:107800009091EB02A091EC02B091ED0289839A83F2
:10781000AB83BC83FE0131968BE090E0AE014B5F01
:107820005F4F0EC02081F999FECF31961FBA92BDED
:1078300081BD20BD0FB6F894FA9AF99A0FBE019651
:10784000E417F50779F78091F2029091F302A09185
:10785000F402B091F50289839A83AB83BC83FE0165
:1078600031968FE090E0AE014B5F5F4F0EC02081FC
:10787000F999FECF31961FBA92BD81BD20BD0FB6DA
:10788000F894FA9AF99A0FBE0196E417F50779F77A
:107890008091F6029091F702A091F802B091F9025E
:1078A00089839A83AB83BC83FE01319683E190E0A8
:1078B000AE014B5F5F4F0EC02081F999FECF31962C
:1078C0001FBA92BD81BD20BD0FB6F894FA9AF99AFD
:1078D0000FBE0196E417F50779F78091FA029091AF
:1078E000FB02A091FC02B091FD0289839A83AB83D5
:1078F000BC83FE01319687E190E0AE014B5F5F4FA4
:107900000EC02081F999FECF31961FBA92BD81BD7C
:1079100020BD0FB6F894FA9AF99A0FBE0196E417B3
:10792000F50779F78091020390910303A091040376
:10793000B091050389839A83AB83BC83FE013196A2
:107940008BE190E0AE014B5F5F4F0EC02081F99953
:10795000FECF31961FBA92BD81BD20BD0FB6F894FF
:10796000FA9AF99A0FBE0196E417F50779F7809114
:10797000060390910703A0910803B091090389833E
:107980009A83AB83BC83FE0131968FE190E0AE0118
:107990004B5F5F4F0EC02081F999FECF31961FBA21
:1079A00092BD81BD20BD0FB6F894FA9AF99A0FBE28
:1079B0000196E417F50779F780910A0390910B037C
:1079C000A0910C03B0910D0389839A83AB83BC8390
:1079D000FE01319683E290E0AE014B5F5F4F0EC037
:1079E0002081F999FECF31961FBA92BD81BD20BD8D
:1079F0000FB6F894FA9AF99A0FBE0196E417F507B4
:107A000079F780910D1990910E19A0910F19B091ED
:107A1000101989839A83AB83BC83FE01319687E278
:107A200090E0AE014B5F5F4F0EC02081F999FECF11
:107A300031961FBA92BD81BD20BD0FB6F894FA9A57
:107A4000F99A0FBE0196E417F50779F780910E03B6
:107A500090910F03A0911003B091110389839A8331
:107A6000AB83BC83FE01319683E390E0AE014B5FB4
:107A70005F4F0EC02081F999FECF31961FBA92BD9B
:107A800081BD20BD0FB6F894FA9AF99A0FBE0196FF
:107A9000E417F50779F78091120390911303A091F1
:107AA0001403B091150389839A83AB83BC83FE01D1
:107AB000319687E390E0AE014B5F5F4F0EC02081AF
:107AC000F999FECF31961FBA92BD81BD20BD0FB688
:107AD000F894FA9AF99A0FBE0196E417F50779F728
:107AE0008091160390911703A0911803B091190388
:107AF00089839A83AB83BC83FE0131968BE390E04C
:107B0000AE014B5F5F4F0EC02081F999FECF3196D9
:107B10001FBA92BD81BD20BD0FB6F894FA9AF99AAA
:107B20000FBE0196E417F50779F780911E03909137
:107B30001F03A0912003B091210389839A83AB8313
:107B4000BC83FE0131968FE390E0AE014B5F5F4F47
:107B50000EC02081F999FECF31961FBA92BD81BD2A
:107B600020BD0FB6F894FA9AF99A0FBE0196E41761
:107B7000F50779F78091220390912303A0912403C4
:107B8000B091250389839A83AB83BC83FE01319630
:107B900083E490E0AE014B5F5F4F0EC02081F99906
:107BA000FECF31961FBA92BD81BD20BD0FB6F894AD
:107BB000FA9AF99A0FBE0196E417F50779F78091C2
:107BC000260390912703A0912803B091290389836C
:107BD0009A83AB83BC83FE01319687E490E0AE01CB
:107BE0004B5F5F4F0EC02081F999FECF31961FBACF
:107BF00092BD81BD20BD0FB6F894FA9AF99A0FBED6
:107C00000196E417F50779F72091A102F999FECFC3
:107C10001FBA8AE690E092BD81BD20BD0FB6F894F0
:107C2000FA9AF99A0FBE2091A602F999FECF1FBACF
:107C30008BE690E092BD81BD20BD0FB6F894FA9A14
:107C4000F99A0FBE2091A702F999FECF1FBA8CE7CF
:107C500090E092BD81BD20BD0FB6F894FA9AF99AD2
:107C60000FBE8091A8029091A902A091AA02B091A2
:107C7000AB0289839A83AB83BC83FE0131968CE689
:107C800090E0AE014B5F5F4F0EC02081F999FECFAF
:107C900031961FBA92BD81BD20BD0FB6F894FA9AF5
:107CA000F99A0FBE0196E417F50779F78091AC02B7
:107CB0009091AD02A091AE02B091AF0289839A83F8
:107CC000AB83BC83FE01319680E790E0AE014B5F51
:107CD0005F4F0EC02081F999FECF31961FBA92BD39
:107CE00081BD20BD0FB6F894FA9AF99A0FBE01969D
:107CF000E417F50779F78091B0029091B102A09155
:107D0000B202B091B30289839A83AB83BC83FE0134
:107D1000319684E790E0AE014B5F5F4F0EC020814B
:107D2000F999FECF31961FBA92BD81BD20BD0FB625
:107D3000F894FA9AF99A0FBE0196E417F50779F7C5
:107D40002091B402F999FECF1FBA88E790E092BD66
:107D500081BD20BD0FB6F894FA9AF99A0FBE8091B2
:107D6000F1189091F218A091F318B091F41889834A
:107D70009A83AB83BC83FE01319685E890E0AE0127
:107D80004B5F5F4F0EC02081F999FECF31961FBA2D
:107D900092BD81BD20BD0FB6F894FA9AF99A0FBE34
:107DA0000196E417F50779F78091F9189091FA1880
:107DB000A091FB18B091FC1889839A83AB83BC8394
:107DC000FE01319689E890E0AE014B5F5F4F0EC037
:107DD0002081F999FECF31961FBA92BD81BD20BD99
:107DE0000FB6F894FA9AF99A0FBE0196E417F507C0
:107DF00079F78091011990910219A0910319B0911E
:107E0000041989839A83AB83BC83FE0131968DE884
:107E100090E0AE014B5F5F4F0EC02081F999FECF1D
:107E200031961FBA92BD81BD20BD0FB6F894FA9A63
:107E3000F99A0FBE0196E417F50779F78091ED18CE
:107E40009091EE18A091EF18B091F01889839A8361
:107E5000AB83BC83FE01319681E990E0AE014B5FBC
:107E60005F4F0EC02081F999FECF31961FBA92BDA7
:107E700081BD20BD0FB6F894FA9AF99A0FBE01960B
:107E8000E417F50779F78091F5189091F618A0910D
:107E9000F718B091F81889839A83AB83BC83FE01ED
:107EA000319685E990E0AE014B5F5F4F0EC02081B7
:107EB000F999FECF31961FBA92BD81BD20BD0FB694
:107EC000F894FA9AF99A0FBE0196E417F50779F734
:107ED0008091FD189091FE18A091FF18B0910019A3
:107EE00089839A83AB83BC83FE01319689E990E054
:107EF000AE014B5F5F4F0EC02081F999FECF3196E6
:107F00001FBA92BD81BD20BD0FB6F894FA9AF99AB6
:107F10000FBE0196E417F50779F780E090E0A0E046
:107F2000B0E089839A83AB83BC83FE0131968DE9EF
:107F300090E0AE014B5F5F4F0EC02081F999FECFFC
:107F400031961FBA92BD81BD20BD0FB6F894FA9A42
:107F5000F99A0FBE0196E417F50779F780E090E0F3
:107F6000A0E0B0E089839A83AB83BC83FE013196A5
:107F700081EA90E0AE014B5F5F4F0EC02081F9991E
:107F8000FECF31961FBA92BD81BD20BD0FB6F894C9
:107F9000FA9AF99A0FBE0196E417F50779F780E08F
:107FA00090E0A0E0B0E089839A83AB83BC83FE01BC
:107FB000319685EA90E0AE014B5F5F4F0EC02081A5
:107FC000F999FECF31961FBA92BD81BD20BD0FB683
:107FD000F894FA9AF99A0FBE0196E417F50779F723
:107FE00020912818F999FECF1FBA80E793E092BD3F
:107FF00081BD822F90E025E0969587952A95E1F73F
:10800000817080BD0FB6F894FA9AF99A0FBE6BE2B0
:1080100078E140E050E07E010894E11CF11C8E0103
:108020000B5F1F4F9A01220F331F220F331F245B58
:108030003C4FFB0180819181A281B38189839A8326
:10804000AB83BC83F7010FC08081F999FECF3196D5
:108050001FBA32BD21BD80BD0FB6F894FA9AF99AC5
:108060000FBE2F5F3F4FE017F10771F74F5F5F4F74
:108070006C5F7F4F49305105A9F6A8958091210288
:1080800090912202A0912302B091240289839A83C5
:10809000AB83BC83FE01319688EC90E0AE014B5F70
:1080A0005F4F0EC02081F999FECF31961FBA92BD65
:1080B00081BD20BD0FB6F894FA9AF99A0FBE0196C9
:1080C000E417F50779F78091270290912802A09193
:1080D0002902B0912A0289839A83AB83BC83FE0173
:1080E00031968CEC90E0AE014B5F5F4F0EC020816B
:1080F000F999FECF31961FBA92BD81BD20BD0FB652
:10810000F894FA9AF99A0FBE0196E417F50779F7F1
:1081100080912F0290913002A0913102B0913202F1
:1081200089839A83AB83BC83FE01319680ED90E016
:10813000AE014B5F5F4F0EC02081F999FECF3196A3
:108140001FBA92BD81BD20BD0FB6F894FA9AF99A74
:108150000FBE0196E417F50779F780912B029091F5
:108160002C02A0912D02B0912E0289839A83AB83B9
:10817000BC83FE01319684ED90E0AE014B5F5F4F12
:108180000EC02081F999FECF31961FBA92BD81BDF4
:1081900020BD0FB6F894FA9AF99A0FBE0196E4172B
:1081A000F50779F720915A02F999FECF1FBA88EDA9
:1081B00090E092BD81BD20BD0FB6F894FA9AF99A6D
:1081C0000FBE20915F02F999FECF1FBA89ED90E0B2
:1081D00092BD81BD20BD0FB6F894FA9AF99A0FBEF0
:1081E00020916002F999FECF1FBA85EF90E092BD11
:1081F00081BD20BD0FB6F894FA9AF99A0FBE80910E
:10820000610290916202A0916302B091640289833D
:108210009A83AB83BC83FE0131968AED90E0AE0178
:108220004B5F5F4F0EC02081F999FECF31961FBA88
:1082300092BD81BD20BD0FB6F894FA9AF99A0FBE8F
:108240000196E417F50779F780916502909166022F
:10825000A0916702B091680289839A83AB83BC8343
:10826000FE0131968EED90E0AE014B5F5F4F0EC088
:108270002081F999FECF31961FBA92BD81BD20BDF4
:108280000FB6F894FA9AF99A0FBE0196E417F5071B
:1082900079F78091690290916A02A0916B02B09186
:1082A0006C0289839A83AB83BC83FE01319682EE94
:1082B00090E0AE014B5F5F4F0EC02081F999FECF79
:1082C00031961FBA92BD81BD20BD0FB6F894FA9ABF
:1082D000F99A0FBE0196E417F50779F720916D0220
:1082E000F999FECF1FBA86EE90E092BD81BD20BD08
:1082F0000FB6F894FA9AF99A0FBE4091190250916C
:108300001A0260911B0270911C0287EE90E00E949D
:10831000F83740911D0250911E0260911F0270912A
:1083200020028BEE90E00E94F83760913702709146
:1083300038028FEE90E00E94E03760913902709130
:108340003A028AEF90E00E94E03760913B02709120
:108350003C028CEF90E00E94E03720918C02F9996A
:10836000FECF1FBA8EEF90E092BD81BD20BD0FB64B
:10837000F894FA9AF99A0FBE80913D0290913E02CC
:10838000A0913F02B091400289839A83AB83BC8362
:10839000FE01319681EF90E0AE014B5F5F4F0EC062
:1083A0002081F999FECF31961FBA92BD81BD20BDC3
:1083B0000FB6F894FA9AF99A0FBE0196E417F507EA
:1083C00079F78091410290914202A0914302B091CD
:1083D000440289839A83AB83BC83FE01319686EF86
:1083E00090E0AE014B5F5F4F0EC02081F999FECF48
:1083F00031961FBA92BD81BD20BD0FB6F894FA9A8E
:10840000F99A0FBE0196E417F50779F7DD2059F1C7
:108410008DE790E040E050E060E070E00E94F837C7
:1084200080E090E0A0E0B0E089839A83AB83BC83D6
:10843000FE01319681E890E0AE014B5F5F4F0EC0C8
:108440002081F999FECF31961FBA92BD81BD20BD22
:108450000FB6F894FA9AF99A0FBE0196E417F50749
:1084600079F70E944938F999FECF1FBA89E690E062
:1084700092BD81BD87E080BD0FB6F894FA9AF99A53
:108480000FBE20E030E040E02836310539F0F999A0
:10849000FECF32BD21BDF89A80B5480F2F5F3F4F08
:1084A000F8E020303F0781F7F999FECF1FBA88E640
:1084B00090E092BD81BD40BD0FB6F894FA9AF99A4A
:1084C0000FBE0F900F900F900F90CF91DF911F91E3
:1084D0000F91FF90EF90DF900895F999FECF12BCB5
:1084E00011BCF89A80B5823061F48BE490E00E9470
:1084F0002A386093D8027093D9028093DA0290935D
:10850000DB02089520E030E090E02836310539F0B4
:10851000F999FECF32BD21BDF89A80B5980F2F5F33
:108520003F4F88E02030380781F7892F0895885C15
:10853000904022E08835920778F464E670E00F946A
:10854000640E6F5F7F4F85E49BE00E94963684E067
:1085500095E060E20C94DC6808950F931F93CF932D
:10856000DF93EC018B018BE49BE0BE010E94963609
:1085700084E095E060E20E94DC68F999FECFD2BD0C
:10858000C1BDF89A60B570E0882777FD8095982F77
:108590000E94153684E095E060E20E94DC68CE011E
:1085A000C6DFC8010E94BC36DF91CF911F910F91A9
:1085B00008950F931F93CF93DF93EC018B0182E516
:1085C0009BE0BE010E94963684E095E060E20E9446
:1085D000DC68F999FECFD2BDC1BDF89A80B5F99992
:1085E000FECF2196D2BDC1BD2197F89A20B5682F44
:1085F000722F882777FD8095982F0E94153684E08A
:1086000095E060E20E94DC68CE0191DFC8010E9423
:10861000BC36DF91CF911F910F910895CF92DF92D9
:10862000EF92FF920F931F938C016B0189E59BE002
:10863000B8010E94963634E0E32E35E0F32EC701F0
:1086400060E20E94DC68C8010E942A380E94153648
:10865000C70160E20E94DC68C80169DFC6010E94B0
:10866000BC361F910F91FF90EF90DF90CF9008954F
:10867000DF92EF92FF920F931F93DF93CF9300D07F
:108680000F92CDB7DEB7182F092F7B01D42E80E6CD
:108690009BE0612F702F0E94963684E095E060E2A7
:1086A0000E94DC68812F902F9C01FE013196AE0163
:1086B0004B5F5F4F09C0F999FECF32BD21BDF89ADB
:1086C00080B581932F5F3F4FE417F507A1F76981CC
:1086D0007A818B819C814D2D0E94EB3684E095E060
:1086E00060E20E94DC68812F902F21DFC7010E9489
:1086F000BC360F900F900F900F90CF91DF911F918C
:108700000F91FF90EF90DF9008958BE490E067E683
:108710007BE084DF81E890E060E77BE043E0A8DF76
:108720008DE790E065E87BE079DF8FE490E068E931
:108730007BE074DF83E590E066EB7BE06FDF8BE04E
:1087400090E069EB7CE044E093DF87E190E066EC49
:108750007CE043E08DDF83E290E06BED7CE043E082
:1087600087DF87E290E065E77CE043E081DF85E832
:1087700090E06FED7BE043E07BDF89E890E06FEE17
:108780007BE043E075DF8DE890E06FEF7BE043E056
:108790006FDF81E990E06FE07CE043E069DF85E92D
:1087A00090E061E27CE043E063DF89E990E063E32D
:1087B0007CE043E05DDF8BE390E066E87CE043E053
:1087C00057DF87E490E06CE97CE043E051DF81E72C
:1087D00093E062EF7CE043E04BDF85E793E06BE002
:1087E0007DE043E045DF8DE993E06DEA7DE043E025
:1087F0003FDF8BE793E06AE37DE0DBDE89E793E030
:1088000062E27DE0D6DE8DE793E060E57DE0D1DEDB
:108810008FE793E06FE67DE0CCDE81E893E06EE8E1
:108820007DE0C7DE85E893E064EC76E043E020DF9E
:1088300089E893E062ED76E043E01ADF8DE893E0AB
:1088400060EE76E043E014DF81E993E06DEE76E0E0
:1088500043E00EDF85E993E060E077E043E008DF86
:1088600089E993E063E177E043E002DF85EA93E0A2
:108870006EEB7DE043E0FCDE89EA93E064ED7DE0B1
:1088800043E0F6DE8DEA93E06AEE7DE043E0F0DE61
:1088900088E293E069ED79E043E0EADE81EA93E083
:1088A0006DEE79E043E0E4DE8CE293E067E37AE0AA
:1088B00043E0DEDE88E493E06CE47AE043E0D8DE77
:1088C00080E293E06BE07AE043E0D2DE84E293E082
:1088D00061E27AE043E0CCDE80E393E065E67AE0B3
:1088E00043E0C6DE84E393E060E77AE043E0C0DE85
:1088F00088E393E06BE77AE043E0BADE8CE393E051
:1089000066E87AE043E0B4DE80E493E061E97AE08F
:1089100043E0AEDE84E493E06CE97AE043E0A8DE75
:1089200080E793E067EA7AE018DE8AE690E06DEA95
:108930007EE013DE8BE690E064EC7EE00EDE8CE7FA
:1089400090E066ED7EE009DE8CE690E068EE7EE089
:1089500043E08EDE80E790E067EF7EE043E088DE74
:1089600084E790E066E07FE043E082DE88E790E025
:1089700065E17FE0F2DD88EC90E06FE27FE043E0CC
:1089800077DE8CEC90E06CE37FE043E071DE80ED1D
:1089900090E061E57FE043E06BDE84ED90E067E628
:1089A0007FE043E065DE88ED90E06DE77FE0D5DDB8
:1089B00089ED90E060E97FE0D0DD85EF90E06EE941
:1089C0007FE0CBDD8AED90E06CEA7FE044E050DEB2
:1089D0008EED90E061EC7FE044E04ADE82EE90E0D4
:1089E0006CEC7FE044E044DE86EE90E067ED7FE0F3
:1089F000B4DD87EE90E06DEE7FE010DE8BEE90E070
:108A00006EEF7FE00BDE8FEE90E06FE070E1D1DD86
:108A10008AEF90E068E270E1CCDD8CEF90E06EE4EC
:108A200070E1C7DD8EEF90E064E770E196DD81EFE5
:108A300090E062E970E143E01BDE86EF90E064EADB
:108A400070E143E015CEEF92FF920F931F93DF93F7
:108A5000CF9300D00F92CDB7DEB760911F19709100
:108A60002019809121199091221920E030E040E0F6
:108A700050E00F94B20A882309F4A9C00F9486032A
:108A800020911B1930911C1940911D1950911E19EC
:108A9000621B730B840B950B28EE33E040E050E033
:108AA0000F948B0E79018A018DE790E00E942A389D
:108AB000E60EF71E081F191F8DE790E0B801A70109
:108AC0000E94F837FE01319621E830E0F999FECF97
:108AD00032BD21BDF89A80B581932F5F3F4F253875
:108AE0003105A1F760911F1970912019809121190A
:108AF000909122192FE632E143E85AE30F94620D78
:108B00009B01AC0169817A818B819C810F94EC0976
:108B100069837A838B839C83FE01319681E890E0A0
:108B2000AE014B5F5F4F0EC02081F999FECF3196A9
:108B30001FBA92BD81BD20BD0FB6F894FA9AF99A7A
:108B40000FBE0196E417F50779F780E090E0A0E00A
:108B5000B0E080931F1990932019A0932119B0932E
:108B600022190F94860360931B1970931C1980932C
:108B70001D1990931E1920E030E040E028363105A1
:108B800039F0F999FECF32BD21BDF89A80B5480F72
:108B90002F5F3F4F88E02030380781F7F999FECFEB
:108BA00088E690E092BD81BDF89A80B5481769F0DB
:108BB000F999FECF1FBA88E690E092BD81BD40BD15
:108BC0000FB6F894FA9AF99A0FBE0E94081B0F90FC
:108BD0000F900F900F90CF91DF911F910F91FF9009
:108BE000EF900895BF92CF92DF92EF92FF920F9392
:108BF0001F93DF93CF9300D00F92CDB7DEB7F999D3
:108C0000FECF89E690E092BD81BDF89AB0B48BE4C6
:108C100090E00E942A386093D8027093D902809322
:108C2000DA029093DB028FE490E00E942A3860938E
:108C3000260570932705809328059093290583E5E1
:108C400090E00E942A386093D4027093D5028093FA
:108C5000D6029093D702FE01319623E030E0F999D5
:108C6000FECF32BD21BDF89A80B581932F5F3F4F73
:108C700027303105A1F789819A81AB81BC8180932E
:108C8000E2029093E302A093E402B093E502FE01B6
:108C9000319627E030E0F999FECF32BD21BDF89A38
:108CA00080B581932F5F3F4F2B303105A1F789812C
:108CB0009A81AB81BC818093E6029093E702A093F6
:108CC000E802B093E902FE0131962BE030E0F99919
:108CD000FECF32BD21BDF89A80B581932F5F3F4F03
:108CE0002F303105A1F789819A81AB81BC818093B6
:108CF000EA029093EB02A093EC02B093ED02FE0126
:108D000031962FE030E0F999FECF32BD21BDF89ABF
:108D100080B581932F5F3F4F23313105A1F78981C2
:108D20009A81AB81BC818093F2029093F302A0936D
:108D3000F402B093F502FE01319623E130E0F99997
:108D4000FECF32BD21BDF89A80B581932F5F3F4F92
:108D500027313105A1F789819A81AB81BC8180934C
:108D6000F6029093F702A093F802B093F902FE0185
:108D7000319627E130E0F999FECF32BD21BDF89A56
:108D800080B581932F5F3F4F2B313105A1F789814A
:108D90009A81AB81BC818093FA029093FB02A093ED
:108DA000FC02B093FD02FE0131962BE130E0F9990F
:108DB000FECF32BD21BDF89A80B581932F5F3F4F22
:108DC0002F313105A1F789819A81AB81BC818093D4
:108DD000020390930303A0930403B0930503FE01E1
:108DE00031962FE130E0F999FECF32BD21BDF89ADE
:108DF00080B581932F5F3F4F23323105A1F78981E1
:108E00009A81AB81BC818093060390930703A09362
:108E10000803B0930903FE01319623E230E0F9998B
:108E2000FECF32BD21BDF89A80B581932F5F3F4FB1
:108E300027323105A1F789819A81AB81BC8180936A
:108E40000A0390930B03A0930C03B0930D03FE0150
:108E5000319627E230E0F999FECF32BD21BDF89A74
:108E600080B581932F5F3F4F2B323105A1F7898168
:108E70009A81AB81BC8180930D1990930E19A093B8
:108E80000F19B0931019FE01319623E330E0F999E0
:108E9000FECF32BD21BDF89A80B581932F5F3F4F41
:108EA00027333105A1F789819A81AB81BC818093F9
:108EB0000E0390930F03A0931003B0931103FE01D0
:108EC000319627E330E0F999FECF32BD21BDF89A03
:108ED00080B581932F5F3F4F2B333105A1F78981F7
:108EE0009A81AB81BC818093120390931303A0936A
:108EF0001403B0931503FE0131962BE330E0F9998A
:108F0000FECF32BD21BDF89A80B581932F5F3F4FD0
:108F10002F333105A1F789819A81AB81BC81809380
:108F2000160390931703A0931803B0931903FE013F
:108F300031962FE330E0F999FECF32BD21BDF89A8A
:108F400080B581932F5F3F4F23343105A1F789818D
:108F50009A81AB81BC8180931E0390931F03A093E1
:108F60002003B0932103FE01319623E430E0F99908
:108F7000FECF32BD21BDF89A80B581932F5F3F4F60
:108F800027343105A1F789819A81AB81BC81809317
:108F9000220390932303A0932403B0932503FE019F
:108FA000319627E430E0F999FECF32BD21BDF89A21
:108FB00080B581932F5F3F4F2B343105A1F7898115
:108FC0009A81AB81BC818093260390932703A09361
:108FD0002803B0932903F999FECF8AE690E092BD69
:108FE00081BDF89A80B58093A102F999FECF8BE6F6
:108FF00090E092BD81BDF89A80B58093A602F99960
:10900000FECF8CE790E092BD81BDF89A80B5809349
:10901000A702FE0131962CE630E0F999FECF32BD71
:1090200021BDF89A80B581932F5F3F4F20373105DE
:10903000A1F789819A81AB81BC818093A80290932A
:10904000A902A093AA02B093AB02FE01319620E7D9
:1090500030E0F999FECF32BD21BDF89A80B58193F9
:109060002F5F3F4F24373105A1F789819A81AB816A
:10907000BC818093AC029093AD02A093AE02B093FA
:10908000AF02FE01319624E730E0F999FECF32BD00
:1090900021BDF89A80B581932F5F3F4F2837310566
:1090A000A1F789819A81AB81BC818093B0029093B2
:1090B000B102A093B202B093B302F999FECF88E750
:1090C00090E092BD81BDF89A80B58093B402FE0114
:1090D000319625E830E0F999FECF32BD21BDF89AEE
:1090E00080B581932F5F3F4F29383105A1F78981E2
:1090F0009A81AB81BC818093F1189093F218A09370
:10910000F318B093F418FE01319629E830E0F9998C
:10911000FECF32BD21BDF89A80B581932F5F3F4FBE
:109120002D383105A1F789819A81AB81BC8180936B
:10913000F9189093FA18A093FB18B093FC18FE014D
:1091400031962DE830E0F999FECF32BD21BDF89A75
:1091500080B581932F5F3F4F21393105A1F7898178
:109160009A81AB81BC818093011990930219A093DD
:109170000319B0930419FE01319621E930E0F99901
:10918000FECF32BD21BDF89A80B581932F5F3F4F4E
:1091900025393105A1F789819A81AB81BC81809302
:1091A000ED189093EE18A093EF18B093F018FE010D
:1091B000319625E930E0F999FECF32BD21BDF89A0C
:1091C00080B581932F5F3F4F29393105A1F7898100
:1091D0009A81AB81BC818093F5189093F618A09387
:1091E000F718B093F818FE01319629E930E0F999A3
:1091F000FECF32BD21BDF89A80B581932F5F3F4FDE
:109200002D393105A1F789819A81AB81BC81809389
:10921000FD189093FE18A093FF18B093001982E0F8
:109220008B1508F082C00BE218E1B80140E050E075
:109230006E010894C11CD11CA5E0EA2EF12CEC0EA5
:10924000FD1E9A01220F331F220F331F245B3C4F58
:10925000F60109C0F999FECF32BD21BDF89A80B55B
:1092600081932F5F3F4FEE15FF05A1F789819A810A
:10927000AB81BC81FB0181939193A193B193BF0119
:109280004F5F5F4F49305105E1F620912B18309127
:109290002C1840912D1850912E18CA01B9010F9425
:1092A0001C0E882361F14CE453E07E010894E11C1C
:1092B000F11CBE016B5F7F4F9A01220F331F220FFB
:1092C000331FF70109C0F999FECF32BD21BDF89ACD
:1092D00080B581932F5F3F4FE617F707A1F789818C
:1092E0009A81AB81BC81F80181939193A193B19351
:1092F0008F014F5F5F4FF3E045355F07E9F6F9995E
:10930000FECF80E793E092BD81BDF89A80B590E0F2
:10931000811191E0892F0E949D9C8FE293E06BE286
:1093200078E149E026E00E94A637A895FE01319633
:1093300028EC30E0F999FECF32BD21BDF89A80B516
:1093400081932F5F3F4F2C3C3105A1F789819A8192
:10935000AB81BC818093210290932202A0932302CF
:10936000B0932402FE0131962CEC30E0F999FECF47
:1093700032BD21BDF89A80B581932F5F3F4F203DCC
:109380003105A1F789819A81AB81BC818093270245
:1093900090932802A0932902B0932A02FE013196ED
:1093A00020ED30E0F999FECF32BD21BDF89A80B5AD
:1093B00081932F5F3F4F243D3105A1F789819A8129
:1093C000AB81BC8180932F0290933002A093310235
:1093D000B0933202FE01319624ED30E0F999FECFD0
:1093E00032BD21BDF89A80B581932F5F3F4F283D54
:1093F0003105A1F789819A81AB81BC8180932B02D1
:1094000090932C02A0932D02B0932E02F999FECFD7
:1094100088ED90E092BD81BDF89A80B580935A02A4
:10942000F999FECF89ED90E092BD81BDF89A80B5A3
:1094300080935F02F999FECF85EF90E092BD81BDE8
:10944000F89A80B580936002FE0131962AED30E0F3
:10945000F999FECF32BD21BDF89A80B581932F5F77
:109460003F4F2E3D3105A1F789819A81AB81BC81A7
:109470008093610290936202A0936302B0936402AE
:10948000FE0131962EED30E0F999FECF32BD21BDBF
:10949000F89A80B581932F5F3F4F223E3105A1F7A7
:1094A00089819A81AB81BC81809365029093660229
:1094B000A0936702B0936802FE01319622EE30E07D
:1094C000F999FECF32BD21BDF89A80B581932F5F07
:1094D0003F4F263E3105A1F789819A81AB81BC813E
:1094E0008093690290936A02A0936B02B0936C021E
:1094F000F999FECF86EE90E092BD81BDF89A80B5D5
:1095000080936D0287EE90E00E942A3860931902E2
:1095100070931A0280931B0290931C028BEE90E0D2
:109520000E942A3860931D0270931E0280931F02CE
:1095300090932002F999FECF8FEE90E092BD81BD0D
:10954000F89A20B5F999FECF80EF90E092BD81BDE9
:10955000F89A80B52093370280933802F999FECFAC
:109560008AEF90E092BD81BDF89A20B5F999FECFBF
:109570008BEF90E092BD81BDF89A80B520933902BF
:1095800080933A02F999FECF8CEF90E092BD81BDB5
:10959000F89A20B5F999FECF8DEF90E092BD81BD8C
:1095A000F89A80B520933B0280933C02FE013196ED
:1095B00021EF30E0F999FECF32BD21BDF89A80B598
:1095C00081932F5F3F4F253F3105A1F789819A8114
:1095D000AB81BC8180933D0290933E02A0933F02F9
:1095E000B0934002FE01319626EF30E0F999FECFAC
:1095F00032BD21BDF89A80B581932F5F3F4F2A3F3E
:109600003105A1F789819A81AB81BC8180934102A8
:1096100090934202A0934302B093440281E08B15E1
:1096200070F4F999FECF8EEF90E092BD81BDF89A6B
:1096300080B580938C02E7E0BE1609F445C381E251
:109640009BE00E94CA36F2E0FB1508F46CC180E092
:1096500090E0A0E0B0E089839A83AB83BC83FE01F5
:10966000319688E293E0AE014B5F5F4F0EC02081E0
:10967000F999FECF31961FBA92BD81BD20BD0FB6BC
:10968000F894FA9AF99A0FBE0196E417F50779F75C
:1096900080E090E0A0EAB0E489839A83AB83BC8346
:1096A000FE0131968CE293E0AE014B5F5F4F0EC03E
:1096B0002081F999FECF31961FBA92BD81BD20BDA0
:1096C0000FB6F894FA9AF99A0FBE0196E417F507C7
:1096D00079F780E090E0A0E2B2E489839A83AB83DB
:1096E000BC83FE01319688E493E0AE014B5F5F4F8F
:1096F0000EC02081F999FECF31961FBA92BD81BD6F
:1097000020BD0FB6F894FA9AF99A0FBE0196E417A5
:10971000F50779F780E090E0A0E0B0E089839A83D4
:10972000AB83BC83FE01319680E293E0AE014B5FD8
:109730005F4F0EC02081F999FECF31961FBA92BDBE
:1097400081BD20BD0FB6F894FA9AF99A0FBE019622
:10975000E417F50779F780E090E0A0E0B0E08983B6
:109760009A83AB83BC83FE01319684E293E0AE0121
:109770004B5F5F4F0EC02081F999FECF31961FBA23
:1097800092BD81BD20BD0FB6F894FA9AF99A0FBE2A
:109790000196E417F50779F780E090E0A0E5B2ECD8
:1097A00089839A83AB83BC83FE01319680E393E087
:1097B000AE014B5F5F4F0EC02081F999FECF31960D
:1097C0001FBA92BD81BD20BD0FB6F894FA9AF99ADE
:1097D0000FBE0196E417F50779F780E090E0A0EF5F
:1097E000B1EC89839A83AB83BC83FE01319684E319
:1097F00093E0AE014B5F5F4F0EC02081F999FECF21
:1098000031961FBA92BD81BD20BD0FB6F894FA9A69
:10981000F99A0FBE0196E417F50779F780E090E01A
:10982000A0E5B2E489839A83AB83BC83FE013196C1
:1098300088E393E0AE014B5F5F4F0EC02081F99942
:10984000FECF31961FBA92BD81BD20BD0FB6F894F0
:10985000FA9AF99A0FBE0196E417F50779F780E0B6
:1098600090E0A0EFB1EC89839A83AB83BC83FE01C7
:1098700031968CE393E0AE014B5F5F4F0EC02081C9
:10988000F999FECF31961FBA92BD81BD20BD0FB6AA
:10989000F894FA9AF99A0FBE0196E417F50779F74A
:1098A00080E090E0A0E0B0E089839A83AB83BC8342
:1098B000FE01319680E493E0AE014B5F5F4F0EC036
:1098C0002081F999FECF31961FBA92BD81BD20BD8E
:1098D0000FB6F894FA9AF99A0FBE0196E417F507B5
:1098E00079F780E090E0A0E7B2E489839A83AB83C4
:1098F000BC83FE01319684E493E0AE014B5F5F4F81
:109900000EC02081F999FECF31961FBA92BD81BD5C
:1099100020BD0FB6F894FA9AF99A0FBE0196E41793
:10992000F50779F704C083E0B81609F060C080E05D
:1099300090E0A9E5B3E489839A83AB83BC83FE01FD
:10994000319681E793E0AE014B5F5F4F0EC02081FF
:10995000F999FECF31961FBA92BD81BD20BD0FB6D9
:10996000F894FA9AF99A0FBE0196E417F50779F779
:1099700080E090E0A8ECB2E489839A83AB83BC8357
:10998000FE01319685E793E0AE014B5F5F4F0EC05D
:109990002081F999FECF31961FBA92BD81BD20BDBD
:1099A0000FB6F894FA9AF99A0FBE0196E417F507E4
:1099B00079F789E793E064EB70E00E94E0378BE78A
:1099C00093E066E470E00E94E0378DE793E064E6A0
:1099D00070E00E94E0378FE793E064E670E00E9459
:1099E000E03781E893E064E670E00E94E037E4E06D
:1099F000EB1508F464C080E090E0A2E5B3E489834D
:109A00009A83AB83BC83FE01319685E893E0AE0177
:109A10004B5F5F4F0EC02081F999FECF31961FBA80
:109A200092BD81BD20BD0FB6F894FA9AF99A0FBE87
:109A30000196E417F50779F780E090E0A5EAB3E432
:109A400089839A83AB83BC83FE01319689E893E0D6
:109A5000AE014B5F5F4F0EC02081F999FECF31966A
:109A60001FBA92BD81BD20BD0FB6F894FA9AF99A3B
:109A70000FBE0196E417F50779F780E090E0A4EBBC
:109A8000B2E489839A83AB83BC83FE0131968DE86F
:109A900093E0AE014B5F5F4F0EC02081F999FECF7E
:109AA00031961FBA92BD81BD20BD0FB6F894FA9AC7
:109AB000F99A0FBE0196E417F50779F704C0F5E0AF
:109AC000BF1609F064C080E090E0A0E0B0E08983B8
:109AD0009A83AB83BC83FE01319681E993E0AE01AA
:109AE0004B5F5F4F0EC02081F999FECF31961FBAB0
:109AF00092BD81BD20BD0FB6F894FA9AF99A0FBEB7
:109B00000196E417F50779F780E090E0A0E0B0E077
:109B100089839A83AB83BC83FE01319685E993E008
:109B2000AE014B5F5F4F0EC02081F999FECF319699
:109B30001FBA92BD81BD20BD0FB6F894FA9AF99A6A
:109B40000FBE0196E417F50779F780E090E0A0E0FA
:109B5000B0E089839A83AB83BC83FE01319689E9A7
:109B600093E0AE014B5F5F4F0EC02081F999FECFAD
:109B700031961FBA92BD81BD20BD0FB6F894FA9AF6
:109B8000F99A0FBE0196E417F50779F704C086E04D
:109B9000B81609F096C080E090E0A8ECB2E48983A2
:109BA0009A83AB83BC83FE0131968DE993E0AE01CD
:109BB0004B5F5F4F0EC02081F999FECF31961FBADF
:109BC00092BD81BD20BD0FB6F894FA9AF99A0FBEE6
:109BD0000196E417F50779F780E090E0A0E0B0E0A7
:109BE00089839A83AB83BC83FE01319685EA93E037
:109BF000AE014B5F5F4F0EC02081F999FECF3196C9
:109C00001FBA92BD81BD20BD0FB6F894FA9AF99A99
:109C10000FBE0196E417F50779F780E090E0A0E029
:109C2000B0E089839A83AB83BC83FE01319689EAD5
:109C300093E0AE014B5F5F4F0EC02081F999FECFDC
:109C400031961FBA92BD81BD20BD0FB6F894FA9A25
:109C5000F99A0FBE0196E417F50779F780E090E0D6
:109C6000A0E0B0E089839A83AB83BC83FE01319688
:109C70008DEA93E0AE014B5F5F4F0EC02081F999F2
:109C8000FECF31961FBA92BD81BD20BD0FB6F894AC
:109C9000FA9AF99A0FBE0196E417F50779F725C0ED
:109CA0002081F999FECF31961FBA92BD81BD20BDAA
:109CB0000FB6F894FA9AF99A0FBE0196E417F507D1
:109CC00079F780E00E94873B0E943AAE1DD30F9047
:109CD0000F900F900F90CF91DF911F910F91FF90F8
:109CE000EF90DF90CF90BF90089580E090E0A0EAE1
:109CF000B0E489839A83AB83BC83FE01319681EA09
:109D000093E0AE014B5F5F4FD9CF0F931F9320E0DD
:109D100030E010E02836310539F0F999FECF32BD38
:109D200021BDF89A80B5180F2F5F3F4F88E0203093
:109D3000380781F7F999FECF88E690E092BD81BDA2
:109D4000F89A00B5F999FECF12BC11BCF89A80B50B
:109D5000823029F4011719F40E94F24513C0F999D1
:109D6000FECF1FBA12BC11BC82E080BD0FB6F894C2
:109D7000FA9AF99A0FBE0E94493880E0011381E0F7
:109D80000E94873B1F910F910895DF93CF9300D0DE
:109D90000F92CDB7DEB7FC018081918191FF32C077
:109DA00093FF30C0268D2130D1F0213028F02230B1
:109DB000F9F0233039F52AC092FF24C023A134A141
:109DC00045A156A1878DF999FECF1FBA32BD21BD9D
:109DD00080BD0FB6F894FA9AF99A0FBE13C092FF9D
:109DE00011C0678D70A183A194A10E94E0370AC0C1
:109DF00092FF08C0478D50A161A172A183A194A1D7
:109E00000E94F83720E030E040E025C083FFFACF21
:109E100023A134A182859385A485B58589839A83FE
:109E2000AB83BC83FE013196AE014B5F5F4F0FC029
:109E30008081F999FECF31961FBA32BD21BD80BD18
:109E40000FB6F894FA9AF99A0FBE2F5F3F4FE417B6
:109E5000F50771F7D7CF2836310539F0F999FECFDC
:109E600032BD21BDF89A80B5480F2F5F3F4F88E083
:109E70002030380781F7F999FECF88E690E092BD4F
:109E800081BDF89A80B5481769F0F999FECF1FBADD
:109E900088E690E092BD81BD40BD0FB6F894FA9A75
:109EA000F99A0FBE0E94F245E0915603F0915703D4
:109EB00080810E941B590F900F900F900F90CF91AF
:109EC000DF910895EF92FF920F931F9380E990ED39
:109ED000A3E0B0E08093D8029093D902A093DA0275
:109EE000B093DB02109226051092270510922805E8
:109EF0001092290580E49EE7A5E0B0E08093D402AB
:109F00009093D502A093D602B093D70220E030E020
:109F100048EC52E42093E2023093E3024093E402DF
:109F20005093E5022093E6023093E7024093E80263
:109F30005093E9022093EA023093EB024093EC0243
:109F40005093ED0280E090E0A0E8BFE38093EE0242
:109F50009093EF02A093F002B093F1020F2EF0E085
:109F6000EF2EF0E0FF2EF8E40F2FF3E41F2FF02D7B
:109F7000E092F202F092F3020093F4021093F502E1
:109F8000E092F602F092F7020093F8021093F902C1
:109F9000E092FA02F092FB020093FC021093FD02A1
:109FA00080E090E0A0E2B2E4809302039093030388
:109FB000A0930403B09305038093060390930703D3
:109FC000A0930803B093090380930A0390930B03B3
:109FD000A0930C03B0930D0380E090E0A0EAB1E4FD
:109FE00080930D1990930E19A0930F19B093101927
:109FF00080E090E0AAE7B4E480930E0390930F030F
:10A00000A0931003B0931103809312039093130352
:10A01000A0931403B0931503809316039093170332
:10A02000A0931803B093190380E090E0AAEFB4E482
:10A0300080931E0390931F03A0932003B0932103EA
:10A040008093220390932303A0932403B0932503CA
:10A050008093260390932703A0932803B0932903AA
:10A0600071E07093A1026FEF6093A60280E5809388
:10A07000A70280E090E0A4E4B3E48093A802909368
:10A08000A902A093AA02B093AB028BE794E1A4E0EB
:10A09000B2E48093AC029093AD02A093AE02B09371
:10A0A000AF0280E090E0A1E9B3E48093B002909326
:10A0B000B102A093B202B093B3026093B4022093B2
:10A0C000ED183093EE184093EF185093F01820934A
:10A0D000F5183093F6184093F7185093F818E0925B
:10A0E000FD18F092FE180093FF181093001920E05D
:10A0F00030E040E050E02093F1183093F2184093A4
:10A10000F3185093F4182093F9183093FA184093E9
:10A11000FB185093FC1820930119309302194093B7
:10A12000031950930419E1E2F2E080E090E0A6E127
:10A13000B3E48093210290932202A0932302B09370
:10A14000240280E090E0A0EFB1E480932702909396
:10A150002802A0932902B0932A0280E090E0A0E2B6
:10A16000B1E480932F0290933002A0933102B09318
:10A17000320280E090E0AAE7B5E480932B0290934E
:10A180002C02A0932D02B0932E0270935A028CE8F9
:10A1900086AF8CE387AF80E090E0A0ECB1E48093E1
:10A1A000610290936202A0936302B09364028EEA0C
:10A1B00097E4A1E6BFE38093650290936602A093C3
:10A1C0006702B093680280E090E0A0EAB2E4809376
:10A1D000690290936A02A0936B02B0936C02609341
:10A1E0006D0210921D0210921E0210921F02109218
:10A1F00020021092190210921A0210921B02109261
:10A200001C0281E090E0909338028093370286E947
:10A2100090E090933A028093390210923C0210929F
:10A220003B0260938C0220933D0230933E024093A8
:10A230003F025093400220934102309342024093E8
:10A2400043025093440280E00E949D9C81E00E9462
:10A25000469C0E9449380E943AAEE0915603F09124
:10A2600057038081E8D750D080E09BE00E94D5362C
:10A270001F910F91FF90EF900895EF92FF920F932F
:10A280001F93CF93DF93EC018B898130B1F5EE8C76
:10A29000FF8C08A119A1C801B70120E030E040E01F
:10A2A00050E00F94B20A882341F1688D70E080E09D
:10A2B00090E00F94520B20E030E040E251E40F9424
:10A2C000620DA80197010F94B90A6FA378A789A717
:10A2D0009AA7698D70E080E090E00F94520B20E027
:10A2E00030E040E251E40F94620DA80197010F9411
:10A2F000B90A6BA77CA78DA79EA7DF91CF911F916D
:10A300000F91FF90EF9008958EE892E0B6CFE09124
:10A31000D102F091D2022781308541855285B90161
:10A32000CA0108952F923F924F925F926F927F924F
:10A330008F929F92AF92BF92CF92DF92EF92FF9255
:10A340000F931F93CF93DF931C01DC0111964C9167
:10A35000453338F44233F8F4842F81508C3058F56B
:10A360000AC0443628F4413630F44C3321F513C08A
:10A37000443609F510C0D1011296EC911297F0E025
:10A38000EE0FFF1FEE5AFC4F208131818CEF9FE0D2
:10A39000821B930B0BC0D1011296EC911297F0E047
:10A3A000EE0FFF1FEE5AFC4F8081918114969C9313
:10A3B0008E93139705C08FEF9FE0F1019483838301
:10A3C000D1011396ED90FC901497453348F4423335
:10A3D00008F053C0842F81508C3008F000C107C0B2
:10A3E0004C3309F4C9C0443609F0F9C0DEC090E02E
:10A3F000FC01EC50FE4E4491440FFC01EE0FFF1F98
:10A40000E050FE4E25913491F90145905490F901A8
:10A410003296659074900CEF1FE00E191F0982E0D0
:10A4200029C0E82FF0E0EE0FFF1FE20FF31F859029
:10A4300094908F5FE82FF0E08150EE0FFF1FE20F46
:10A44000F31FC591D491081519058CF4B301882721
:10A4500077FD8095982F0F94540B5B016C01B80128
:10A4600064197509882777FD8095982F44C08E5F01
:10A470003E0124018417A8F273C04E52842F90E04D
:10A48000FC01EC50FE4E4491440FFC01EE0FFF1F07
:10A49000E050FE4E25913491F90145905490F90118
:10A4A00032966590749082E058C0E82FF0E0EE0F8D
:10A4B000FF1FE20FF31F859094908F5FE82FF0E06D
:10A4C0008150EE0FFF1FE20FF31FC591D491E814E6
:10A4D000F9040CF03FC0B301882777FD8095982FD1
:10A4E0000F94540B5B016C01E418F508B701882741
:10A4F00077FD8095982F0F94540B7B018C01C61922
:10A50000D709BE01882777FD8095982F0F94540BAB
:10A510009B01AC01C801B7010F94620D7B018C0156
:10A5200084189508B401882777FD8095982F0F949B
:10A53000540B9B01AC01C801B7010F94B90A9B01F0
:10A54000AC01C601B5010F94EC0920E030E040E019
:10A550005EE323C08E5F3E012401841708F4A5CF7B
:10A56000BE01882777FD8095982F0F94540B20E02B
:10A5700030E040E05EE32AC0B701882777FD809590
:10A58000982F0F94540B20E030E04AE754E40F94E6
:10A59000620D20E030E040E859E30F94620DF101D4
:10A5A00067837087818792871AC0B701882777FDF4
:10A5B0008095982F0F94540B20E030E04AEF53E43D
:10A5C0000F94620D20E030E040E859E30F94620DF3
:10A5D000D10117966D937D938D939C931A97DF917C
:10A5E000CF911F910F91FF90EF90DF90CF90BF9090
:10A5F000AF909F908F907F906F905F904F903F9023
:10A600002F900895CF92DF92EF92FF920F931F93B6
:10A61000CF93DF936C01FC0143875487658776876E
:10A62000CB01BA0120E030E040E051E40F94620D2C
:10A630000F94210BDB01F6018181853340F48233D5
:10A6400008F068C081508C3008F0DCC007C08C3343
:10A6500009F4B2C0843609F0D5C0BFC090E0FC0157
:10A66000EC50FE4E1491110FFC01EE0FFF1FE05055
:10A67000FE4E65917491FB0125913491FB01329658
:10A68000E590F49082E03BC0E82FF0E0EE0FFF1F72
:10A69000E60FF71F459154918F5FE82FF0E081504E
:10A6A000EE0FFF1FE60FF71FC591D491CA17DB0706
:10A6B0001CF50CEF1FE0021B130B241B350BB9011B
:10A6C000882777FD8095982F97012A1B3B0B4427FD
:10A6D00037FD4095542F0F94380EEC1AFD0A970160
:10A6E000442737FD4095542F0F94AD0E020F131FD2
:10A6F000F6011683058386C08E5F7E019A0181175D
:10A7000008F4C2CF8CEF9FE0841B950BF601968373
:10A71000858378C08E5290E0FC01EC50FE4E64912F
:10A72000660FFC01EE0FFF1FE050FE4E4591549165
:10A73000FA01E590F490FA0132960591149182E0C5
:10A7400037C0E82FF0E0EE0FFF1FE40FF51F259153
:10A7500034918F5FE82FF0E08150EE0FFF1FE40F80
:10A76000F51FC591D491AC17BD07FCF4B701621B6E
:10A77000730B882777FD8095982F98012A1B3B0B38
:10A78000442737FD4095542F0F94380E0C1B1D0B9A
:10A790009801442737FD4095542F0F94AD0EE20EDB
:10A7A000F31EF601F682E5822DC08E5F8E017901DF
:10A7B000861708F4C6CF23C0BD01882777FD809592
:10A7C000982F3CE0660F771F881F991F3A95D1F7A5
:10A7D00028EE33E040E050E010C0BD01882777FD4F
:10A7E0008095982F2CE0660F771F881F991F2A9558
:10A7F000D1F724EF31E040E050E00F94AD0EF601C8
:10A8000036832583DF91CF911F910F91FF90EF90B9
:10A81000DF90CF900895EF92FF920F931F93809156
:10A82000281882FD02C080E03FC0E091CF02F09185
:10A83000D002E780F0840185128585EA98E060E027
:10A8400070E00E949636C801B7010F94210B665F35
:10A850007F4F6753714018F484EC98E002C08FEA90
:10A8600098E00E94BC36E091D102F091D202E780DC
:10A87000F084018512858AE998E00E943236C80189
:10A88000B7010F94210B665F7F4F6753714018F03B
:10A890008FEA98E002C084EC98E00E94BC368EEC0F
:10A8A00098E00E94BF3681E01F910F91FF90EF90DA
:10A8B0000895EF92FF920F931F930F948603AB01BD
:10A8C000BC0183E998E00E948736E0911502F0E030
:10A8D000EE0FFF1FE153FD4F008111813AEEE32E91
:10A8E00034E0F32EF8014781508561857285C701F8
:10A8F00022E00E949337F80143855485658576856B
:10A90000C70120E00E949337F8018081E2E3F5E07F
:10A91000E80FF11D6081C70170E00E9464361F914D
:10A920000F91FF90EF900895DF92EF92FF920F93B7
:10A930001F937B018C01D42E20E030E046EE52E4E0
:10A940000F94C00C18165CF40F2EF0E0EF2EF0E020
:10A95000FF2EF6EE0F2FF2E41F2FF02D14C0C801CA
:10A96000B70120E030E040E050E00F94B20A8823C5
:10A9700054F40F2EF0E0EF2EF0E0FF2EF0E00F2F5A
:10A98000F0E01F2FF02D6091990270919A02809152
:10A990009B0290919C02A80197010F94B20A882310
:10A9A00019F18EE892E0B801A7012CDEDD2079F0E4
:10A9B000C801B70120E030E040EF51E40F94C00C33
:10A9C00018162CF48091CE0281608093CE024091C3
:10A9D000990250919A0260919B0270919C028EE8BC
:10A9E00097E020E00E94CB371F910F91FF90EF90EE
:10A9F000DF9008952F923F924F925F926F927F92D5
:10AA00008F929F92AF92BF92CF92DF92EF92FF927E
:10AA10000F931F93DF93CF93CDB7DEB7E3970FB6B6
:10AA2000F894DEBF0FBECDBF9BAB8AAB48A359A342
:10AA30006AA37BA32CA30DA30F9486036D8B7E8B3F
:10AA40008F8B988FAAA9BBA996968C9190E095952B
:10AA500087951C01442437FC4094542C89E997E0E5
:10AA60000E94CA36E091CF02F091D0021682158280
:10AA700080E090E0A0E0B0E083879487A587B68768
:10AA8000E081F0E0EE5CFA4F1082E091D102F091AB
:10AA9000D2021682158283879487A587B687E081C4
:10AAA000F0E0EE5CFA4F1082BCA1B0931702AAA9A5
:10AAB000BBA9EC91F0E0EE5CFA4F96968C91808306
:10AAC000BCA1BB2321F480918C0280938D022D893F
:10AAD0003E894F89588D298B3A8B4B8B5C8B790142
:10AAE0008A0129863A864B865C861B8E1A8E31E057
:10AAF000398F80E090E0A0EAB1E489839A83AB8348
:10AB0000BC835C016D01A8958AA99BA90BDCAAA94D
:10AB1000BBA91796BC91BEA7EAA9FBA9F085FFA720
:10AB2000AAA9BBA91996BC91B8ABEAA9FBA9F28561
:10AB3000F9AB0F9486033B014C0169817A818B81CB
:10AB40009C812EA53FA548A959A90F94B20A882334
:10AB500044F48EA59FA5A8A9B9A989839A83AB833C
:10AB6000BC83C601B5012EA53FA548A959A90F94DC
:10AB7000B20A87FD06C08EA59FA5A8A9B9A95C0148
:10AB80006D01298D222309F441C06EA57FA588A9F6
:10AB900099A928A139A14AA15BA10F94C00C18164C
:10ABA0000CF08FC1A40193012E193F09400B510BEA
:10ABB0008CA1882329F484EC99E0A0E0B0E004C0E3
:10ABC0008CED95E0A0E0B0E082179307A407B507ED
:10ABD00008F077C1AAA9BBA9EC916E2F70E06E5C5A
:10ABE0007A4F822DB9858B1BFB0180832D873E8791
:10ABF0004F87588B698A7A8A8B8A9C8A28A139A1C7
:10AC00004AA15BA129833A834B835C836EA57FA510
:10AC100088A999A928A139A14AA15BA10F94B20AD8
:10AC200088230CF04DC1A401930189899A89AB89CD
:10AC3000BC89281B390B4A0B5B0B9CA1992329F07B
:10AC400088EB9BE0A0E0B0E004C088E893E1A0E0DE
:10AC5000B0E082179307A407B50708F031C1AA8DA9
:10AC6000BB8DAB2B09F412C18D859E85AF85B8894C
:10AC7000820F931FA41FB51F8C8F9D8FAE8FBF8F28
:10AC80006D857E858F859889621B730B840B950B70
:10AC900029853A854B855C850F94380E2C8D3D8D2A
:10ACA0004E8D5F8D0F94AD0E220D331D441D551D2D
:10ACB000243131054105510534F464E1262E312C4F
:10ACC000412C512C14C0AAA9BBA996968C9190E056
:10ACD00044977C010027F7FC0095102F19012A01E9
:10ACE000E216F3060407150714F417012801EAA970
:10ACF000FBA926A1822F869590E0A0E0B0E0821506
:10AD00009305A405B5052CF029863A864B865C860A
:10AD100010C0822F90E001979C01442737FD409599
:10AD2000542F221933094409550929873A874B873B
:10AD30005C878CEA97E0B201A1010E94873684EB20
:10AD400097E049855A856B857C850E94873689EB1B
:10AD500097E0B601A50122E00E94933780EC97E0CE
:10AD600049815A816B817C8122E00E94CB374A8DD8
:10AD70005B8D433051050CF489C069857A858B85DC
:10AD80009C850F94540B20E030E040E850E40F9491
:10AD9000620D7B018C0169817A818B819C81A60186
:10ADA00095010F94EB0920ED3FE049E450E40F9446
:10ADB000620D9B01AC01C801B7010F94B90A7B0178
:10ADC0008C016C8D7D8D8E8D9F8D0F94540B20E0AA
:10ADD00030E04AE754E40F94B90A5B016C0187EC58
:10ADE00097E0B801A70122E00E9493378DEC97E02D
:10ADF000B601A50122E00E94CB37C801B7012AE9BC
:10AE000039E949E15FE30F94620D6D837E838F839F
:10AE100098879B01AC010F94EC09A60195010F9452
:10AE2000B90A7B018C016AA7FBA60CA71DA76D813F
:10AE30007E818F819885A60195010F94620D20E097
:10AE400030E040E05EE30F94620D5B016C016EA3A5
:10AE5000BFA2C8A6D9A683ED97E00E94BC3680EEBB
:10AE600097E04D815E816F81788522E00E94CB372B
:10AE700086EE97E0A701B80122E00E94CB378CEE66
:10AE800097E0A501B60122E00E94CB37AAA9BBA991
:10AE9000EC912E2F30E02E5C3A4F8985820DF9011E
:10AEA00080832A8D3B8D2F5F3F4F3B8F2A8F8401FC
:10AEB0007301A8A0B9A0CAA0DBA031E0398F01C0FE
:10AEC000198E68A179A18AA19BA120E030E040EA17
:10AED00051E40F94EC099B01AC016EA57FA588A9F4
:10AEE00099A90F94C00C18161CF482EF97E031C09A
:10AEF000D401C3012D893E894F89588D821B930B44
:10AF0000A40BB50B895E9340A040B04038F080E0C0
:10AF10000E940B1C6D8A7E8A8F8A988E660C771C25
:10AF2000881C991C6E187F08800A910A89899A8961
:10AF3000AB89BC89681A790A8A0A9B0A91E8691662
:10AF40009FE4790692E1890690E0990650F18BE141
:10AF500098E00E94BF36E091CF02F091D0021682B5
:10AF6000158280E090E0A0E0B0E083879487A58719
:10AF7000B687E081F0E0EE5CFA4F1082E091D102FA
:10AF8000F091D2021682158283879487A587B687AF
:10AF9000E081F0E0EE5CFA4F10828FEF80931702B1
:10AFA00062C0AA8DBB8D16970CF454C088E398E05C
:10AFB0000E94CA36E091CF02F091D002168215822B
:10AFC00080E090E0A0E0B0E083879487A587B68713
:10AFD000E081F0E0EE5CFA4F1082E091D102F09156
:10AFE000D2021682158283879487A587B687E0816F
:10AFF000F0E0EE5CFA4F10828FEF80931702BDA154
:10B00000BB2389F12D813E814F815885AAA9BBA917
:10B010005A962D933D934D935C935D972AA53BA53E
:10B020004CA55DA5C901DA01EAA9FBA9868F978F16
:10B03000A0A3B1A32EA13FA148A559A5C901DA013A
:10B0400082A393A3A4A3B5A381E0838B80E00E9495
:10B05000873B09C085E29CE10E945FD685E29CE1C6
:10B060000E94D9FF50CDE3960FB6F894DEBF0FBE15
:10B07000CDBFCF91DF911F910F91FF90EF90DF90A7
:10B08000CF90BF90AF909F908F907F906F905F9088
:10B090004F903F902F90089560E080912602882382
:10B0A00009F461E0809125020D94EA059F92AF9228
:10B0B000BF92CF92DF92EF92FF920F931F93CF93A5
:10B0C000DF937B018C01942EA22EE091CF02F091B0
:10B0D000D002638574858585968520E030E040E761
:10B0E00051E40F94C00C181614F4BB2402C0BB2406
:10B0F000B394C801B70120E030E042E853E40F9474
:10B10000C00C18165CF40F2EF0E0EF2EF0E0FF2ECE
:10B11000F2E80F2FF3E41F2FF02D14C0C801B70180
:10B1200020E030E040E050E00F94B20A882354F46D
:10B130000F2EF0E0EF2EF0E0FF2EF0E00F2FF0E00A
:10B140001F2FF02DC92CDD24F601EE0FFF1FE15358
:10B15000FD4FC081D181CE01B801A70153DAAA20E9
:10B1600081F0C801B70120E030E040EF51E40F94D6
:10B17000C00C181634F4FE01E05CFF4F8081816042
:10B180008083C801B70120E030E048E452E40F9426
:10B19000C00C88237CF086E790E0C89EF001C99E31
:10B1A000F00DD89EF00D1124E85EFD4FEC58FF4FD6
:10B1B00081918083692D70E080E090E00F94520BC4
:10B1C000AB01BC0183E897E020E00E94933786E75B
:10B1D00094E0B801A70120E00E94CB37E091CF02B4
:10B1E000F091D002638574858585968520E030E0F6
:10B1F00040E751E40F94C00C18162CF0BB2079F4F2
:10B200000E9423450CC0BB2051F00F94860360932D
:10B210001B1970931C1980931D1990931E19DF91AF
:10B22000CF911F910F91FF90EF90DF90CF90BF9043
:10B23000AF909F9008952F923F924F925F926F929E
:10B240007F928F929F92AF92BF92CF92DF92EF92B6
:10B25000FF920F931F93DF93CF9300D00F92CDB740
:10B26000DEB72091F0173091F1174091F21750910D
:10B27000F317E0915603F0915703238F348F458FD6
:10B28000568F88E192E09093570380935603209362
:10B2900018183093191840931A1850931B18E090FF
:10B2A0002102F09022020091230210912402E092E8
:10B2B000EE02F092EF020093F0021093F10260E0D0
:10B2C00070E080E89FE3A80197010F94B90A6093AA
:10B2D000AC177093AD178093AE179093AF17A090F3
:10B2E0002702B0902802C0902902D0902A02A09292
:10B2F000FE02B092FF02C0920003D092010360915F
:10B300002B0270912C0280912D0290912E0260935D
:10B310002A0370932B0380932C0390932D03609347
:10B320001A0370931B0380931C0390931D03A801C1
:10B3300097010F94620D0F94260B6093BC177093C6
:10B34000BD178093BE179093BF176093CC1770936F
:10B35000CD178093CE179093CF17C801B7012091D6
:10B360002F023091300240913102509132020F94FD
:10B37000620D9B01AC0160E074E284E798E40F94F5
:10B38000B90A0F948F0B0F94260B962E60939B1780
:10B39000C601B501A80197010F94620D9B01AC0194
:10B3A00060E074E284E798E40F94B90A0F948F0B7D
:10B3B0000F94260B60939C17603118F08FE08093F8
:10B3C0009C1780919C17891510F090929C176091A2
:10B3D0009C1770E080E090E00F94520BA801970159
:10B3E0000F94620D9B01AC0160E074E284E798E485
:10B3F0000F94B90A7B018C01A60195010F94B20A42
:10B40000882344F4E092FE02F092FF0200930003CE
:10B410001093010387E492E00E943D51A090F4173D
:10B42000B090F517C090F617D090F7176090F81706
:10B430007090F9178090FA179090FB172090FC17E6
:10B440003090FD174090FE175090FF17809105191E
:10B4500090910619A0910719B091081989839A83D0
:10B46000AB83BC830091560310915703D80111960A
:10B470006D917D918D919C9114979095809570958B
:10B4800061957F4F8F4F9F4F0F94540B2091A017C2
:10B490003091A1174091A2175091A3170F94620DFC
:10B4A00060931119709312198093131990931419C2
:10B4B000F80165817681878190859095809570955A
:10B4C00061957F4F8F4F9F4F0F94540B2091A4177E
:10B4D0003091A5174091A6175091A7170F94620DB0
:10B4E0006093151970931619809317199093181972
:10B4F0008091291880FF26C000D00F92809102030E
:10B5000090910303A0910403B0910503EDB7FEB73A
:10B5100081839283A383B483C601B501A4019301FF
:10B52000820171010F2EF0E8AF2EFFE4BF2EF3EC85
:10B53000CF2EF7E4DF2EF02D0E94F8A90F900F9088
:10B540000F900F9089819A81AB81BC8180930519FE
:10B5500090930619A0930719B093081980E00E94F0
:10B5600093970F900F900F900F90CF91DF911F91B5
:10B570000F91FF90EF90DF90CF90BF90AF909F9092
:10B580008F907F906F905F904F903F902F90089595
:10B5900088E192E090935703809356030E9A0C9A99
:10B5A0008091250261E00F9437058091260288235F
:10B5B00029F48091250261E00F94EA050F94860337
:10B5C00060935602709357028093580290935902E9
:10B5D00080910101806280930101809102018F7D41
:10B5E000809302010E9484510C940E672F923F9227
:10B5F0004F925F926F927F928F929F92AF92BF9283
:10B60000CF92DF92EF92FF920F931F93DF93CF932E
:10B61000CDB7DEB72B970FB6F894DEBF0FBECDBF08
:10B62000A8950FEC12E01C830B838CE892E09A83C0
:10B6300089831F821E8292E39D8380911702AE81CF
:10B64000A81709F441C2EB81FC8180809180C4017C
:10B650000E949251FE81FF2329F5D40117966D9126
:10B660007D918D919C911A9720E030E048E452E45E
:10B670000F94B20A882394F4F40163857485858558
:10B68000968520E030E048E452E40F94B20A882323
:10B690002CF4A981BA8111961C9204C0E981FA8127
:10B6A00080818183D0902818D2FC2CC0D4011796B9
:10B6B000ED90FD900D911C911A97C801B70120E003
:10B6C00030E040E251EC0F94B20A87FD0AC0C80195
:10B6D000B70120E030E046E953E40F94C00C18169F
:10B6E0008CF4809158038F5F809358038B3018F44B
:10B6F000B1E0BF8307C0E4E0DE2AD09228188BD8DF
:10B70000F1E0FF838091281882FDDEC12224D4015C
:10B7100013962D913C91149715968D919C911697A7
:10B72000281739071CF4222423940FC08401005CDD
:10B730001F4FF801808180FF08C08D8163E00E9467
:10B7400091F5D8018C918E7F8C93F40187A5E82F19
:10B75000F0E03C96EE0FFF1FEE0FFF1FE80DF91D06
:10B76000D4011796AD90BD90CD90DC901A97A08231
:10B77000B182C282D382382E3394B3E03B22F401EB
:10B7800037A68389813009F0CAC0E384F484058533
:10B790001685C801B70120E030E040EA51E40F947B
:10B7A000B20A87FDB4C0C801B701A60195010F9484
:10B7B000EB092B013C0120E030E040EA51E40F941A
:10B7C000C00C181624F4D40196966C91A1C0C30144
:10B7D000B20120E030E040EA51EC0F94B20A87FD5C
:10B7E00096C0D4015A96ED90FD900D911C915D97F5
:10B7F000E886F9860A871B87C301B20154962D910A
:10B800003D914D915C9157970F94EC097B018C0110
:10B81000F401A3A4B4A4C5A4D6A4A60195010F94D1
:10B82000B20A87FD11C0D4019796AD90BD90CD901E
:10B83000DC909A97C801B701A60195010F94C00C3E
:10B84000181614F057016801F401A48AB58AC68A53
:10B85000D78A688579858A859B85A30192010F9493
:10B86000620D7B018C01C601B501D4015E962D915C
:10B870003D914D915C9191970F94620D2DEC3CECB4
:10B880004CEC5DE30F94620D9B01AC01C801B70164
:10B890000F94EC097B018C01D4019F96EC919F974A
:10B8A000F0E03C96EE0FFF1FEE0FFF1FE80DF91DB5
:10B8B000608171818281938117962D913D914D9187
:10B8C0005C911A970F94EB09F40122A133A144A1D2
:10B8D00055A10F94620D2FED3FE445E550E40F9420
:10B8E000620D9B01AC01C801B7010F94EC090F94E4
:10B8F000210B9B01AC0177FD0AC0D40196968C9177
:10B9000090E0B901821793071CF4BC0101C060E00C
:10B91000D401EC91F0E0EE5CFA4F6083B5C0833067
:10B9200009F07DC0F4014384548465847684C301A6
:10B93000B20120E030E040EA51E40F94B20A87FD02
:10B940006AC0C301B201A60195010F94EB097B0106
:10B950008C0120E030E040EA51E40F94C00C18164E
:10B9600024F4D40196968C9157C0C801B70120E009
:10B9700030E040EA51EC0F94B20A87FD4CC0F4016C
:10B98000648975898689978920E030E040E450E435
:10B990000F94620D7B018C01E32DF0E03C96EE0FDD
:10B9A000FF1FEE0FFF1FE80DF91DC601B501208135
:10B9B0003181428153810F94EB092FED3FE445E53E
:10B9C00050E40F94620D9B01AC01C801B7010F94C4
:10B9D000EC0920E030E040E85EE30F94620DD40112
:10B9E00054966D937D938D939C9357975A962D9172
:10B9F0003D914D915C915D970F94620DA60195016B
:10BA00000F94EC09A30192010F94C00C18161CF0BE
:10BA1000F401808D01C080E0D401EC9131C082300E
:10BA200041F50F9486039B01AC01F4018785908951
:10BA3000A189B28979018A01E81AF90A0A0B1B0B5C
:10BA4000D801C70189589341A040B040E8F0E08197
:10BA5000222011F480E001C08FEFF0E0EE5CFA4F9D
:10BA60008083D4011F962D933D934D935C93529701
:10BA70000BC0D401EC91222011F480E001C08FEFC3
:10BA8000F0E0EE5CFA4F8083F40167817085818578
:10BA9000928520E030E042E853E40F94C00C181681
:10BAA00034F4D401EC91F0E0EE5CFA4F1082809116
:10BAB0005603909157038F968816990629F42220F1
:10BAC00011F02F9A01C02F98BE81BF5FBE83ED8118
:10BAD000EE5CED830B811C810E5F1F4F1C830B837B
:10BAE00089819A818A589F4F9A838983B23009F05D
:10BAF000A4CD9F81992339F480915803882319F0AC
:10BB00008150809358038091281882FF17C0E091DC
:10BB1000CF02F091D002E081F0E0EE5CFA4F1082AB
:10BB2000E091D102F091D202E081F0E0EE5CFA4FB8
:10BB3000108280912E03886080932E032B960FB67F
:10BB4000F894DEBF0FBECDBFCF91DF911F910F9153
:10BB5000FF90EF90DF90CF90BF90AF909F908F902D
:10BB60007F906F905F904F903F902F900895FC01D1
:10BB70008081918180FD02C024E001C026E083FD28
:10BB80002C5F84FD2C5F85FD2C5F86FD2C5F90FD76
:10BB90002C5F91FD2F5F92FD2C5F93FD2C5FAC011C
:10BBA0004270507094FF19C02E5F3281452B09F00E
:10BBB0002E5F82FD2E5F30FD2C5F31FD2C5F32FD4C
:10BBC0002C5F97FF11C0848190E00196813591052B
:10BBD00014F080E590E0280F07C0452B09F02F5F97
:10BBE00082FD2F5F97FD205F822F08958091C4030F
:10BBF00090E00196817090708093C403809133042B
:10BC00008F5F80933304089580913304882319F45F
:10BC100020E030E008C09091C30385E3989F900135
:10BC20001124275A3C4FC9010895CF93DF93EC01AB
:10BC3000888181FF12C084E095E06DE40E94DC6899
:10BC40006E817F81882777FD8095982F0E94153619
:10BC500084E095E060E20E94DC68888182FF12C087
:10BC600084E095E067E40E94DC6868857985882730
:10BC700077FD8095982F0E94153684E095E060E26C
:10BC80000E94DC688881998191FF12C084E095E070
:10BC900064E50E94DC686E8D70E0882777FD8095F2
:10BCA000982F0E94153684E095E060E20E94DC68DF
:10BCB000888183FF09C04A855B856C857D8580E925
:10BCC00093E022E00E949337888184FF09C04E856B
:10BCD0005F856889798983E993E022E00E94933740
:10BCE000888185FF09C04A895B896C897D8986E9DD
:10BCF00093E022E00E949337888186FF09C04E8935
:10BD00005F89688D798D89E993E024E00E949337FB
:10BD10008881998190FF09C04A8D5B8D6C8D7D8DE6
:10BD20008CE993E022E00E9493378881998192FF09
:10BD300008C04F8D58A169A17AA18FE993E00E94B4
:10BD400087368881998193FF08C04BA15CA16DA1C2
:10BD50007EA182EA93E00E9487368A8180FF09C033
:10BD60004FA158A569A57AA585EA93E022E00E9433
:10BD700093378A8181FF09C04BA55CA56DA57EA57F
:10BD800088EA93E022E00E9493378A8182FF09C00B
:10BD90004FA558A969A97AA98BEA93E022E00E94ED
:10BDA00093378881998197FF04C08BA99CA90E9431
:10BDB000B7350E94F91ADF91CF9108950F931F9321
:10BDC000CF93DF93EC018B01709129047250F8013D
:10BDD00040E050E020E030E01FC0672F763108F0EF
:10BDE00065E1DF01962F8D91480F511D4F3F5105A1
:10BDF00010F04F5F5040240F351F2F3F310510F0DA
:10BE00002F5F3040915079F76150862F90E06F5F3F
:10BE10000196E80FF91F761B7723F9F68181281B1D
:10BE200031098081481B5109242B352B232B51F0DC
:10BE300080912E0382FF04C080E593E00E94BF360C
:10BE400080E0CDC0F801219131913983288334FFFE
:10BE50000CC0D80112968D919C9113979B838A8375
:10BE6000329637FF04C0419103C01B821A8240E121
:10BE7000888180FF0EC0819191919D838C83A0E089
:10BE8000B0E080932F0490933004A0933104B093DA
:10BE90003204888199819C012270307094FF0EC019
:10BEA000232B21F0819191919F838E83888182FF42
:10BEB00010C081919191998788870BC0232B19F02D
:10BEC00081918E831F82888182FF03C08191888740
:10BED0001986888183FF08C081919191A191B191C8
:10BEE0008A879B87AC87BD87888184FF08C0819142
:10BEF0009191A191B1918E879F87A88BB98B8881F1
:10BF000085FF08C081919191A191B1918A8B9B8B02
:10BF1000AC8BBD8B888186FF08C081919191A191E6
:10BF2000B1918E8B9F8BA88FB98F8881998190FF5B
:10BF300008C081919191A191B1918A8F9B8FAC8F13
:10BF4000BD8F8881998191FF02C081918E8F8881F8
:10BF5000998192FF08C081919191A191B1918F8FA8
:10BF600098A3A9A3BAA38881998193FF08C081915E
:10BF70009191A191B1918BA39CA3ADA3BEA38A8102
:10BF800080FF08C081919191A191B1918FA398A751
:10BF9000A9A7BAA78A8181FF08C081919191A19137
:10BFA000B1918BA79CA7ADA7BEA78A8182FF08C0CD
:10BFB00081919191A191B1918FA798ABA9ABBAABA7
:10BFC0008881998197FF08C0FCABEBABE40FF11DB2
:10BFD000108281E080932A041092380481E0DF917E
:10BFE000CF911F910F910895EF92FF920F931F939E
:10BFF000DF93CF930F920F92CDB7DEB77C018B0109
:10C00000CB01BE016F5F7F4F0E945A16FC018981F0
:10C010009A810817190751F4D70112968D919C91B6
:10C020001397906813969C938E931297CF010F905D
:10C030000F90CF91DF911F910F91FF90EF90089596
:10C04000EF92FF920F931F93DF93CF930F920F9274
:10C05000CDB7DEB77C018B01CB01BE016F5F7F4F97
:10C060004AE050E00E94B7179C0189819A81081725
:10C07000190731F4F7018281938190689383828359
:10C08000C9010F900F90CF91DF911F910F91FF90F9
:10C09000EF900895EF92FF920F931F93CF93DF934A
:10C0A0008C017B01DC0111961C921E9213961C924E
:10C0B0001E921297CB016EE470E00E941219BC012F
:10C0C0000097A9F06F5F7F4FC801BADF60932F041C
:10C0D000709330048093310490933204F80180818E
:10C0E0009181816091838083CB0164839583C701B3
:10C0F0006DE470E00E941219BC010097C9F06F5FF7
:10C100007F4FC8019DDFD80117967C936E931697D9
:10C110008D919C9111979C01226011963C932E93D6
:10C120006F3F710529F020F0826090618D939C93A0
:10C13000F801808181FFB8C186819781873191059F
:10C1400099F08C31910581F08D31910569F08E3136
:10C15000910551F08032910539F08537910509F04C
:10C16000A3C102C0319601C0F70180818D34D1F79F
:10C1700001C0319680818032E1F701C03196808123
:10C180008032E1F3D801D396EC93D397D496FC9305
:10C190000DC0D80116968D919C9117978537910502
:10C1A00011F0203231F02A3221F031962081222301
:10C1B00081F7108281E080932A04F80180819181C7
:10C1C000906828C16F5F7F4FC8013ADFD801199688
:10C1D0007C936E9318978D919C9111979C0124608C
:10C1E00011963C932E936F3F710529F020F08460E7
:10C1F00090618D939C93C70168E570E00E941219CD
:10C20000BC01009771F06F5F7F4FC801EDDEF80150
:10C210006287738784879587808191818860918305
:10C220008083C70169E570E00E941219BC01009784
:10C2300089F06F5F7F4FC801D7DED8011E966D93DE
:10C240007D938D939C9351978D919C9111978061D3
:10C250008D939C93C7016AE570E00E941219BC019E
:10C26000009771F06F5F7F4FC801BEDEF801628BEF
:10C27000738B848B958B8081918180629183808385
:10C28000C70165E470E00E941219BC01009789F0B3
:10C290006F5F7F4FC801A8DED80156966D937D93DE
:10C2A0008D939C9359978D919C91119780648D9358
:10C2B0009C93C70166E470E00E941219BC010097CC
:10C2C00071F06F5F7F4FC8018FDEF801628F738F4F
:10C2D000848F958F80819181916091838083C70144
:10C2E00064E570E00E941219BC01009771F06F5F65
:10C2F0007F4FC801A5DED8015E966C935E978D9145
:10C300009C91119792608D939C93C70163E570E0B7
:10C310000E941219BC01009771F06F5F7F4FC80136
:10C320008FDEF801678F70A381A392A38081918132
:10C33000946091838083C70160E570E00E941219C8
:10C34000BC01009789F06F5F7F4FC80179DED8018B
:10C3500093966D937D938D939C9396978D919C91DD
:10C36000119798608D939C93C70169E470E00E94D7
:10C370001219BC01009799F06F5F7F4FC80134DE3E
:10C38000F80167A370A781A792A78281938181603A
:10C390009383828380819181906191838083C7019F
:10C3A0006AE470E00E941219BC010097D1F06F5F3F
:10C3B0007F4FC80119DED8019B966D937D938D93B5
:10C3C0009C939E9712968D919C91139782601396E1
:10C3D0009C938E9312978D919C91119790618D9360
:10C3E0009C93C70162E570E00E941219BC0100979E
:10C3F00099F06F5F7F4FC801F7DDF80167A770AB59
:10C4000081AB92AB828193818460938382838081AC
:10C410009181906191838083C7016AE270E00E94FC
:10C420001219EC010097D1F0BC016F5F7F4FC8017A
:10C4300007DE90E004C0D7018D917D019827EC16AE
:10C44000FD06C9F7961751F080912E0382FF04C0B4
:10C4500080E593E00E94BF3690E01EC0F801828123
:10C46000938197FD06C08081918186709270892B9F
:10C4700029F5809138048F5F8093380480912E03D2
:10C4800082FF04C080E793E00E94BF3690E0809175
:10C490003804833008F091E0892FDF91CF911F910C
:10C4A0000F91FF90EF900895C70167E470E00E943C
:10C4B0001219BC01009709F085CE9DCE1092380468
:10C4C000EACFAF92BF92CF92DF92FF920F931F936A
:10C4D000DF93CF93CDB7DEB7C558D0400FB6F894F1
:10C4E000DEBF0FBECDBF8C0186E3C82ED12CCC0E93
:10C4F000DD1E5E010894A11CB11C90E080E00F5F7E
:10C500001F4F01501040F801F4900F5F1F4FFF20A4
:10C5100091F0FAE0FF1679F02BE3F21611F491E0B6
:10C5200007C0992329F4F601E80FF11DF0828F5F0F
:10C530008F3428F302C08823A9F0F601E80FF11D1B
:10C540001082C501B60140E0A5DD882359F089813C
:10C550009A8186709270892B29F0C5010E94C91CAE
:10C560000E94DCADFF2049F6CB57DF4F0FB6F894A1
:10C57000DEBF0FBECDBFCF91DF911F910F91FF9016
:10C58000DF90CF90BF90AF900895CF93DF93EC01F1
:10C5900080912E0380FF06C086E493E00E9432362D
:10C5A000CE0143DBDF91CF9108959C01809133044C
:10C5B000882381F0C901E9DF8091C3038F5F8093F5
:10C5C000C303823011F41092C3038091330481506D
:10C5D00080933304089584E095E0E0D5109225041B
:10C5E00080912604882311F08EE101C08EE08093B3
:10C5F000D3020E94F91A40912B0450912C046091AF
:10C600002D0470912E044F5F5F4F6F4F7F4F8EE36D
:10C6100093E00E9442368AE193E00C94BC36CF92BC
:10C62000DF92EF92FF920F931F93CF93DF93EC0172
:10C63000888181FF38C08E819F818E369105A9F453
:10C6400080912F0490913004A0913104B091320474
:10C6500080932B0490932C04A0932D04B0932E046C
:10C660008AE193E00E94BC3688C08037910511F4BE
:10C670000E94CF198E819F818A599240A1F48091A6
:10C680002B0490912C04A0912D04B0912E040196BE
:10C69000A11DB11D80932B0490932C04A0932D0415
:10C6A000B0932E046DC0888180FF56C000912B048A
:10C6B00010912C0420912D0430912E0468017901F1
:10C6C0000894C11CD11CE11CF11C40912F04509115
:10C6D00030046091310470913204D701C60184277F
:10C6E0009527A627B727892B79F1C801841B950BBD
:10C6F0008897F8F08091D30287FF18C080912E03AD
:10C7000082FF12C08CEB93E0B701A6010E9478363D
:10C7100040912F04509130046091310470913204A3
:10C7200081ED93E00E94423656DF2AC0815080930B
:10C73000D3021092250487ED93E00E9442368AE1ED
:10C7400093E00E94BC361CC040932B0450932C04F1
:10C7500060932D0470932E0449DA40912F04509178
:10C76000300460913104709132048CE493E00E94B3
:10C77000423680912604809327048FEF8093D30262
:10C78000DF91CF911F910F91FF90EF90DF90CF90AD
:10C790000895BF92CF92DF92EF92FF920F931F9373
:10C7A000CF93DF9380913304823008F021C28091CF
:10C7B0002A04882309F4F6C180913304882309F4FC
:10C7C000F1C116C28091D30287FF04C08091250475
:10C7D0008823A9F08091340490913504A091360407
:10C7E000B0913704A7019601281B390B4A0B5B0B4C
:10C7F000293C31054105510510F0EDDE1FC0809147
:10C800003304882309F0A6C0809134049091350444
:10C81000A0913604B0913704A7019601281B390B6B
:10C820004A0B5B0BDA01C901895E9340A040B0401E
:10C8300008F490C084ED99E00E94BC36C0923404A4
:10C84000D0923504E0923604F092370483C0909180
:10C85000D30297FD0FC080912704882359F080915F
:10C86000C503882321F491509093D3024BC0B0921A
:10C87000D30248C08091C503882309F443C08823AC
:10C88000880F880B802380932604809126048823B8
:10C89000F9F0113009F461C0812F8450823028F4FE
:10C8A00085EC93E064D980932904809129041817BA
:10C8B00009F04AC09091C40385E3989FE0011124D8
:10C8C000C75ADC4FCE0165EC73E041E077DA2AC04D
:10C8D000A12FB0E01197FD01EB53FC4FE081EE2357
:10C8E00051F0EA3041F0ED3031F080912804882396
:10C8F00001F5EA33F1F4AB53BC4F1C9210922804BB
:10C90000113019F41092250428C09091C40385E3D6
:10C91000989FE0011124C75ADC4FCE0165EC73E00B
:10C9200041E0B8DB882319F0CE0179DE02C153DE85
:10C9300000C1EB3311F4009328048091280488236C
:10C9400019F011501093250480912504803629F4A4
:10C9500042DE4EC101E09EE1B92E84E095E0D2D3E3
:10C96000181619060CF02CC110912504103608F089
:10C9700027C1C0923404D0923504E0923604F0927C
:10C98000370484E095E0EBD3E12FF0E0EB53FC4F6C
:10C9900080831F5F10932504113009F076CF57CFA5
:10C9A00080912504882309F4D3C022C10F94860303
:10C9B0006093340470933504809336049093370465
:10C9C0008DEC99E10E9416CBEC014FEF8F3F94075D
:10C9D00071F58EEA93E00E94BC3685E29CE162E24A
:10C9E00077E141E020E00E9460D54091EE1950913E
:10C9F000EF196091F0197091F1198DEC99E10E9495
:10CA0000AFC38DEC99E10E9416CBEC015FEF8F3F35
:10CA1000950729F488E097E10E94BF36B3C085E20C
:10CA20009CE169EF76E141E020E00E9460D5209131
:10CA3000EE193091EF194091F0195091F1192F5FD3
:10CA40003F4F4F4F5F4F2093EE193093EF194093B4
:10CA5000F0195093F11980912504E82FF0E0EB5381
:10CA6000FC4FC083182F1F5F10932504113041F431
:10CA7000109226048091C50387FF02C010932604FC
:10CA8000809126048823F1F0123008F461C0812FD0
:10CA90008450823028F485EC93E069D8809329048F
:10CAA00080912904181709F053C08091C40325E32D
:10CAB000829FC0011124875A9C4F65EC73E040E0CF
:10CAC0007DD934C0C12FD0E0BE0161507040FB0160
:10CAD000EB53FC4FE081EA3071F0ED3009F076C0A5
:10CAE0000AC080912804882311F4EA3321F01F350D
:10CAF00008F07AC021C06B537C4FFB01108203C049
:10CB0000CB53DC4F188210922804113019F4109284
:10CB100025041EC08091C40325E3829FC001112417
:10CB2000875A9C4F65EC73E040E0B4DA882309F043
:10CB30005DD8109225045CC0EB3319F481E080933A
:10CB4000280480912804882319F01150109325049B
:10CB50002091EA193091EB194091EC195091ED199F
:10CB60008091EE199091EF19A091F019B091F119FF
:10CB700082179307A407B50728F48091250480360F
:10CB800008F414CF1092F6198DE793E00E94BC369A
:10CB9000109225041092280480912A188D7F80938A
:10CBA0002A1826C010922A040F9486036B017C0178
:10CBB00084E095E0A7D2181619060CF4CBCE02CE6D
:10CBC0008091F619882309F0EBCE12C08091EA1902
:10CBD0009091EB19A091EC19B091ED198217930780
:10CBE000A407B50709F07DCFEA3309F089CF83CFD9
:10CBF000DF91CF911F910F91FF90EF90DF90CF9039
:10CC0000BF900895AB01BC0130EC2227B0E4AA1B11
:10CC100018F06A177B0720F06A1B7B0BA22BB32B43
:10CC200036952795B327A227441F551F661F771FE8
:10CC300040FFEECF18F0A617B70720F4530B6A0B8E
:10CC40007B0BA395550F661F771F10F0A617B7072C
:10CC5000A31FB31F5B2F4A2FCA0108954F925F9203
:10CC6000AF92BF92CF92DF92EF92FF920F9320E2AA
:10CC70008030920708F079C022E08030920708F0F7
:10CC80004AC08A30910510F48AE090E0A12C24E299
:10CC9000B22E24EFC22ED12CEE24FF18DD20A1F4F9
:10CCA000CC2009F012C001E1AA1CBB1C0A9509F4B2
:10CCB00031C0EE1CFF1CE81AF90A20F4E80EF91E38
:10CCC0008894F2CF0894F0CF12C009E1AA1CBB1CD3
:10CCD000CC1C0A9509F41EC0EE1CFF1CE81AF90AC8
:10CCE00020F4E80EF91E8894F1CF0894EFCF01E20A
:10CCF000AA1CBB1CCC1CDD1C0A9509F40BC0EE1C45
:10CD0000FF1CE81AF90A20F4E80EF91E8894F0CF07
:10CD10000894EECF51C0E6E4F7E1282F2F719695E5
:10CD200087959695879596958795969587958E7F05
:10CD3000E80FF91FA590B5902501059040180590C2
:10CD40005008249DC001259D900DE12D880F991F4D
:10CD5000EE1F880F991FEE1F880F991FEE1FA91A4B
:10CD6000BE0ACC24DD24112427C0E8E4F9E19C01AB
:10CD70003F709695969596959E7FE90FF11DA5902B
:10CD8000B59025010590401805905008249DC001DC
:10CD9000359DE02D259D900DE11D349D900DE11DEB
:10CDA000907F9295E2958E2F807F982BEF70A91A35
:10CDB000BE0ACC24DD241124B501C6010F91FF90D9
:10CDC000EF90DF90CF90BF90AF905F904F9008951D
:10CDD00014BCEEE6F0E080818260808314BC80E4C5
:10CDE00088BD8081846080831092800010928200D0
:10CDF000EFE6F0E0108289E0809381008CED9FEFF8
:10CE00009093890080938800808182608083089558
:10CE1000E0913904F0913A041995089580E48093E3
:10CE20007C0010924B0310924E0310924D0310920F
:10CE300053031092520310924C031092500310921D
:10CE40004F03109255031092540387EC80937A009D
:10CE500080917A0086FDFCCF8091780090917900D6
:10CE6000E0915103F0E0EE50FE4E949193FF04C028
:10CE700080917B00886003C080917B00877F8093D6
:10CE80007B0080917C009770807E982B90937C0033
:10CE900080917A00806480937A0008951F920F92A7
:10CEA0000FB60F9211242F933F934F938F939F931D
:10CEB00047B58091281881FF3BC080919D179091C4
:10CEC0009E17181619063CF580911B05813019F143
:10CED000169A81E006C080911B058F3F11F11698CC
:10CEE0008FEF80931B05485D11C0149A20919D1708
:10CEF00030919E1780911B05992787FD9095281BDF
:10CF0000390B30939E1720939D17149880919C178E
:10CF1000480F47BD0DC080919D1790919E1797FDBA
:10CF2000DACF80919D1790919E17892BF1F6EECF65
:10CF30009F918F914F913F912F910F900FBE0F9026
:10CF40001F9018951F920F920FB60F920BB60F926B
:10CF500011242F938F939F93EF93FF932091C600FB
:10CF60009091C0049F5F9F778091C104981741F012
:10CF7000E091C004F0E0E05CFB4F20839093C0049C
:10CF8000FF91EF919F918F912F910F900BBE0F907A
:10CF90000FBE0F901F9018951F920F920FB60F9211
:10CFA0000BB60F9211248F939F93EF93FF93909161
:10CFB000020580910305981731F48091C1008F7D9F
:10CFC0008093C1000EC0E0910305F0E0EE53FB4FEB
:10CFD0009081809103058F5F8F73809303059093F9
:10CFE000C600FF91EF919F918F910F900BBE0F9014
:10CFF0000FBE0F901F901895AF92BF92DF92EF92E5
:10D00000FF920F931F93CF93DF93EC017A018B0173
:10D01000DD24403081EE580780E0680780E0780723
:10D0200011F0DD24D394E1E0AE2EB12CEC85FD852A
:10D03000DD2069F0C5010E8802C0880F991F0A948F
:10D04000E2F7808360E079E08DE390E005C0108234
:10D0500060E874E88EE190E0A80197010F948B0ED0
:10D060002150304040405040569547953795279580
:10D0700080E12030380720F0DD2011F0DD24D6CF0C
:10D08000E885F9853083EA85FB852083EE85FF8579
:10D09000408121E030E0C9010A8802C0880F991F51
:10D0A0000A94E2F7482B4083EE85FF854081C90151
:10D0B0000B8802C0880F991F0A94E2F7482B40831F
:10D0C000EE85FF854081C9010C8802C0880F991F39
:10D0D0000A94E2F7482B4083EE85FF8580810D8816
:10D0E00002C0220F331F0A94E2F7209528232083E1
:10D0F000DF91CF911F910F91FF90EF90DF90BF9044
:10D10000AF900895DC011496ED91FC911597E058CD
:10D11000FF4F2191808130E020583F4F281B31097B
:10D120002F773070C9010895DC011496ED91FC91C0
:10D130001597E058FF4F9081E058F040DF01AF575E
:10D14000BF4F8C91981719F42FEF3FEF06C08C91C9
:10D15000E80FF11D8081282F30E0C9010895DC011E
:10D160001496ED91FC911597E058FF4F9081E0588F
:10D17000F040DF01AF57BF4F8C91981719F42FEF94
:10D180003FEF0AC08C91E80FF11D90818C918F5F69
:10D190008F778C93292F30E0C9010895FC01868197
:10D1A0009781DC01A05CBF4FFC01EF5BFF4F9C91BE
:10D1B00080819817E1F70895CF93DF93EC01EE811A
:10D1C000FF81E05CFF4F9081E054F0409F5F9F73D0
:10D1D000DF01AF5BBF4F8C919817E9F3E05CFF4F25
:10D1E0008081E054F040E80FF11D6083EE81FF8103
:10D1F000E05CFF4F9083EE85FF85208181E090E029
:10D200000D8802C0880F991F0A94E2F7282B20830B
:10D2100081E090E0DF91CF91089510920705109280
:10D2200006058BE393E0909305058093040580E465
:10D2300094E0909309058093080582EC94E0909324
:10D240000B0580930A0585EC90E090930D05809383
:10D250000C0584EC90E090930F0580930E0580EC14
:10D2600090E0909311058093100581EC90E09093ED
:10D2700013058093120586EC90E09093150580933A
:10D28000140584E08093160583E08093170587E0FA
:10D290008093180585E08093190581E080931A0535
:10D2A00008951F920F920FB60F920BB60F92112492
:10D2B0002F933F934F935F936F937F938F939F939E
:10D2C000AF93BF93CF93DF93EF93FF9388B5805CC9
:10D2D00088BD90912005992391F4809132058E7F2D
:10D2E00080931C0581112C9A8091330580931D0534
:10D2F000882329F08091020180628093020170915D
:10D300002105772359F48091350580931F058823E3
:10D3100029F08091020180648093020180911C05B4
:10D32000891719F49E3F09F02C9880911F058717E3
:10D3300039F47F3F29F0809102018F7B80930201B5
:10D3400080911D05891739F49E3F29F080910201D3
:10D350008F7D8093020178948091480390914903D6
:10D36000019690934903809348038658914038F082
:10D37000109249031092480381E080934A03809100
:10D380007A0086FD4EC060915103862F90E0409157
:10D39000780050917900DC01AA0FBB1FED01C35B3F
:10D3A000DC4F28813981420F531F59834883FC0188
:10D3B000E55BFC4F80818F5F8083803268F183E082
:10D3C000569547958A95E1F7AE5ABC4F11965C93F6
:10D3D0004E93198218821082862F8F5F809351039B
:10D3E000823010F010925103E0915103F0E0EE50C2
:10D3F000FE4E949193FF04C080917B00886003C02F
:10D4000080917B00877F80937B0080917C00977068
:10D41000807E982B90937C0080917A00806480932A
:10D420007A0072FF04C085E29CE10E9461D680917F
:10D4300021058F5F80932105809120058E5F809369
:10D440002005FF91EF91DF91CF91BF91AF919F9117
:10D450008F917F916F915F914F913F912F910F909D
:10D460000BBE0F900FBE0F901F9018951F920F923A
:10D470000FB60F920BB60F9211242F933F934F9339
:10D480005F936F937F938F939F93AF93BF93EF932C
:10D49000FF9380913B04882309F0DAC080E070910B
:10D4A0003E04772381F470913D04772319F4609151
:10D4B0003C0491F0709389006093880010923C04C2
:10D4C00010923D0408C060913D0460587040609324
:10D4D0003D0470933E0481E0882309F0B9C081E0E7
:10D4E00080933B0488E49EEE9093890080938800AB
:10D4F00080918B17882309F42EC0B8D5F89488231F
:10D50000E1F47F3FD1F010923C0410923D04109260
:10D510003E04809184009091850024E6820F911D45
:10D520006817790728F4909389008093880012C0C7
:10D5300070938900609388000DC07058804060939C
:10D540003C0470933D0480933E0490E890938900DE
:10D55000109288007BC08091E117882309F437C0BE
:10D560000E942AA180914F1890915018A0915118B3
:10D57000B0915218F894AA23E1F49F3FD1F0109291
:10D580003C0410923D0410923E04A0918400B0919E
:10D59000850024E6A20FB11D8A179B0728F4B093DB
:10D5A0008900A093880012C090938900809388001E
:10D5B0000DC09058A04080933C0490933D04A093EC
:10D5C0003E04B0E8B0938900109288003FC080917B
:10D5D000360590913705892B11F520915F18309110
:10D5E000601821153105B1F080919D1790919E171B
:10D5F000821B930B90939E1780939D1710925B183C
:10D6000010925C1810925D1810925E1810926018BB
:10D6100010925F1880919D1790919E1709C080917C
:10D62000360590913705019790933705809336051D
:10D6300010923C0410923D0410923E0410923F045C
:10D640008CED9FEF909389008093880010923B04AB
:10D65000FF91EF91BF91AF919F918F917F916F91CA
:10D660005F914F913F912F910F900BBE0F900FBE86
:10D670000F901F901895FF920F931F93FFB6F89489
:10D6800084E090E00F9409028C010F94A6022DB75C
:10D690003EB7FFBE201B310BC9011F910F91FF90B8
:10D6A00008951F9384B7182F10FF04C088EE93E0ED
:10D6B0000E94CA3611FF04C080EF93E00E94CA3670
:10D6C00012FF04C08FEF93E00E94CA3613FF04C01C
:10D6D0008FE094E00E94CA3615FF04C08EE194E00A
:10D6E0000E94CA3614BE1F910895CF92DF92EF9226
:10D6F000FF920F931F93CF93DF93FC016B01642F75
:10D70000922F8091281881FFAEC020915B18309134
:10D710005C1840915D1850915E18992339F4790195
:10D720008A0120E0EF01C15FDE4F29C010E0EF0168
:10D73000C15FDE4F09C088819981AA81BB81280F12
:10D74000391F4A1F5B1F1F5F1617A8F3ED5EFE4FC0
:10D75000E080F18002811381E351F140E216F3068B
:10D7600004071507ECF079018A011AC088819981B4
:10D77000AA81BB81E81AF90A0A0B1B0B2F5F261737
:10D78000A8F3E55EFE4F80819181A281B381EB51C8
:10D79000F140E816F9060A071B0714F47C018D0115
:10D7A000E15EFE4F80819181B601AC012227579F37
:10D7B000D001649FC001659F900DA11DB21F749F91
:10D7C000900DA11DB21F11248E0D9F1DA01FB11F12
:10D7D000CD01BB2797FDB095AB2FAC01F89480919C
:10D7E0009D1790919E1720915F1830916018821BB1
:10D7F000930B840F951F90939E1780939D1714167B
:10D80000150684F4121613066CF080919D17909102
:10D810009E17E0915603F091570325A536A5820F78
:10D82000931F10C057FF12C037FD10C080919D1785
:10D8300090919E17E0915603F091570325A536A5C8
:10D84000821B930B90939E1780939D1750936018A3
:10D8500040935F187894E0925B18F0925C18009304
:10D860005D1810935E18DF91CF911F910F91FF907B
:10D87000EF90DF90CF9008952F923F924F925F925A
:10D880006F927F928F929F92AF92BF92CF92DF92D0
:10D89000EF92FF920F931F93DF93CF93CDB7DEB735
:10D8A0002A970FB6F894DEBF0FBECDBF9A8789873F
:10D8B000FC01808180FD4FC1818180FD4CC12CC065
:10D8C0002E5F3F4FC901A0E0B0E0841B950BA60B73
:10D8D000B70BB595A79597958795BC0168167906FE
:10D8E00008F4C301681A790AF20171826082E9853D
:10D8F000FA85E150FF4F408151819B014617570740
:10D9000008F49A01421B530B51834083E985FA8541
:10D910008081816080831FC129853A85235C3F4FC8
:10D92000F901E080F18002811381FD97FA87E98790
:10D93000E75BFF4FC801B7012081318142815381EC
:10D940000F94620D69837A838B839C83E985FA85C2
:10D95000E35BFF4FC801B7012081318142815381D0
:10D960000F94620D6D837E838F8398876BE0C62E44
:10D9700061E0D62E29853A85C20ED31E275F3E4F21
:10D980003A872987F901A080B180B50180E090E055
:10D990000F94520B7B018C0129813A814B815C8170
:10D9A0000F94620D0F94260B3B014C01F60171831D
:10D9B000608329853A852C5F3F4F3A872987C801C4
:10D9C000B7012D813E814F8158850F94620D0F94D0
:10D9D000260B1B012C01E985FA8571836083ED50CC
:10D9E000F140C501889F5001999F6001899F882758
:10D9F000B00CC11CD81EB00CC11CD81E1124930140
:10DA0000229FC001339FD001239F2227900DA11D8B
:10DA1000B21F900DA11DB21F11245DEF452E512C98
:10DA20004E0E5F1EA6019501281B390B4A0B5B0B9E
:10DA3000CA01B901EF5FFE4FFA87E987E080F18004
:10DA400002811381EE0CFF1C001F111FA80197011A
:10DA50000F948B0E39010894611C711CF2017182C4
:10DA600060829101229FC001339FD001239F222712
:10DA7000900DA11DB21F900DA11DB21F1124A81A57
:10DA8000B90ACA0ADB0AC601B501A80197010F94B9
:10DA90008B0E79018A010894E11CF11CE985FA8555
:10DAA000F292E292EF5FF04037E1832E31E0932E65
:10DAB0008E0E9F1EED5EFE4FFA87E98760817181B1
:10DAC000828193810F94540B5B016C0129813A810F
:10DAD0004B815C810F94620D29813A814B815C817D
:10DAE0000F94620D0F94210BF40160837183828384
:10DAF000938329853A85285F3F4F3A872987C60156
:10DB0000B5012D813E814F8158850F94620D2D8185
:10DB10003E814F8158850F94620D0F94210BE9854A
:10DB2000FA85608371838283938393012E0D3F1D59
:10DB300036964081518162817381E152F140FA87CA
:10DB4000E987C901A0E0B0E084179507A607B707E9
:10DB50000CF0B6CEDBCE2A960FB6F894DEBF0FBE21
:10DB6000CDBFCF91DF911F910F91FF90EF90DF908C
:10DB7000CF90BF90AF909F908F907F906F905F906D
:10DB80004F903F902F900895FF920F931F93282F4F
:10DB9000162F80918B17882309F042C0809136059B
:10DBA00090913705892BE1F52223D1F133E0A5E2ED
:10DBB000B1E0FF24F39407E040E553EC60E070E04F
:10DBC000315020918A17822F90E08A9FF0018B9F1D
:10DBD000F00D9A9FF00D1124E85CFA4FF18200835A
:10DBE0001086832F810F82834383548365837683DA
:10DBF0002F5F20938A17203110F010928A1780919E
:10DC00002A18806180932A189FB7F89480918B1707
:10DC10008F5F80938B179FBF332391F681E001C004
:10DC200080E01F910F91FF9008952F923F924F92A5
:10DC30005F926F927F928F929F92AF92BF92CF929C
:10DC4000DF92EF92FF920F931F93DF93CF93CDB7A5
:10DC5000DEB768970FB6F894DEBF0FBECDBF9A8BC4
:10DC6000898B788F6F8B5C8B4B8B3E8B2D8BDA0186
:10DC700018962D903D904D905C901B97F901E08493
:10DC8000F18402851385DB0118966D907D908D904F
:10DC90009C901B97C201B1016E197F09800B910BFB
:10DCA00014962D913D914D915C9117970F94380EDC
:10DCB0005B016C01E618F70808091909EB89FC8972
:10DCC0002481358146815781C801B7010F94380EF0
:10DCD000A60EB71EC81ED91E6218730884089508C0
:10DCE000AD89BE8914962D913D914D915C91179708
:10DCF000C401B3010F94380EA60EB71EC81ED91E5C
:10DD0000E989FA89A082B182C282D382AB89BC89B7
:10DD10002D903D904D905C90ED89FE8960807180E2
:10DD200082809380AF89B88DAD90BD90CD90DC900E
:10DD3000C401B3016A197B098C099D09EB89FC892F
:10DD400020853185428553850F94380E7B018C01E7
:10DD5000C201B1016619770988099909AF89B88D9F
:10DD600018962D913D914D915C911B970F94380E13
:10DD7000E60EF71E081F191FA218B308C408D5081D
:10DD8000ED89FE892085318542855385C601B5011F
:10DD90000F94380EE60EF71E081F191FA989BA89BD
:10DDA0001496ED92FD920D931C931797EB89FC89C5
:10DDB0002480358046805780AD89BE891496ED90C9
:10DDC000FD900D911C911797EF89F88D64807580F7
:10DDD00086809780C201B1016E197F09800B910B7B
:10DDE00020813181428153810F94380E5B016C0197
:10DDF000E618F70808091909AB89BC892D913D91EE
:10DE00004D915C91C801B7010F94380EA60EB71E54
:10DE1000C81ED91E6218730884089508ED89FE890A
:10DE20002081318142815381C401B3010F94380EA6
:10DE3000A60EB71EC81ED91EA989BA891896AD921A
:10DE4000BD92CD92DC921B97AB89BC8914968D91C3
:10DE50009D910D90BC91A02D8D879E87AF87B88B2B
:10DE6000ED89FE89208431844284538464807580E6
:10DE700086809780AB89BC8918968D919D910D9075
:10DE8000BC91A02D89879A87AB87BC87AF89B88D55
:10DE900018968D919D910D90BC91A02D8D839E83A0
:10DEA000AF83B887AF89B88D14968D919D910D90F1
:10DEB000BC91A02D89839A83AB83BC83C201B1013D
:10DEC0002D853E854F8558890F94380E7B018C0136
:10DED000C401B30129853A854B855C850F94380EC2
:10DEE000E61AF70A080B190BEF89F88D20813181AA
:10DEF00042815381C801B7010F94380E5B016C0158
:10DF0000C401B3012D813E814F8158850F94380E95
:10DF10007B018C01C201B10129813A814B815C8175
:10DF20000F94380EE61AF70A080B190BAB89BC8957
:10DF30002D913D914D915C91C801B7010F94380E20
:10DF4000A60EB71EC81ED91E69857A858B859C854D
:10DF500029813A814B815C810F94380E7B018C01C1
:10DF60006D857E858F8598892D813E814F8158856D
:10DF70000F94380EE61AF70A080B190BED89FE8983
:10DF80002081318142815381C801B7010F94380E3D
:10DF9000A60EB71EC81ED91EA989BA891C96AD92B5
:10DFA000BD92CD92DC921F9768960FB6F894DEBFB3
:10DFB0000FBECDBFCF91DF911F910F91FF90EF90DA
:10DFC000DF90CF90BF90AF909F908F907F906F9099
:10DFD0005F904F903F902F9008958F929F92AF92B5
:10DFE000BF92CF92DF92EF92FF920F931F936C013B
:10DFF000CB01BA0148015901F601208131814281EA
:10E0000053810F94380EF601E484F5840685178554
:10E01000E61AF70A080B190B2481358146815781CE
:10E02000C501B4010F94380EE61AF70A080B190B54
:10E03000C801B7010F94540B7B018C01F601608578
:10E040007185828593850F94540B9B01AC01C801A7
:10E05000B7010F94B90A1F910F91FF90EF90DF90D5
:10E06000CF90BF90AF909F908F9008956F927F92C6
:10E070008F929F92AF92BF92CF92DF92EF92FF92D8
:10E080000F931F93CF93DF938091881790918917F7
:10E09000892B09F029C281E090E0A0E0B0E08093F4
:10E0A000DE029093DF02A093E002B093E102809140
:10E0B0008C1790E025E231E0829FF001839FF00D04
:10E0C000929FF00D1124E85CFA4FF0938917E093CA
:10E0D0008817818187FF15C08091DC029091DD0255
:10E0E0008E179F0709F44AC07894F093DD02E093FD
:10E0F000DC0260918B178DED93E070E00E94643636
:10E100003DC078948FEF9FEF9093DD028093DC0207
:10E1100080912E0385FF26C080918C178F5F80939E
:10E120008C17803110F010928C1710928917109272
:10E130008817F89480918B17815080938B1780916A
:10E140008B17882329F480912A188F7E80932A18B0
:10E1500080918B17882309F07AC785E29CE164E7F8
:10E1600079E16AC0E0918817F0918917818180FF79
:10E1700030C090918B178281891748F010928917CF
:10E180001092881720ED37E040E050E067C7238108
:10E1900034814581568180918C178F5F80938C17D5
:10E1A000803110F010928C171092891710928817F6
:10E1B000F89480918B17815080938B1780918B17E7
:10E1C000882309F04BC780912A188F7E80932A18E4
:10E1D00045C78091281886FF52C780919D1890915D
:10E1E0009E18A0919F18B091A018B7FD48C78091C4
:10E1F0008C178F5F80938C17803110F010928C17E2
:10E200001092891710928817F89480918B1781507B
:10E2100080938B1780918B17882329F480912A187B
:10E220008F7E80932A1880918B17882309F00FC75F
:10E2300085E29CE16FE679E140E020E00E9460D554
:10E2400006C71298808186608083A0918817B0915C
:10E250008917FD01E75AFF4F8081882309F483C0A5
:10E260008150808390E09C0173E0220F331F7A95E8
:10E27000E1F7281B390BC901815A9F4F8A0F9B1F59
:10E2800090939217809391175F988A9880910801D4
:10E290008E7F80930801E0918817F0918917A20F73
:10E2A000B31FA15ABF4F80859C91892B8087E09135
:10E2B0008817F09189178781EF01C55ADF4F8430A5
:10E2C000F9F4288139814A815B81DA01C901B59568
:10E2D000A7959795879581A392A3A3A3B4A3858FB0
:10E2E000968FA78FB0A3818F928FA38FB48F209327
:10E2F000931730939417409395175093961720C017
:10E3000088819981AA81BB8181A392A3A3A3B4A38D
:10E31000858F968FA78FB0A3818F928FA38FB48F95
:10E32000880F991FAA1FBB1F88839983AA83BB8369
:10E330008093931790939417A0939517B093961783
:10E34000E0918817F0918917E55AFF4F80819181FC
:10E35000A281B3818093971790939817A0939917F0
:10E36000B0939A1704C01092921710929117E091EF
:10E370008817F09189178781EF5DFE4F843029F46B
:10E3800080819181A281B38108C080819181A28125
:10E39000B381880F991FAA1FBB1F80938D1790937D
:10E3A0008E17A0938F17B0939017E0918817F09174
:10E3B0008917808180FD02C0CF015EDAE091881765
:10E3C000F0918917E55FFE4F8081918190931A1932
:10E3D00080931919109257181092581810925918C2
:10E3E00010925A18109253181092541810925518EF
:10E3F00010925618F894E0919117F0919217309777
:10E4000009F18081282F30E0C90181719070419716
:10E4100011F4899801C0899AC9018272907082971B
:10E4200011F48F9801C08F9A247430702434310510
:10E4300021F480910B018D7F03C080910B018260DC
:10E4400080930B018091281881FD0BC0E091881703
:10E45000F091891780858878883811F4169A01C060
:10E460001698E0918817F0918917E95EFE4F808138
:10E470009181A281B38180935B1890935C18A093E3
:10E480005D18B0935E183C9760817181EB50F1404C
:10E49000CF0140E020E029D980912319E09188172D
:10E4A000F09189178823C9F08781843009F0ECC581
:10E4B0001092231980914F1890915018A0915118E3
:10E4C000B09152189C01AD01220F331F441F551FFC
:10E4D000280F391F4A1F5B1FC1C58781843009F48B
:10E4E000D3C581E0809323197894E0918817F09147
:10E4F0008917B780A6E0AA2EAB2024E0B21619F047
:10E5000083E08B198783AA2009F4C7C0C0919117B3
:10E51000D0919217209709F4C0C0E0918817F0912C
:10E52000891741818091281886FF45C08881282F4E
:10E5300030E0C901847490708034910509F0ADC554
:10E540004B9BABC580858F7880871882EF5DFE4F2F
:10E5500080819181A281B38180939D1890939E18B0
:10E56000A0939F18B093A018108211821282138278
:10E5700094C0C901817190704197E9F422723070A2
:10E5800022323105C1F4649903C08CC54A9B13C083
:10E5900080858F7880871882EF5DFE4F8081918122
:10E5A000A281B38180939D1890939E18A0939F1889
:10E5B000B093A01872C044FF70C08881817181310E
:10E5C000C1F4649B16C0EF5DFE4F80819181A281F2
:10E5D000B381E152F1408093A1189093A218A093C7
:10E5E000A318B093A41888818F7E888380858F7E3E
:10E5F0008087888182728232D1F48091030180FF0A
:10E6000016C0EF5DFE4F80819181A281B381E152FE
:10E61000F1408093A5189093A618A093A718B093E3
:10E62000A81888818F7D888380858F7D80879881D9
:10E63000892F8171813139F4649B05C09F7E988355
:10E6400080858F7E80879881892F8272823249F4FB
:10E650008091030180FF05C09F7D988380858F7D19
:10E660008087888184748434C1F44A9B16C0EF5D2E
:10E67000FE4F80819181A281B381E152F14080936C
:10E680009D1890939E18A0939F18B093A01888810E
:10E690008F7B888380858F7B8087E0918817F091BE
:10E6A0008917EF5DFE4FE080F18002811381809138
:10E6B0002F03282F30E040E050E0E216F306040775
:10E6C000150714F4A80197016901F8941E141F049A
:10E6D000100611060CF059C400E010E0E1E06E2EC7
:10E6E000712C812C912C77E0F72E8EC2101611061A
:10E6F00024F481E090E00F94ED03E0918817F0910D
:10E700008917608567FF42C085A196A1A7A1B0A522
:10E71000258936894789508D821B930BA40BB50B35
:10E7200085A396A3A7A3B0A7B7FF30C080912818F0
:10E7300081FF13C06878683831F480919D179091FB
:10E740009E17019605C080919D1790919E17019785
:10E7500090939E1780939D1701C0149AE09188179B
:10E76000F091891785A196A1A7A1B0A520918D1739
:10E7700030918E1740918F1750919017820F931FF1
:10E78000A41FB51F85A396A3A7A3B0A7E0919117D7
:10E79000F0919217309709F42AC2808184FF2BC030
:10E7A000C0918817D09189172181328140E050E0D3
:10E7B000898D9A8DAB8DBC8D821B930BA40BB50BF1
:10E7C000898F9A8FAB8FBC8FB7FF15C0889A898DC0
:10E7D0009A8DAB8DBC8D20919317309194174091F9
:10E7E000951750919617820F931FA41FB51F898FFD
:10E7F0009A8FAB8FBC8FA0919117B09192178C918B
:10E8000085FF2DC0E0918817F091891713962D91FF
:10E810003C91149740E050E0858D968DA78DB0A176
:10E82000821B930BA40BB50B858F968FA78FB0A37C
:10E83000B7FF15C08E9A858D968DA78DB0A12091BA
:10E840009317309194174091951750919617820F16
:10E85000931FA41FB51F858F968FA78FB0A3C0915C
:10E860009117D0919217888186FF50C0E091881748
:10E87000F09189172D813E8140E050E081A192A165
:10E88000A3A1B4A1821B930BA40BB50B81A392A3EC
:10E89000A3A3B4A3B7FF3AC080910B018860809313
:10E8A0000B0181A192A1A3A1B4A120919317309152
:10E8B00094174091951750919617820F931FA41F9C
:10E8C000B51F81A392A3A3A3B4A32091951830915F
:10E8D00096184091971850919818888184748434C0
:10E8E00029F08FEF9FEFAFEFBFEF04C081E090E022
:10E8F000A0E0B0E0820F931FA41FB51F809395186E
:10E9000090939618A0939718B093981880919717A2
:10E9100090919817A0919917B0919A170197A10912
:10E92000B1098093971790939817A0939917B09374
:10E930009A170097A105B10509F059C120918817D0
:10E9400030918917F901E75AFF4F8081882309F434
:10E950004AC16092DE027092DF028092E0029092E1
:10E96000E1028081815080838F9DE0011124C15A92
:10E97000DF4FC20FD31FD0939217C0939117E0912E
:10E980008817F0918917E55AFF4F20813181428124
:10E990005381EB55F040DA01C901B595A7959795DC
:10E9A000879581A392A3A3A3B4A3858F968FA78FE6
:10E9B000B0A3818F928FA38FB48F2093971730933A
:10E9C00098174093991750939A178881282F30E011
:10E9D00080FF02C0899801C0899A21FF02C08F98E8
:10E9E00001C08F9A22FF04C080910B018D7F03C06C
:10E9F00080910B01826080930B018091E117882345
:10EA000009F4F5C0CD2B09F4F2C02077307020371F
:10EA1000310509F0ECC088988E9880910B01877FB2
:10EA200080930B0182E090E00F94ED038091E11759
:10EA3000E0919117F091921718160CF067C0808141
:10EA400080FF02C0889A18C0E0918817F09189175A
:10EA5000818D928DA38DB48D209193173091941751
:10EA60004091951750919617820F931FA41FB51FC1
:10EA7000818F928FA38FB48FE0919117F0919217AD
:10EA8000808181FF02C08E9A18C0E0918817F091B2
:10EA90008917858D968DA78DB0A120919317309100
:10EAA00094174091951750919617820F931FA41FAA
:10EAB000B51F858F968FA78FB0A3E0919117F09126
:10EAC0009217808182FF06C080910B01886080933D
:10EAD0000B0118C0E0918817F091891781A192A1CC
:10EAE000A3A1B4A120919317309194174091951749
:10EAF00050919617820F931FA41FB51F81A392A355
:10EB0000A3A3B4A38091E117815066C0808180FFE8
:10EB100019C0E0918817F0918917818D928DA38D8E
:10EB2000B48D20919317309194174091951750917F
:10EB30009617820F931FA41FB51F818F928FA38FEB
:10EB4000B48F01C0889AE0919117F091921780815B
:10EB500081FF19C0E0918817F0918917858D968DF6
:10EB6000A78DB0A1209193173091941740919517DC
:10EB700050919617820F931FA41FB51F858F968FF4
:10EB8000A78FB0A301C08E9AE0919117F0919217D0
:10EB9000808182FF19C0E0918817F091891781A1C7
:10EBA00092A1A3A1B4A12091931730919417409101
:10EBB000951750919617820F931FA41FB51F81A31D
:10EBC00092A3A3A3B4A305C080910B018860809396
:10EBD0000B018091E1178F5F8093E11781E090E056
:10EBE0000F94ED0304C01092921710929117889819
:10EBF0008E9880910B01877F80930B01809128185C
:10EC000081FF14980F5F1F4F0C151D050CF46ECD7E
:10EC100085E0B82209F48CC17894C0918817D0910E
:10EC20008917C350DF4F68817981CD5FD0409B0148
:10EC300040E050E08091571890915818A0915918D1
:10EC4000B0915A18281739074A075B0708F494C08F
:10EC50001092DE021092DF021092E0021092E102A6
:10EC600020915318309154184091551850915618CE
:10EC7000CB5FDE4F88819981AA81BB81BA01A9014E
:10EC8000589F212D5A9F302D412D599F200D311D08
:10EC90004B1F689F200D311D4B1F699F300D411D7B
:10ECA000789F300D411D6A9F400D799F400D46951C
:10ECB000379527954695379527951124269688816F
:10ECC0009981820F931F90931A1980931919FE014D
:10ECD000329122912817390720F430931A19209382
:10ECE00019192091191930911A199EE2213E3907FC
:10ECF00090F08DE5213C380740F084E080932F03AD
:10ED0000369527953695279509C082E080932F0385
:10ED10003695279503C081E080932F03C9010E9497
:10ED20002E669B01AC0120934F18309350184093EE
:10ED30005118509352188091531890915418A091E3
:10ED40005518B0915618820F931FA41FB51F8093BA
:10ED5000531890935418A0935518B0935618609177
:10ED6000191970911A1980918817909189174C2D53
:10ED700021E00E94756BDCC0FE01EF5DFE4FC150CB
:10ED8000DF4F88819981CF5FD040A0E0B0E0208143
:10ED900031814281538182179307A407B5077CF024
:10EDA000898182FD84C110925318109254181092D8
:10EDB00055181092561889818460898378C1109201
:10EDC000DE021092DF021092E0021092E102672B45
:10EDD00009F457C05DC0E35FFE4FC081D181ED50A3
:10EDE000F1400EC0E35FFE4F20813181ED50F140D4
:10EDF000CB018C1B9D0BEC018217930708F4E901F2
:10EE0000CF01BE014C2D20E00E94756B9EE2C13EF9
:10EE1000D90790F02DE5C13CD20740F084E0809303
:10EE20002F03D695C795D695C79509C082E08093E4
:10EE30002F03D695C79503C081E080932F03CE01A1
:10EE40000E942E669B01AC0120934F1830935018FE
:10EE50004093511850935218809153189091541820
:10EE6000A0915518B0915618820F931FA41FB51F7B
:10EE70008093531890935418A0935518B093561834
:10EE800057C0C75FDE4F68817981C950D14004C047
:10EE90006091191970911A19CE0140E021E00E9489
:10EEA000756BE0918817F0918917E350FF4F8081CF
:10EEB0009181ED5FF040892BD9F5E75FFE4F8081AE
:10EEC0009181E950F1402EE2813E920700F1E75036
:10EED000FF4F815C9D4578F084E080932F03808113
:10EEE0009181A281B38102E0880F991FAA1FBB1FE5
:10EEF0000A95D1F715C082E080932F03808191811C
:10EF0000A281B381880F991FAA1FBB1F09C081E08E
:10EF100080932F03E750FF4F80819181A281B381BD
:10EF200080934F1890935018A0935118B093521893
:10EF3000AA2059F19601442737FD4095542F80911E
:10EF4000571890915818A0915918B0915A18820FDB
:10EF5000931FA41FB51F8093571890935818A09320
:10EF60005918B0935A18E0918817F0918917EF5DFE
:10EF7000FE4F80819181A281B381821B930BA40BF0
:10EF8000B50B80839183A283B383E0918817F091BE
:10EF90008917878120914F1830915018409151184E
:10EFA00050915218843019F479018A0106C0790110
:10EFB0008A0116950795F794E794AA2009F44CC0A6
:10EFC000EF5DFE4F80819181A281B381E152F140DA
:10EFD000181619061A061B061CF48085807FE1F5B9
:10EFE00080918C178F5F80938C17803110F0109276
:10EFF0008C171092891710928817F89480918B17AC
:10F00000815080938B1780918B17882329F48091EE
:10F010002A188F7E80932A1880918B17882341F4B9
:10F0200085E29CE16AE679E140E020E00E9460D55B
:10F03000A8019701559547953795279520934F1827
:10F0400030935018409351185093521807C028EE2F
:10F0500033E040E050E002C0A8019701B901CA01C5
:10F06000DF91CF911F910F91FF90EF90DF90CF90A4
:10F07000BF90AF909F908F907F906F900895808504
:10F0800088230CF0DFC8DDC820914F18309150184C
:10F090004091511850915218E1CF8434910509F0F4
:10F0A0008ACA67CA8091030180FD72CA6FCAE09163
:10F0B0008817F09189172091531830915418409176
:10F0C000551850915618EB5FFE4F80819181A281B7
:10F0D000B381E550F140389FC12D3A9FD02D212DAD
:10F0E000399FC00DD11D2B1F489FC00DD11D2B1F57
:10F0F000499FD00D211D589FD00D211D4A9F200DE5
:10F10000599F200D2695D795C7952695D795C795D4
:10F1100011246091191970911A196C177D0708F460
:10F120005ACE60CECF93DF93C82FD0E004C00E94A8
:10F13000C9630E94711C80918B179E01280F311D9D
:10F1400021313105A4F7DF91CF9108952F923F929D
:10F150004F925F926F927F928F929F92AF92BF92E7
:10F16000CF92DF92EF92FF920F931F93DF93CF9393
:10F17000CDB7DEB7EF970FB6F894DEBF0FBECDBFA9
:10F180004C017EAB6DAB58AF4FAB09AF1AAF2BAF95
:10F190003CAFEDAEDA01AD90BD90CD90DD90BCAB53
:10F1A000ABABC601B501F4012081318142815381AD
:10F1B0000F94EC096BA37CA38DA39EA3AFA9B8AD5C
:10F1C0001496ED90FD900D911C911797C801B70111
:10F1D000F40124813581468157810F94EC096F8FAA
:10F1E00078A389A39AA320911818309119184091F7
:10F1F0001A1850911B182FA738AB49AB5AAB809106
:10F20000F0179091F117A091F217B091F3178BA717
:10F210009CA7ADA7BEA72091AC173091AD17409128
:10F22000AE175091AF172FA338A749A75AA7D601F9
:10F23000C501B0588B8F9C8FAD8FBE8FA8019701F1
:10F2400050582F8B388F498F5A8FADA9BEA96D9119
:10F250007D918D919C912BA13CA14DA15EA10F941C
:10F26000EB095B016C01EDA9FEA9648175818681C2
:10F2700097812F8D38A149A15AA10F94EB093B0129
:10F280004C016B8D7C8D8D8D9E8DA40193010F940F
:10F29000620D7B018C016F89788D898D9A8DA60115
:10F2A00095010F94620D9B01AC01C801B7010F9449
:10F2B000EB091B012C016B8D7C8D8D8D9E8DA60124
:10F2C00095010F94620D7B018C016F89788D898D7A
:10F2D0009A8DA40193010F94620D9B01AC01C801AA
:10F2E000B7010F94EC099B01AC01C201B1010F946D
:10F2F0005F0A5B016C0120E030E040E050E00F94D9
:10F30000B20A882354F4C601B5012BED3FE049EC65
:10F3100050E40F94EC095B016C01FDADFF2351F04B
:10F32000C601B5012BED3FE049EC50E40F94EB0929
:10F330005B016C01C601B5019F7729AD3AAD4BADBC
:10F340005CAD0F94620D3B014C012FE632E143E8C6
:10F350005AE30F94B20A87FDE5C1E0900519F090D9
:10F3600006190091071910910819C801B70120E08A
:10F3700030E040E752E40F94C00C1816F4F4C801D2
:10F38000B7012DE83AE748E85CE30F94620D0F946B
:10F39000210B9B016430710514F023E030E0B901CA
:10F3A000882777FD8095982F0F94540B9B01AC0113
:10F3B000C401B3010F94B90A02C0C401B3010F9490
:10F3C0008F0B0F94260B7E8B6D8B2D893E89232B03
:10F3D00021F441E050E05E8B4D8BAD89BE89BD01CB
:10F3E00080E090E00F94520B7B018C01C601B501C7
:10F3F000A80197010F94B90A698B7A8B8B8B9C8B30
:10F400002FA538A949A95AA98BA59CA5ADA5BEA52C
:10F41000281B390B4A0B5B0B2FA738AB49AB5AABF8
:10F42000CA01B9010F94540B2FA138A549A55AA5BB
:10F430000F94620DA80197010F94B90A6D877E871A
:10F440008F87988B69897A898B899C8920E030E045
:10F4500040E05FEB0F94620D29893A894B895C8902
:10F460000F94620D20E030E040E85FE30F94EC0978
:10F4700069877A878B879C876BA57CA58DA59EA5C0
:10F480000F94540B2FA138A549A55AA50F94620DCE
:10F4900069837A838B839C83A1E0B0E0BFAFAEAF7A
:10F4A00099240DC1892D992787FD909583709070BF
:10F4B000892B41F40E94C9630E94711C85E29CE182
:10F4C0000E945FD6B8E1B9150CF446C06B8D7C8DF7
:10F4D0008D8D9E8D29893A894B895C890F94620DA7
:10F4E0007B018C016F89788D898D9A8D29853A856C
:10F4F0004B855C850F94620D9B01AC01C801B7017F
:10F500000F94EC097B018C016B8D7C8D8D8D9E8D14
:10F5100029853A854B855C850F94620D5B016C01F2
:10F520006F89788D898D9A8D29893A894B895C8973
:10F530000F94620D9B01AC01C601B5010F94EB095C
:10F540006B8F7C8F8D8F9E8F9394C701D8018F8B8B
:10F55000988FA98FBA8F61C0EEADFFADBF0180E07B
:10F5600090E00F94520B29893A894B895C890F945A
:10F57000620D7B018C01C8010F94B60A6D837E83F6
:10F580008F839887B701C8010F94C50D3B014C01CB
:10F59000AFA9B8ADED90FD900D911C9117FB1095A2
:10F5A00017F91095EBA9FCA9208031804280538087
:10F5B000C801B7012D813E814F8158850F94620D9E
:10F5C0005B016C01C201B101A40193010F94620DB2
:10F5D0009B01AC01C601B5010F94EC096B8F7C8FC8
:10F5E0008D8F9E8FC801B701A40193010F94620D06
:10F5F0007B018C01C201B1012D813E814F81588573
:10F600000F94620D9B01AC01C801B7010F94EB0987
:10F610006F8B788F898F9A8F992469817A818B81FA
:10F620009C812D853E854F8558890F94EC0969830F
:10F630007A838B839C8300D00F92CDB6DEB608947C
:10F64000C11CD11C6BA17CA18DA19EA12B8D3C8DD9
:10F650004D8D5E8D0F94EC097B018C016F8D78A12F
:10F6600089A19AA12F89388D498D5A8D0F94EC0963
:10F670009B01AC0180E89FE4A3ECB7E4F601808332
:10F680009183A283B383C801B7010F2EF0E8EF2E58
:10F69000FFE4FF2EF3EC0F2FF7E41F2FF02DA980CE
:10F6A000BA80CB80DC800E94F8A92EAD3FAD2F5FE1
:10F6B0003F4F3FAF2EAF0F900F900F900F904EAD7A
:10F6C0005FAD8D899E894817590708F4EBCE00D0AD
:10F6D0000F92ADA9BEA96D917D918D919C911397CB
:10F6E00014962D913D914D915C9117971C96AD907C
:10F6F000BD90CD90DC901F970F2EF0E8EF2EFFE429
:10F70000FF2EF3EC0F2FF7E41F2FF02DEDB7FEB710
:10F71000E182F282038314830E94F8A90F900F9074
:10F720000F900F90EF960FB6F894DEBF0FBECDBFCF
:10F73000CF91DF911F910F91FF90EF90DF90CF90CD
:10F74000BF90AF909F908F907F906F905F904F9001
:10F750003F902F9008952F923F924F925F926F9219
:10F760007F928F929F92AF92BF92CF92DF92EF9251
:10F77000FF920F931F93DF93CF93CDB7DEB72F97F1
:10F780000FB6F894DEBF0FBECDBF20918A172A8333
:10F79000422F50E05B874A8785E291E0489FD00185
:10F7A000499FB00D589FB00D1124A85CBA4FB8877F
:10F7B000AF837FB7F89460918C17B0918A17B9879F
:10F7C0006B1729F06F3011F460E001C06F5F20E02B
:10F7D00030E040E050E005E211E018C0862F90E0F4
:10F7E000809FF001819FF00D909FF00D1124E85C47
:10F7F000FA4F83819481A581B6816F3011F460E066
:10F8000001C06F5F280F391F4A1F5B1F283CEFEABA
:10F810003E07E0E04E07E0E05E0740F4F9856F1731
:10F82000E9F604C04A8141504A8302C025E231E032
:10F830005A815617A1F0852F90E0829FF001839F97
:10F84000F00D929FF00D1124E85CFA4F808181FD4C
:10F8500006C08A81882331F79FE09A83E9CFAA8185
:10F86000B985AB17B9F02A2F30E085E291E0289FE7
:10F87000F001299FF00D389FF00D1124E85CFA4F3C
:10F88000808181FF07C0AF3011F41A8203C0EA8182
:10F89000EF5FEA83FA812985F217F9F485E291E0B6
:10F8A0004A855B85489F8001499F100D589F100D28
:10F8B0001124085C1A4FD80111968C911197806819
:10F8C00011968C9311977FBF8C9184608C938F815C
:10F8D00098850E943C6CF801CEC63A81232F30E017
:10F8E0003C832B8385E291E0289FF001299FF00D56
:10F8F000389FF00D1124E85CFA4F81818068818384
:10F900007FBF4985442311F4EFE002C0E985E1504F
:10F910002E2E33248091281881FF97C085E291E034
:10F92000289EB001299E700D389E700D1124685CD0
:10F930007A4FDB0118962C91EA85FB85E89FD00170
:10F94000E99FB00DF89FB00D1124A85CBA4F18962E
:10F950004C911897922F991F9927991F842F881FD0
:10F960008827881F981709F470C0842F90E030E032
:10F97000822B932B80739070892B09F466C0FB0156
:10F980008081826080838C9184608C93E35BFF4FE5
:10F99000D080E180F2800381FD01E75BFF4FC080F2
:10F9A000B180A28093806D2D7E2D8F2D902F2C2DD8
:10F9B0003B2D4A2D592D0F94B20A87FD04C0DC2C33
:10F9C000EB2CFA2C092D25E231E0229EF001239E3A
:10F9D000F00D329EF00D1124E85CFA4FEB5BFF4F07
:10F9E0008D2D9E2DAF2DB02F80839183A283B38365
:10F9F0004A855B85C901489F9001499F300D589FFA
:10FA0000300D1124285C3A4F275B3F4F4D2D5E2D62
:10FA10006F2D702FD9014D935D936D937C93139748
:10FA20002954304038968D2D9E2DAF2DB02F8083D8
:10FA30009183A283B383ED54F04080818E7F8083D5
:10FA4000F90180818E7F80834EC185E291E0289EFE
:10FA50004001299E900C389E900C112428E335E03B
:10FA6000820E931E4AE550E0840E951EEA85FB85C2
:10FA7000E89FD001E99FB00DF89FB00D1124A20FAF
:10FA8000B31FA65ABF4FBF87AE87D4019C91E6EA49
:10FA9000FFEF8E0E9F1EAE85BF858C91AA55B0409C
:10FAA000BF87AE879817E1F4F40141AC52AC63AC68
:10FAB00074ACD996CD90DD90ED90FC90DC97C301AD
:10FAC000B201A70196010F94C00CF401EB5BFF4F4C
:10FAD00018160CF404C1408251826282738203C101
:10FAE000AE85BF8599966D917D918D919C919C97E6
:10FAF000F40121A532A543A554A50F94EB097B0180
:10FB00008C01AE85BF859D966D917D918D919C9167
:10FB1000D097F40125A536A547A550A90F94EB0968
:10FB20005B016C01AE85BF85D1966D917D918D9104
:10FB30009C91D497F40121A932A943A954A90F9407
:10FB4000EB093B014C01C801B701A80197010F94D3
:10FB5000620D7B018C01C601B501A60195010F94D0
:10FB6000620D9B01AC01C801B7010F94EC097B0148
:10FB70008C01C401B301A40193010F94620D9B0198
:10FB8000AC01C801B7010F94EC090F94CF0D4B01E4
:10FB90005C01C0900D19D0900E19E0900F19F090F3
:10FBA0001019A70196010F94C00C18165CF00F2EC7
:10FBB000F0E04F2EF0E05F2EF0E86F2EFFE37F2E97
:10FBC000F02D08C0C701B601A50194010F94B90A30
:10FBD0002B013C0185E291E02A853B85289FD001DD
:10FBE000299FB00D389FB00D1124A85CBA4F289EF4
:10FBF000F001299EF00D389EF00D1124E85CFA4FBB
:10FC0000D5966D917D918D919C91D89725A936A916
:10FC100047A950AD0F94EB094B015C01E894B7F88C
:10FC2000E0915603F0915703C788D08CE18CF28C99
:10FC3000C501B401A70196010F94C00C181684F4F5
:10FC4000C701B601A50194010F94B90A6B017C01AB
:10FC5000C301B201A70196010F94B20A882314F4DC
:10FC60007301620105E211E0209EF001219EF00D7A
:10FC7000309EF00D1124E85CFA4FC701B60121ADAA
:10FC800032AD43AD54AD0F94620D6B017C014A85DA
:10FC90005B85409FF001419FF00D509FF00D1124B6
:10FCA000E85CFA4F01ADB2ACA3AC94AC202F3B2D75
:10FCB0004A2D592D0F94B20A87FD06C0802F9B2D27
:10FCC000AA2DB92D6C017D0185E291E0289EF001FD
:10FCD000299EF00D389EF00D1124E358FA4FC08292
:10FCE000D182E282F38230E085E291E0289EF00149
:10FCF000299EF00D389EF00D1124E85CFA4F8085A6
:10FD0000807F803809F431E020E085E291E0AA8527
:10FD1000BB85A89FF001A99FF00DB89FF00D11249D
:10FD2000E85CFA4F8085807F803809F421E0321743
:10FD300051F105E211E0209EF001219EF00D309E70
:10FD4000F00D1124E85CFA4F8081826080832A855F
:10FD50003B85209FF001219FF00D309FF00D112475
:10FD6000E85CFA4F8081846080838F8198850E944F
:10FD70003C6C4B815C81409FF001419FF00D509F96
:10FD8000F00D112476C45985252F30E085E291E0ED
:10FD9000289FD001299FB00D389FB00D1124A85C79
:10FDA000BA4FA35BBF4FAD90BD90CD90DC90139741
:10FDB000AD54B040BF87AE875983A5E22A2EA1E09B
:10FDC0003A2EB981BB2319F4EFE0E98303C0F9812E
:10FDD000F150F9832981422E5524429C7001439CA5
:10FDE000F00C529CF00C112448E355E0E40EF51E93
:10FDF0008AE590E0E80EF91EAE85BF85A65ABF4F92
:10FE0000F701908126EA3FEFE20EF31E8C91AA558E
:10FE1000B040BF87AE87981709F059C0F701EB5B78
:10FE2000FF4FC601B50120813181428153810F947A
:10FE3000B20A882309F04BC04E855F854F5A5F4F49
:10FE4000DA017C9011968C90119712969C901297E3
:10FE500013960C911397A155B040BF87AE87F70159
:10FE6000E35BFF4FA082B182C282D382672D782DDF
:10FE7000892D902FA60195010F94B20A882334F49E
:10FE8000D601C5017A2C892E9A2E0B2FEE85FF857F
:10FE9000E75BFF4F872D982DA92DB02F808391838D
:10FEA000A283B383E954F040FF87EE87429CF001C0
:10FEB000439CF00D529CF00D1124E85CFA4F8081B8
:10FEC0008E7F8083AE85BF858C918E7F8C93EE85EF
:10FED000FF85818181FF05C061AC72AC83AC94ACBD
:10FEE00014C0C601B501A60195010F94620DEE85FF
:10FEF000FF85EF5BFF4F20813181428153810F9459
:10FF0000EC090F94CF0D3B014C01429C7001439CC6
:10FF1000F00C529CF00C112428E335E0E20EF31EA5
:10FF200045E450E0E40EF51ED7010C911196CC90FB
:10FF300011971296BC9012971396AC90EBEBFFEFD3
:10FF4000EE0EFF1EB301C401202F3C2D4B2D5A2D68
:10FF50000F94C00C88230CF498C0F701E35BFF4FAB
:10FF60006081718182819381202F3C2D4B2D5A2DF0
:10FF70000F94B20A882381F1D7018C918E7F8C93E4
:10FF8000F701EF5AFF4F9080818072806380D02EFE
:10FF9000EC2CFB2C0A2D692D782D872D962D2D2DDF
:10FFA0003C2D4B2D5A2D0F94B20A87FD04C0D92C3D
:10FFB000E82CF72C062D429CF001439CF00D529C3E
:10FFC000F00D1124EB57FA4F8D2D9E2DAF2DB02F34
:10FFD00080839183A283B383429CF001439CF00D04
:10FFE000529CF00D1124E358FA4FD080E180F2804A
:10FFF0000381EE85FF85E75BFF4F60817181828120
:020000021000EC
:1000000093812D2D3E2D4F2D502F0F94B20A882312
:1000100071F1EE85FF85EF5AFF4FC080B180A2805D
:100020009380E155F040FF87EE876C2D7B2D8A2D64
:10003000992D2D2D3E2D4F2D502F0F94B20A87FD57
:1000400004C0DC2CEB2CFA2C092D2E853F85275B78
:100050003F4F8D2D9E2DAF2DB02FF90180839183C1
:10006000A283B383E954F04080818E7F8083429CD9
:10007000F001439CF00D529CF00D1124EB57FA4F08
:10008000A080B180C280D38063C02E853F852F5A67
:100090003F4FD901DC901196EC9011971296FC908D
:1000A000129713960C911397A155B040BF87AE8756
:1000B0006D2D7E2D8F2D902F9301A4010F94B20AE8
:1000C000882324F4D62CE72CF82C092DEE85FF8507
:1000D000E75BFF4F8D2D9E2DAF2DB02F8083918339
:1000E000A283B383E954F040FF87EE87429CF0017E
:1000F000439CF00D529CF00D1124E757FA4FA0805D
:10010000B180C280D380B301C401A60195010F94D0
:10011000B20A87FD04C0C301D4015C016D01429C99
:10012000F001439CF00D529CF00D1124E85CFA4F55
:10013000E35BFF4FA082B182C282D382ED54F040D4
:1001400080818E7F8083AE85BF858C918E7F8C93DE
:10015000B981EA81BE1761F0429C9001439C300D49
:10016000529C300D1124285C3A4F3F872E8729CEB0
:1001700085E291E0AB81BC81A89FA001A99F500DB1
:10018000B89F500D1124485C5A4F475B5F4FFA01EE
:1001900080809180A280B380E954F040FF87EE8791
:1001A00019811F3011F410E001C01F5F212F30E0D2
:1001B0003E832D8345E251E0249F1001259F300CA2
:1001C000349F300C112488E395E0280E391EAE854B
:1001D000BF85A65ABF4FEAE5F0E02E0E3F1E9C9168
:1001E000AA55B040BF87AE87D1018C91E6EAFFEFF8
:1001F0002E0E3F1E981781F5FDE4EF2EF12C2E8573
:100200003F85E20EF31EF901EB5BFF4FD7016D91C5
:100210007D918D919C9120813181428153810F94F8
:10022000B20A8823C9F4EE85FF85E75BFF4FFF879D
:10023000EE87DF0180829182A282B382A954B0400E
:10024000F70180809180A280B3808C9182608C9332
:10025000D1018C918460F0C0EE85FF85818181FFA2
:1002600005C051AC62AC73AC04AD16C0C501B4019D
:10027000A50194010F94620DEE85FF85EF5BFF4FA2
:1002800020813181428153810F94EC090F94CF0D6D
:10029000562E672E782E092F2E853F85235B3F4FE4
:1002A0003D872C87652D762D872D902FD9012D9197
:1002B0003D914D915C910F94C00CEE85FF85EF5AF6
:1002C000FF4F18160CF0BAC0C080D180E280F380D6
:1002D000C501B401A70196010F94B20A87FD03C0BE
:1002E0007501640118C0C701B601A70196010F94FA
:1002F000620DEE85FF85EF5BFF4F208131814281EA
:1003000053810F94EC090F94CF0DEC85FD8560832C
:100310007183828393832E853F85275B3F4FD9016D
:10032000CD92DD92ED92FD92DC901196EC901197BA
:100330001296FC90129713960C9113971897CC90E5
:100340001196BC9011971296AC90129713969C90B0
:100350001397A554B040BF87AE876D2D7E2D8F2D8E
:10036000902F2C2D3B2D4A2D592D0F94B20A87FD2D
:1003700004C0DC2CEB2CFA2C092D2D813E8145E2AA
:1003800051E0249FF001259FF00D349FF00D1124C2
:10039000E757FA4F80809180A280B3806D2D7E2D2B
:1003A0008F2D902FA50194010F94B20A87FD06C0EE
:1003B0008D2D9E2DAF2DB02F4C015D018D819E8125
:1003C000A5E2B1E08A9F70018B9FF00C9A9FF00C20
:1003D0001124E8E3F5E0EE0EFF1E29E430E0E20E22
:1003E000F31ED7018D929D92AD92BC921397E7EBCD
:1003F000FFEFEE0EFF1EEE85FF85E35BFF4FAE8540
:10040000BF85AB5BBF4F60817181828193812D91EC
:100410003D914D915C910F94B20A882349F4AE85C9
:10042000BF858C9182608C93F7018081846080838A
:10043000AE85BF858C918E7F8C93AFC0AE85BF8516
:100440008C9186608E7F8C93C080D180E280F38017
:10045000C701B601A50194010F94C00C18161CF039
:100460007501640116C0C701B601A70196010F947A
:10047000620DEE85FF85EF5BFF4F20813181428168
:1004800053810F94EC090F94CF0D562E672E782EC2
:10049000092FEE85FF85E75BFF4FDF01C082D18228
:1004A000E282F3821896FC901196EC9011971296C6
:1004B000DC9012971396CC901397A155B040BF874C
:1004C000AE876F2D7E2D8D2D9C2D252D362D472D04
:1004D000502F0F94B20A87FD04C05F2C6E2C7D2C28
:1004E0000C2DEE85FF85E35BFF4FFF87EE87852DA3
:1004F000962DA72DB02F80839183A283B383389745
:10050000F080E180D280C380652D762D872D902FDD
:100510002F2D3E2D4D2D5C2D0F94B20A87FD04C06A
:100520005F2C6E2C7D2C0C2D2D813E8145E251E0FF
:10053000249FF001259FF00D349FF00D1124E75703
:10054000FA4F80809180A280B380652D762D872D13
:10055000902FA50194010F94B20A87FD06C0852D46
:10056000962DA72DB02F4C015D018D819E81A5E2B6
:10057000B1E08A9FF0018B9FF00D9A9FF00D11243E
:10058000E85CFA4FE75BFF4F80829182A282B382E0
:10059000E954F040808184608083B9851B1719F08D
:1005A0003F862E86FECDF101EF5AFF4F0081F1808C
:1005B000E280D380602F7F2D8E2D9D2DA50194018B
:1005C0000F94B20A87FD06C0802F9F2DAE2DBD2D42
:1005D0004C015D01F101E75BFF4F80829182A282B5
:1005E000B382E5E2EE2EE1E0FE2EE9818E2F90E06F
:1005F0008E9D80018F9D100D9E9D100D1124085C15
:100600001A4FC8010E943C6C2FB7F894D80111967C
:100610008C9111978F7711968C93B981BF3011F41B
:10062000198203C0E981EF5FE983F9818F2F90E0A0
:100630008E9DF0018F9DF00D9E9DF00D1124E85CC4
:10064000FA4F8181806881832FBF80918A17298129
:10065000281759F68F8198850E943C6C85E291E0BD
:100660004A855B85489FF001499FF00D589FF00D2A
:100670001124E85CFA4F81818F7781832F960FB622
:10068000F894DEBF0FBECDBFCF91DF911F910F91C8
:10069000FF90EF90DF90CF90BF90AF909F908F90A2
:1006A0007F906F905F904F903F902F9008952F9282
:1006B0003F924F925F926F927F928F929F92AF92F2
:1006C000BF92CF92DF92EF92FF920F931F93DF932F
:1006D000CF93CDB7DEB7A6970FB6F894DEBF0FBEA7
:1006E000CDBF3C0179A368A34AA325E530E0620EA3
:1006F000731ED301AD90BD90CD90DC90EBEAFFEF7F
:100700006E0E7F1ED30118968C918073209105196F
:100710003091061940910719509108198823D9F092
:100720009090CD188090CE185090CF184090D0184F
:10073000C901DA017C018D01692D782D852D942D5B
:10074000A80197010F94B20A87FD09C0892D982D41
:10075000A52DB42D02C0C901DA017C018D01C601AD
:10076000B50120E034E244E75BE40F94620DA80198
:1007700097010F94B90A1B012C018091281890E071
:1007800036E0969587953A95E1F7B82FB170BB8F13
:1007900080918B178A30C0F5C201B10120E034E2AC
:1007A00044E758E40F94B20A882374F5E0908B175D
:1007B00060E074E284E798E4A20191010F94EB09F0
:1007C00020E030E040E450E40F94620D5B016C01E6
:1007D000FF240894E11CF11C0027F7FC0095102F62
:1007E000C801B7010F94540B9B01AC01C601B501C0
:1007F0000F94B90A9B01AC01C201B1010F94EC093D
:100800001B012C01E1E0EB8FC201B1010F94210B20
:10081000D30113966D937D938D939C93169785E2E8
:100820009CE10E945FD6F301EF5DFE4F6081718114
:10083000828193810F94540B5B016C01F3018084DE
:10084000982C84FE28C0A8A1B9A16D917D918D91AD
:100850009C919F7720E034E244E75BE40F94620DC3
:100860007B018C01C601B5012091F2023091F302A7
:100870004091F4025091F5020F94620D9B01AC017E
:10088000C801B7010F94B90A0F94210B69837A83C9
:100890008B839C8304C019821A821B821C8295FE62
:1008A00028C0E8A1F9A164817581868197819F772D
:1008B00020E034E244E75BE40F94620D7B018C019D
:1008C000C601B5012091F6023091F7024091F8027D
:1008D0005091F9020F94620D9B01AC01C801B70160
:1008E0000F94B90A0F94210B6D837E838F839887B1
:1008F00004C01D821E821F82188696FE2AC0A8A1EF
:10090000B9A118966D917D918D919C911B979F77C0
:1009100020E034E244E75BE40F94620D7B018C013C
:10092000C601B5012091FA023091FB024091FC0210
:100930005091FD020F94620D9B01AC01C801B701FB
:100940000F94B90A0F94210B69877A878B879C874C
:1009500004C019861A861B861C8687FE28C0E8A15B
:10096000F9A164857585868597859F7720E034E2B7
:1009700044E75BE40F94620D7B018C01C601B50175
:100980002091FE023091FF0240910003509101033B
:100990000F94620D9B01AC01C801B7010F94B90A15
:1009A0000F94210B6D877E878F87988B04C01D86DF
:1009B0001E861F86188AA8A1B9A15096ED90FD90B9
:1009C0000D911C915397C801B70120E030E040E041
:1009D00050E00F94C00CE89417F98823ACF0C801DC
:1009E000B70120E034E244E75BE40F94620D7B0141
:1009F0008C01C601B5012091FA023091FB024091B1
:100A0000FC025091FD0214C0C801B70120E034E29D
:100A100044E75BE40F94620D7B018C01C601B501D4
:100A20002091FE023091FF0240910003509101039A
:100A30000F94620D9B01AC01C801B7010F94B90A74
:100A40000F94210B698B7A8B8B8B9C8B19890A896C
:100A5000FB88EC88C201B101A60195010F94B90A87
:100A60000F94210B5B016C01212F302F4F2D5E2D38
:100A7000C901DA01BC01CD016631B2E07B07B0E00B
:100A80008B07B0E09B0724F466E172E080E090E021
:100A90006D8B7E8B8F8B988F6A157B058C059D05E2
:100AA00024F4AD8ABE8ACF8AD88EE9EFF0E06E0ECC
:100AB0007F1E8D899E89AF89B88DF30180839183D4
:100AC000A283B38327E03FEF620E731EBC01CD010A
:100AD0000F94540B7B018C01F301EF5DFE4F60819D
:100AE0007181828193810F94540B9B01AC01C801E9
:100AF000B7010F94620D6B017C0160E074E284E742
:100B00009BE4A70196010F94B90A1B012C01D301A4
:100B100018968C911897082F10E084FF2EC0199614
:100B20006D917D918D919C911C970F94540B9B011D
:100B3000AC01C701B6010F94B90A0F94210B698368
:100B40007A838B839C83C201B101E8A1F9A1208142
:100B50003181428153810F94620DD30199966D9337
:100B60007D938D939C939C970171107000311105BA
:100B700069F4DC01CB01B05804C080E090E0A0E053
:100B8000B0E0F30181A792A7A3A7B4A7D301189659
:100B90008C911897082F10E085FF2EC01D966D913F
:100BA0007D918D919C9150970F94540B9B01AC01BA
:100BB000C701B6010F94B90A0F94210B6D837E8390
:100BC0008F839887C201B101E8A1F9A12481358101
:100BD000468157810F94620DD3019D966D937D934D
:100BE0008D939C93D097027210700032110569F4B6
:100BF000DC01CB01B05804C080E090E0A0E0B0E0A0
:100C0000F30185A796A7A7A7B0ABD30118968C913F
:100C10001897082F10E086FF2EC051966D917D9198
:100C20008D919C9154970F94540B9B01AC01C7017B
:100C3000B6010F94B90A0F94210B69877A878B87C5
:100C40009C87C201B101E8A1F9A1208531854285C7
:100C500053850F94620DD301D1966D937D938D933F
:100C60009C93D497047410700034110569F4DC016E
:100C7000CB01B05804C080E090E0A0E0B0E0F30108
:100C800081AB92ABA3ABB4ABD30118961C91189770
:100C900017FF30C055966D917D918D919C9158971D
:100CA0000F94540B9B01AC01C701B6010F94B90A14
:100CB0000F94210B6D877E878F87988BC201B101BE
:100CC000E8A1F9A124853585468557850F94620DE5
:100CD000D301D5966D937D938D939C93D897187877
:100CE000103841F4DC01CB01B058F30185AB96AB71
:100CF000A7ABB0AF8D899E89AF89B88D898B9A8B50
:100D0000AB8BBC8BF301EB5AFF4F60817181828109
:100D10009381A20191010F94620DD301D9966D9335
:100D20007D938D939C93DC9718968C91E82FF0E03F
:100D3000FA8FE98FCF01887890708838910529F073
:100D400020EC37E13F8F2E8F04C080EB97E19F8F1F
:100D50008E8F29EA922E9FE5292E83E6382E08E50C
:100D6000802E44245524AA24BB2480E190E0042C46
:100D700002C0880F991F0A94E2F7A98DBA8D8A23C1
:100D80009B23892B51F1E1E0F0E0EC0FFD1FEA0D10
:100D9000FB1D60817181828193810F94540B7B01D3
:100DA0008C01EE8DFF8DEA0DFB1D608171818281CA
:100DB00093810F94520B9B01AC01C801B7010F94B2
:100DC000620D6B017C01692D722D832D982DA70179
:100DD00096010F94B20A882334F4892D922DA32D05
:100DE000B82D6C017D010894411C511CE4E0F0E039
:100DF000AE0EBF1EF4E04F16510439F0D701C60104
:100E00009C2C292E3A2E8B2EB0CF21E231E0620E9F
:100E1000731EF30180819181A281B3812FED3EEF9A
:100E2000620E731EB595A79597958795F30185A3D7
:100E300096A3A7A3B0A760E070E080E89FE321AD90
:100E400032AD43AD54AD0F94B90A2DE330E0620EDC
:100E5000731ED3016D937D938D939C931397E3EC55
:100E6000FFEF6E0E7F1ED3011296EC91F0E0EE0FB5
:100E7000FF1FEE0FFF1FEC0FFD1F61817281838149
:100E800094810F94540B9B01AC01C701B6010F94E0
:100E9000B90A0F94260BE1E0F1E06E0E7F1ED3013C
:100EA0006D937D938D939D933D010F94520B20E0A4
:100EB00030E040E858E40F94620D20E034E244E76B
:100EC0005BE40F94B90A0F94260BF30160837183DE
:100ED000828393832BEF3EEF620E731E83010F5BC1
:100EE0001F4F85E590E0680E791ED3012D913D914D
:100EF0004D915C91EBEAFFEF6E0E7F1ECA01B901C6
:100F00000F94EC09A70196010F94620DD301D996B5
:100F10002D913D914D915C91DC970F94620D20E0F5
:100F200034E244E75BE40F94B90AF801608371830B
:100F30008283938360910D1970910E1980910F191E
:100F40009091101920E030E040E05FE30F94620DD3
:100F50007B018C01D30118968C9187FF3AC0807772
:100F6000E0915603F0915703882331F16789708D22
:100F7000818D928D20E030E040E05FE30F94620DC0
:100F8000F30121AD32AD43AD54AD0F94620DD301E9
:100F9000D5962D913D914D915C91D8975F770F94A7
:100FA000B90A5B016C01C801B701A60195010F9454
:100FB000B20A87FD0EC00FC06789708D818D928D3A
:100FC00020E030E040E05FE30F94620D5B016C01D4
:100FD00002C057016801F3018281823048F4E09039
:100FE000CD18F090CE180091CF181091D0180AC0EB
:100FF000823081F4E090D118F090D2180091D3188B
:101000001091D418C801B701A60195010F94B20A36
:10101000882314F486017501D301D996DC90D99701
:10102000DA96CC90DA97DB96BC90DB97DC96AC90A6
:10103000C801B7012D2D3C2D4B2D5A2D0F94B20A0E
:1010400087FD06C08D2D9C2DAB2DBA2D7C018D0109
:10105000E1E5F0E06E0E7F1ED301ED92FD920D935F
:101060001C931397F30112930293F292E292DF0121
:101070001E930E93FE92EE923D01E7EBFFEF6E0E94
:101080007F1ED301D996AD90BD90CD90DC90DC97BA
:10109000C801B701A80197010F94620DF301EF5B3E
:1010A000FF4F20813181428153810F94EC097B01F4
:1010B0008C01C601B501A60195010F94620D9B013B
:1010C000AC01C801B7010F94C00C882324F0F301D0
:1010D00081818260818329EF30E0620E731ED3012B
:1010E0002D913D914D915C9160E074E284EF90E030
:1010F0000F948B0E3D8F2C8FE0E1F0E06E0E7F1E83
:10110000D3012D933C93E7EFFEEF6E0E7F1ED301CC
:1011100018969C91892F807711F097FDC0C0EFE061
:10112000F1E06E0E7F1ED3011D921D921D921D9245
:101130003D01FD0110821182128213822CE030E009
:10114000620E731ED3011D921C92E1EEFEEF6E0E35
:101150007F1E38C0F0922B05E0922A058BA19CA13E
:10116000ADA1BEA180932E0590932F05A0933005CD
:10117000B093310560912C0570912D05882777FD7E
:101180008095982F0F94540B9B01AC01C201B101C3
:101190000F94C00C1816B4F4C201B1010F94210BC6
:1011A00070932D0560932C05F30185A996A9A7A935
:1011B000B0ADBF7780932E0590932F05A093300597
:1011C000B093310585E29CE10E945FD60E94AB7B23
:1011D00029EF30E0620E731EF30180819181A281BC
:1011E000B38127E03FEF620E731E8F5C9740A040F3
:1011F000B04018F08B8D882329F084E0D301179636
:101200008C9315C081E0F301878321E231E0620E07
:10121000731EF30180819181A281B3812FED3EEF96
:10122000620E731EF30185A396A3A7A3B0A7FAA12C
:10123000FF2331F086E490E09093370580933605E4
:1012400080918A178F5F80938A17803110F01092F7
:101250008A1780912A18806180932A189FB7F89482
:1012600080918B178F5F80938B179FBFA6960FB6C9
:10127000F894DEBF0FBECDBFCF91DF911F910F91CC
:10128000FF90EF90DF90CF90BF90AF909F908F90A6
:101290007F906F905F904F903F902F900895D30173
:1012A000D596AD90BD90CD90DC90D897D601C50174
:1012B000BF778BA39CA3ADA3BEA380905603909051
:1012C0005703BC01CD01D40199962D913D914D91CB
:1012D0005C919C970F94620D2FE632E143E85AE34C
:1012E0000F94620D2091EE023091EF024091F002D6
:1012F0005091F1020F94620D1B012C01EFE1F1E01E
:101300006E0E7F1E20E030E040E857E40F94620D3F
:101310007B018C012C8D3D8DB90180E090E00F9414
:10132000520B9B01AC01C801B7010F94B90A0F948D
:10133000260BD3016D937C93F40165A176A187A15F
:1013400090A520E030E040E857E40F94620DA6013C
:1013500095010F94620DA60195010F94620D0F94F3
:10136000210B7B018C0124EF3FEF620E731ED30132
:101370006D937D938D939C931397EDEEFEEF6E0E20
:101380007F1E2C8D3D8D229FB001339FC001239F76
:101390002227700D811D921F700D811D921F112437
:1013A000FFE0CF2EF1E0DF2EC60CD71C21E031E0AC
:1013B000620E731ED3012D913D914D915C91EFEF23
:1013C000FEEF6E0E7F1E220F331F441F551F0F941A
:1013D0008B0EC801B7010F94AD0ED6012D933D932E
:1013E0004D935C93139778011127F7FC1095012F0B
:1013F00080912A0590912B05AA2797FDA095BA2FD9
:101400008E159F05A007B1070CF4A4CEB3CE4F9262
:101410005F926F927F928F929F92AF92BF92CF9284
:10142000DF92EF92FF920F931F93CF93DF93EC0124
:101430002B01809128182091791830917A184091C9
:101440007B1850917C18A0907518B0907618C090B9
:101450007718D0907818688079808A809B8087FF81
:1014600035C18C819D81AE81BF81281B390B4A0B10
:101470005B0BCA01B9010F94540B9B01AC010F9493
:10148000620D9B01AC0160916518709166188091A6
:101490006718909168180F94EB097B018C01A618CE
:1014A000B708C808D908C601B5010F94540B9B01B1
:1014B000AC010F94620D9B01AC01C801B7010F9400
:1014C000EB097B018C0120E030E040E050E00F941C
:1014D000C00C88230CF4D1C1C801B7010F94CF0D03
:1014E00020E030E040E05FE30F94EC097B018C01E9
:1014F000688579858A859B850F94540B9B01AC0187
:10150000C801B7010F94EC090F948F0B0F94210BB6
:10151000F20160837183828393836091811870915B
:10152000821880918318909184182C813D814E817E
:101530005F81621B730B840B950B0F94540B9B0103
:10154000AC010F94620D9B01AC0160916918709120
:101550006A1880916B1890916C180F94EB097B01BD
:101560008C0160917D1870917E1880917F18909108
:101570008018288139814A815B81621B730B840B3F
:10158000950B0F94540B9B01AC010F94620D9B01C2
:10159000AC01C801B7010F94EB097B018C0120E07D
:1015A00030E040E050E00F94C00C88230CF465C19B
:1015B000C801B7010F94CF0D20E030E040E05FE3B9
:1015C0000F94EC097B018C01688579858A859B8560
:1015D0000F94540B9B01AC01C801B7010F94EC09A7
:1015E0000F948F0B0F94210BF20164837583868314
:1015F00097836091891870918A1880918B189091C7
:101600008C182C813D814E815F81621B730B840B92
:10161000950B0F94540B9B01AC010F94620D9B0131
:10162000AC0160916D1870916E1880916F18909157
:1016300070180F94EB097B018C01609185187091F3
:1016400086188091871890918818288139814A815D
:101650005B81621B730B840B950B0F94540B9B01E6
:10166000AC010F94620D9B01AC01C801B7010F944E
:10167000EB097B018C0120E030E040E050E00F946A
:10168000C00C88230CF4F9C0C801B7010F94CF0D2A
:1016900020E030E040E05FE30F94EC097B018C0137
:1016A000688579858A859B850F94540B9B01AC01D5
:1016B000C801B7010F94EC090F948F0B0F94210B05
:1016C000F2016087718782879387D5C08C819D8165
:1016D000AE81BF81281B390B4A0B5B0BCA01B901D4
:1016E0000F94380EE0906518F09066180091671816
:1016F00010916818E61AF70A080B190BA601950154
:101700002619370948095909CA01B9010F94380E39
:10171000E61AF70A080B190B17FDAFC0C801B7018D
:101720000E940266A0E0B0E0288539854A855B8585
:10173000820F931FA41FB51FF20180839183A283A0
:10174000B383209181183091821840918318509171
:1017500084188C819D81AE81BF81281B390B4A0B77
:101760005B0BCA01B9010F94380EE0906918F09034
:101770006A1800916B1810916C18E61AF70A080B9A
:10178000190B20917D1830917E1840917F1850914F
:10179000801888819981AA81BB81281B390B4A0B4B
:1017A0005B0BCA01B9010F94380EE61AF70A080B51
:1017B000190B17FD62C0C801B7010E940266A0E0C4
:1017C000B0E0288539854A855B85820F931FA41F69
:1017D000B51FF20184839583A683B783209189186E
:1017E00030918A1840918B1850918C188C819D8172
:1017F000AE81BF81281B390B4A0B5B0BCA01B901B3
:101800000F94380EE0906D18F0906E1800916F18DC
:1018100010917018E61AF70A080B190B2091851819
:101820003091861840918718509188188881998145
:10183000AA81BB81281B390B4A0B5B0BCA01B9017A
:101840000F94380EE61AF70A080B190B17FD15C08E
:10185000C801B7010E940266A0E0B0E02885398582
:101860004A855B85820F931FA41FB51FF2018087F5
:101870009187A287B38781E001C080E0DF91CF919B
:101880001F910F91FF90EF90DF90CF90BF90AF909E
:101890009F908F907F906F905F904F9008952F92C0
:1018A0003F924F925F926F927F928F929F92AF92F0
:1018B000BF92CF92DF92EF92FF920F931F93DF932D
:1018C000CF93CDB7DEB7C85AD0400FB6F894DEBF7D
:1018D0000FBECDBFCC56DF4F8883C459D040CB5606
:1018E000DF4F6883C559D040CA56DF4F4883C65979
:1018F000D04069E1662E712C6C0E7D1E430155248B
:10190000AA24BB2459E5252E312C2C0E3D1EF501B1
:10191000E45FF74E95012C51384E80819181A28170
:10192000B381F9012081318142815381821B930B64
:10193000A40BB50BF40180839183A283B383F3E0FE
:101940005F1639F5C0900B19D0900C1924E6C21619
:10195000D104F9F06DA17EA18FA198A50F94540B2D
:101960007B018C01B60180E090E00F94520B9B014B
:10197000AC01C801B7010F94620D2AE037ED43E2D4
:101980005CE30F94620D0F94210B6DA37EA38FA3D4
:1019900098A781010A0D1B1DD4016D917D918D9138
:1019A0009D914D010F94540BF501E056F84E2081A6
:1019B0003181428153810F94620D9F77F8016083DA
:1019C000718382839383539424E030E0A20EB31E8C
:1019D00034E0531609F09BCF60911F1970912019C4
:1019E0008091211990912219D1011C962D913D9140
:1019F0004D915C911F970F94EC0960931F197093A0
:101A000020198093211990932219FE01B996C1578C
:101A1000DF4F1882CF58D04060E070E041E0E42E04
:101A2000F12C00E110E0D3012D913D914D915C919D
:101A300057FD17C02083318342835383C701062E8D
:101A400002C0880F991F0A94E2F7C157DF4FB8818F
:101A5000CF58D040B82BC157DF4FB883CF58D040B4
:101A60000BC088279927DC01821B930BA40BB50BB5
:101A700080839183A283B38380819181A281B3818A
:101A80000097A105B10591F0C801062E02C0880F8C
:101A9000991F0A94E2F7C157DF4F2881CF58D040F1
:101AA000282BC157DF4F2883CF58D0406F5F7F4F1F
:101AB00044E050E0640E751E34966430710509F000
:101AC000B2CFC157DF4F5881CF58D040052F10E01B
:101AD000C80180779070892B09F473C054FD0BC046
:101AE0000F2EF0E0CF2EF0E0DF2EF0E0EF2EF0E052
:101AF000FF2EF02D0DC0FE01E75AFF4F20813181EE
:101B000042815381CA01B9010F94620D6B017C01BE
:101B100005FF13C0FE01E75AFF4F2481358146813E
:101B20005781CA01B9010F94620D9B01AC01C70135
:101B3000B6010F94EC096B017C0106FF13C0FE0196
:101B4000E75AFF4F2085318542855385CA01B90187
:101B50000F94620D9B01AC01C701B6010F94EC0913
:101B60006B017C01C701B6010F94CF0DF62EE72E55
:101B7000D82EC92EFE01E75AFF4F84859585A6858C
:101B8000B7859C01AD015F77C057DF4F288339834C
:101B90004A835B83C059D0406F2D7E2D8D2D9C2DA7
:101BA0000F94B20A87FD35C08F2D9E2DAD2DBC2D13
:101BB000C057DF4F88839983AA83BB83C059D04025
:101BC00028C0C157DF4F3881CF58D04037FD01C002
:101BD0008BC7CDA0DEA0EFA0F8A4809128188E7F3F
:101BE0008093281881E00E949278CB56DF4F88813D
:101BF000C559D04061E00E94C46D80918A17882E3B
:101C00009924CC56DF4F4881C459D0404423E1F495
